:020000040800F2
:10000000005000208DA90008D3A90008D5A9000838
:10001000D7A90008D9A90008DBA900080000000042
:10002000000000000000000000000000DDA9000842
:10003000DFA9000800000000E1A90008050A000887
:10004000E7A90008E9A90008EBA90008EDA9000844
:10005000EFA90008F1A90008F3A90008F5A9000814
:10006000F7A90008F9A90008FBA90008FDA90008E4
:10007000F599000801AA000803AA000805AA0008CB
:1000800007AA000809AA00080BAA00080DAA000880
:100090000FAA000811AA000813AA000815AA000850
:1000A00017AA000819AA00081BAA00081DAA000820
:1000B0006176000821AA000823AA000825AA0008E2
:1000C00027AA000829AA00082BAA00082DAA0008C0
:1000D0002FAA0008CD7400080D39000835AA0008C1
:1000E00037AA000839AA00083BAA000810B5054C39
:1000F000237833B9044B13B10448AFF300800123D4
:10010000237010BDA802002000000000BCFA000807
:1001100008B5064B1BB106480649AFF300800648F8
:10012000036813B1054B03B1984708BD00000000F8
:10013000BCFA0008AC020020A80200200000000069
:10014000154B002B08BF134B9D46A3F5803A0021A9
:100150008B460F461348144A121A0AF09EFD0F4BA5
:10016000002B00D098470E4B002B00D09847002062
:10017000002104000D000D48002802D00C48AFF308
:1001800000800AF03DFD2000290007F099FB0AF0ED
:1001900023FD00BF00000800005000200000000008
:1001A00000000000A8020020183A00200000000013
:1001B0000000000070B5354D86B02C681CB10123DD
:1001C0002B6006B070BD684609F0EEFF01A809F08B
:1001D000F5FD4FF400400AF047F9112001210AF023
:1001E000AFF94FF400602023C4F201006946ADF876
:1001F00000308DF8034009F073FF4FF400700121C7
:100200000AF09EF94FF4105001264FF46023C4F217
:10021000010001A9039301948DF808408DF809406D
:1002200004948DF8146009F0A3FD4FF41050C4F24B
:10023000010005213246234609F0F2FD4FF410502B
:10024000C4F20100314609F0C3FD4FF41050C4F26E
:10025000010009F0C7FD4FF41050C4F2010009F08D
:10026000C7FD0028F7D14FF41050C4F2010009F087
:10027000C3FD4FF41050C4F2010009F0C3FD002883
:10028000F7D1034B01221A6099E700BFC802002092
:100290007C3800204FF4105008B5C4F20100012151
:1002A00009F0B4FD40F2C423C2F2000301221A6037
:1002B00008BD00BF38B50D4C054623680BB90020BA
:1002C00038BD4FF41050C4F20100022109F0F8FDCE
:1002D0000028F4D04FF41050C4F2010009F0ECFDF6
:1002E000002328802360012038BD00BFC402002005
:1002F00070B448F6396301EB4104951EC3F6E3037D
:100300000229C1EBC40183FB014348F21F54D8BF4B
:100310001546C5F2EB14D8BF013A84FB0264C91735
:10032000C1EB630128180818D51CD317043032EA32
:10033000220228BF2A46A3EB641100EBA202C3EB02
:10034000E413521842F29340D218C9F2492080FBBC
:100350000230D3178018C3EBA000C0EBC000101A06
:1003600070BC704770B40646002922D00078F0B106
:1003700000231846F25CA2F13004E4B2092CA2F189
:1003800041050DD9052DA2F161049CBFA2F13704EE
:10039000E4B205D9052C9ABFA2F15704E4B20024B7
:1003A0000133DDB204EB0010A94280B2E2D870BC88
:1003B00070470846FBE700BF4FF48050C4F20100CD
:1003C0004FF40051002209F0FDBE00BF4FF48050F1
:1003D000C4F201004FF40051012209F0F3BE00BF46
:1003E00000B583B001A809F0DFFE102001210AF05A
:1003F000A7F84FF40053ADF804304FF480500223B7
:10040000C4F2010001A98DF8063010238DF80730E1
:1004100009F066FEFFF7DAFF03B000BD00B583B058
:1004200001A809F0C1FE042001210AF089F8402347
:100430004FF40060ADF80430C4F20100482301A974
:100440008DF8073009F04CFE03B000BD4FF400609A
:10045000402108B5C4F2010009F0AEFED0F1010060
:1004600038BF002008BD00BFF0B4114A0346106831
:10047000D8B110490E68104964360D680F49013D26
:100480000C680F495E610F680E491D610968DF60E5
:1004900099600D49096859600021072C08BF0C4676
:1004A0009C610F2419621C601160F0BC704700BF92
:1004B000F4020020CC02002008030020E00200200B
:1004C000D002002004030020DC02002070B582B0BE
:1004D00001A809F069FE4FF44064082001210AF0E8
:1004E0002FF8C4F201044FF4807301A902262046BC
:1004F000ADF8043004238DF807308DF8066009F05C
:10050000EFFD01A809F050FE082001210AF018F8BB
:100510004FF40075204601A91023ADF804508DF862
:1005200006608DF8073009F0DBFD204629460122E0
:1005300009F048FE02B070BDF8B5A44C2368FF2B4B
:1005400056D04FF44060C4F201004FF4807109F0BE
:1005500033FE0546002833D0FFF72EFF2368012025
:10056000012B9A4D33D04AD3022B4DD0984B1A68A9
:10057000904200F08680974E022132682960911FD8
:100580001229186063D9052A94BF9348934806F04E
:1005900067FF934F934806F063FF002323603B6897
:1005A0000F2B00F0CC81102B6ED0FF2B3AD00133F3
:1005B0003B2B3B6000F0CE8134D90023236031E037
:1005C000FFF704FF23682846012B804DCBD1804BD9
:1005D0001A68824229D01860002814BF0322022220
:1005E0007F4B2260FF221A607A4B00221A60F8BD0E
:1005F0007D4B1A68642A19D001321A60F8BD0123B4
:100600002B60734B1860F8BD714B1A68904238D05C
:10061000704E032132682960782A186012D9704B15
:1006200000221A6000233360F8BDF8BD4FF440602B
:10063000C4F201004FF40071002209F0C3FD002351
:100640002360F8BD4A2AEDD800232B60EAE7644F07
:100650000F2A3B6834D8232B00F097813A2B00F007
:1006600085811C2B9CD1614A1268D0079FD56048B8
:1006700006F0F6FE5B4806F0F3FE002323603B68BD
:100680008EE7544B1A68B7E75A4A002313605A4A58
:100690001360564A1360594A1360594A1360594A05
:1006A0001360594A1360594A1360594A1360594AF2
:1006B0001360594A1360594A136011233B60B1E734
:1006C000A3F11102292A3FF66BAF01A151F822F0E4
:1006D00037090008A1050008A1050008A1050008C8
:1006E000310900082B090008250900081F09000826
:1006F00019090008130900080D090008FD08000881
:10070000F7080008F1080008EB080008E5080008F1
:10071000DF080008D9080008C9080008C308000855
:10072000BD080008B7080008B3080008AF080008B3
:10073000AB080008A50800089F08000899080008F1
:10074000930800088D08000887080008830800083F
:100750007F0800086D0800085B08000849080008C9
:100760003708000825080008BB070008A90700088B
:100770009707000879070008214A126812F001055E
:100780007FF415AF264806F06BFE164806F068FEAB
:1007900025603B6804E72149194A0D681068503507
:1007A00001300D601060FEE61C49154A0D681068A6
:1007B000283501300D601060F5E61849104A0D68C3
:1007C0001068143501300D601060ECE62000002048
:1007D000F0020020D802002040BD000860BD0008E3
:1007E0001C00002074DF0008D40200200C0300204D
:1007F00080BD0008F4020020E4020020EC0200208A
:1008000000030020F8020020DC0200200403002086
:10081000E0020020D002002008030020CC020020CB
:10082000C8BD00086549664A0D6810680A35013080
:100830000D601060B7E66149614A0D6810680835BF
:1008400001300D601060AEE65C495D4A0D681068CD
:10085000043501300D601060A5E65849584A0D680E
:100860001068023501300D6010609CE65349544A0F
:100870000D681068013501300D60106093E6514934
:10088000D1E75049D8E74F494D4ADFE74D494C4A37
:10089000E5E74C494A4AEBE74B49494AD6E74A491A
:1008A000474ADCE74849464AE2E7484986E747497C
:1008B000B9E74649C0E74549414AC7E74349404A85
:1008C000CDE742493E4AD3E7414A126812F001059A
:1008D0007FF46DAE3F4856E73F493D4A6FE73E49DA
:1008E0003B4AA1E73C493A4AA7E73B49384AADE7CA
:1008F0003949374AB3E73849354AB9E7374A1268C0
:1009000012F001057FF453AE35483CE73549334AD0
:100910004CE73449314A52E73249304A84E7314999
:100920002E4A8AE72F492D4A90E72E492B4A96E70F
:100930002C492A4A9CE72C4A0121116033E62B4BB3
:100940001A6822B12A4A0121116000221A6010237C
:100950003B6067E6274B204A196812689142264996
:1009600022D0204800681A6008605BE6144A1268CA
:10097000D2077FF51CAE214806F072FD204806F034
:100980006FFD00223B682A600AE6114A1268D1070F
:100990007FF50DAE0F4806F063FD194806F060FDC7
:1009A00000232B603B68FBE50E480C6800680134AF
:1009B0008442D8D10D4C01252560D4E7CC0200201B
:1009C0000003002008030020E0020020D0020020E5
:1009D000EC020020A4BD0008040300200C0300204A
:1009E00080BD0008DC020020F8020020E4020020A4
:1009F000F4020020E8020020FC020020C8BD00082C
:100A000074DF0008034B1A6812B11A68013A1A60C1
:100A1000704700BF80380020064B074A1B68012B37
:100A20001EBF064B1B68B0FBF3F010601368002B71
:100A3000FCD17047100300208038002028000020DF
:100A4000044B054A1B6803FB00F010601368002B81
:100A5000FCD170472400002080380020084B4FF460
:100A60007A711B6810F1FF3001FB03F1054A06D3D0
:100A700011601368002BFCD110F1FF30F8D27047E1
:100A80002400002080380020012810B423D0022840
:100A90002CD01C4B64221A601B4B0A221A6042F2B3
:100AA00010710320194A4EF210031468CEF20003AD
:100AB000B4FBF1F101394FF46D425960CEF20002FE
:100AC000F02182F8231000229A6007221A60104B4E
:100AD000186010BC70470B4B44F2402118600A4B61
:100AE0004FF47A721A60C0F20F01DBE7054B0A225D
:100AF0001A60054B48F2A06164221A60C0F201013D
:100B0000D0E700BF2800002024000020F4010020CE
:100B1000100300202DE9F00140F2941240F2581326
:100B200040F26011C2F20003C2F20001C2F2000200
:100B3000D2F8008093F800C05F789E780D784C78EA
:100B400040F2541040F26C0240F270038978C2F215
:100B50000002C2F20003C2F20000C0F8008082F876
:100B600000C0577096701D705C709970BDE8F00100
:100B7000704700BF40F2211008F04ABF40F25D10FC
:100B800008F046BFF8B506460F4640F2211440F281
:100B90005D1520463146013408F0C0FFAC42F8D163
:100BA00007B9F8BDBDE8F840FFF7E8BF70B540F2FF
:100BB0007002C2F200029578147856784CF2EC1369
:100BC000C0F6000382B033F8144033F8162033F82F
:100BD0001530014601A88DF804408DF805208DF8E8
:100BE0000630FFF7CFFF02B070BD00BF00B583B085
:100BF0000023014601A88DF804308DF805308DF8EA
:100C00000630FFF7BFFF03B000BD00BF0E2A30B4AF
:100C100036D81F4B0C789B5C48F6890204FB03F422
:100C2000C8F68802A2FB0452C2F3C70202700C7815
:100C300014B10AB9012202704C7848F6890204FB0B
:100C400003F4C8F68802A2FB0452C2F3C702427042
:100C50004C7814B10AB9012242708C7848F68902A6
:100C600004FB03F3C8F68802A2FB0342C2F3C702E7
:100C700082708B7813B10AB90123837030BC70473E
:100C80000B7803704B7843708B788370F6E700BF66
:100C9000E0C2000810B5104B104C1A6882B0204614
:100CA0000F49FFF7B3FF0F4B1B689BB10E4BA178A9
:100CB0002078627833F8104033F8122033F811307E
:100CC00001A801218DF804408DF805208DF806302B
:100CD000FFF758FF02B010BD540100207000002043
:100CE0006C0000205C010020ECC100080E4B1B686A
:100CF000032B18D8DFE803F013100A020B4B002275
:100D00003F2119705A709A70FFF7C4BF084B012237
:100D100000201A60FFF76ABF0020FFF767BF054B8E
:100D20001868FFF743BF70472C0400206C000020B8
:100D3000780400205C01002030B5234B8DB01B6887
:100D4000002B20D0214D00242A462346116914325D
:100D5000890741BF0CA800EB840141F82C3C013409
:100D600001330B2BF2D1002C1FD1194A23461460FA
:100D700003EB830305EB83056B689847154B002253
:100D80001A600DB030BD1249124A09680F4801EBD4
:100D90008101156800EB81008468691CA142116023
:100DA000EFD3416813608847EBE70AF00BFAB0FB1A
:100DB000F4F303FB14000CAA02EB800353F82C3C61
:100DC000034A1360D4E700BF7404002078000020B9
:100DD0003C030020700300202DE9F00F0C0682B0C8
:100DE0004BD46FEA020ADFF808C10AF1090A3F4B47
:100DF000072A88BF4FF0000A00F10806C2F1070871
:100E0000042703EBC10B8244CDF80480B61A0124F9
:100E1000ACF14805072A16D801990BEB07090346E0
:100E2000112B0CD819F8048C48FA01F818F0010FAE
:100E30001ABF4FF004080CF803800CF8034001338C
:100E40000139B342ECD1BAF1110F9FBF07EBC708CC
:100E5000534651464FEA480801D905E01946013387
:100E60004144112B6C54F9D901370C2F0CF1120CA1
:100E7000D0D102B0BDE8F00F7047B0394C2932D85C
:100E8000DFE801F02F313131313131313131313160
:100E900031313131313131312D3131313131313146
:100EA000313131313131313131312B313131313138
:100EB00029313127313131312D3131313131313138
:100EC000313131313131313131312B313131313118
:100ED0002900052185E7042183E7032181E7022119
:100EE0007FE701217DE720217BE700BFECBD000803
:100EF000D0380020B0F5907F10D248F63963C3F6A1
:100F0000E303A3FB00239B08DA0742BF03EBC30301
:100F1000C0EB83001130013008F000BE704700BF05
:100F200070B5294B82B01A6806460AB901261E60C0
:100F3000264A274B11785478907833F8111033F8FB
:100F4000142033F810300024224D8DF800108DF855
:100F500001208DF802308DF804408DF805408DF8A1
:100F600006400BE0FFF7C6FF15F8013C013443F0E3
:100F70000103B4F5907F05F8013C16D015F8013B4C
:100F8000204603F00203DBB26946002BEAD120467B
:100F900001A9FFF7AFFF15F8013C013423F001036D
:100FA000B4F5907F05F8013CE8D116B10A4B1B68F7
:100FB00033B1FFF7DFFD094B01221A6002B070BDAB
:100FC0000120FFF7F3FDF6E76C030020600100202D
:100FD000ECC10008883800202C0400208438002050
:100FE00008B5064B1A6822B1002210461A60FFF7B6
:100FF00097FF034B01221A6008BD00BF7404002054
:101000008438002008B50D4B0D481A680D49FFF7CC
:10101000FDFD0D4B1B68032B03D00C4B1B68990780
:1010200008D40B4B1B6803B908BD0120BDE808407C
:10103000FFF776BFFFF76EFDF3E700BF94010020D6
:1010400060010020580100202C04002074000020C2
:101050005C0100202DE9F041864B84B01A683AB952
:1010600085490B68002B00F0E48004B0BDE8F081F6
:10107000824A4CF6CD401678CCF6CC40A0FB061048
:101080007D49002400091C600C60DFF8088200F034
:10109000B580C8F8000055784CF6CD43CCF6CC436B
:1010A000A3FB05031B09DFF8F0C102D1002D40F0BE
:1010B000BE80CCF8003094784CF6CD43CCF6CC43CF
:1010C000A3FB04231B096E4F02D1002C40F0AD801E
:1010D0006C4A3B606C4B00201070507090701E701A
:1010E0005D709C70D8F800301C4693B1664A147845
:1010F000A34240F2968014B1002010700124614A8E
:101100005E4815780078EB18834200F2A2801370D5
:101110000124DCF800308BB15B48427893427CD9E3
:1011200012B1002242700124564A54485578407842
:10113000EB18834200F29280537001243868002833
:1011400063D0514B9A78904263D912B100229A70C1
:1011500001244C4D494AAF7896783818B0429CBF6C
:10116000C0B2A87003D9B7424FD0AE7030464749DD
:1011700092F800C092F801E06C782F785A781D78C8
:101180009B7831F81C8031F8177031F81EC031F8A7
:10119000122031F816E031F8133031F8146031F8CC
:1011A000104031F815008DF80A40394D8DF8048053
:1011B0008DF805C08DF806E08DF808708DF809608F
:1011C0008DF80C008DF80D208DF80E30002407E00E
:1011D000012B34D0032B37D00134B4F5907F0AD0E3
:1011E000635D022BF4D1204602A90134FFF782FE91
:1011F000B4F5907FF4D1FFF7BDFC36E7002E3FF445
:1012000048AF0123C8F8003045E764BB01230B60F9
:101210002BE7121A9A7001249BE7D21A427001241C
:1012200082E7E41A1470012469E7012350E70123DF
:101230003FE7DFF86080DFF860C0114F52E72046DB
:1012400003A9FFF757FEC7E7204601A9FFF752FEA3
:10125000C2E785421CBF107001245AE785421CBFBB
:10126000507001246AE7054A064D9678A878064B27
:101270007DE700BF74040020843800206001002056
:10128000800400204003002044030020ECC100083B
:1012900088380020840300206403002070B5154ABC
:1012A000154B94781178557833F8111033F81520D0
:1012B00033F8143082B00024104E05468DF800102B
:1012C0008DF801208DF802308DF804408DF805402E
:1012D0008DF80640A35D20462B4201A918BF694640
:1012E0000134FFF707FEB4F5907FF3D1FFF742FC1E
:1012F00002B070BD60010020ECC1000888380020F9
:101300002DE9F8435A4B5B4E1A682AB93768002F0B
:1013100000F09980BDE8F883DFF8608100221A6050
:101320003260C8F80020544C4FF0000E7746A446B7
:101330000EEBCE056D0012230CEB05095A1EA91801
:10134000605C611810F0010F46D0112A05EB03070D
:101350004BD01CF8077020F00100FF0740D4087044
:10136000002A47D0023B0127002BE7D10EF1010EE6
:10137000BEF1100FDCD10120FFF790FF002F5ED0EF
:10138000D8F800300127012B08BF3B4CC2D1DFF851
:10139000E8E04FF0000CF1460CEBCC056D000023AB
:1013A00009EB0508EA18A15CA21801F00600022862
:1013B00027D00133112BF5D90CF1010CBCF1100F22
:1013C0000EF1120EE8D10420FFF768FF002FA1D123
:1013D00001233360BDE8F8831346002BAED1C5E787
:1013E00013460127002BA9D1C0E720F0010089F89E
:1013F0001100B7E70EF1010E0127BEF1100F97D1D2
:10140000B9E73BB301F00400C0B20028D1D141F0EC
:101410000401112B117022D00133EA18A25C02F0F2
:101420000202D2B24AB1112B19D001331EF80320A7
:1014300002F00202D2B2002AF5D10127BAE7012355
:10144000C8F80030A3E7DFF83480D8F80030002B6C
:1014500099D168E741F0040188F80010DCE70CF14D
:10146000010C0127BCF1100F0EF1120E94D1AAE766
:10147000740400208438002088380020780300207D
:101480002DE9F00F6A4B1A6832B96A4A1368002BCB
:1014900067D0BDE8F00F704700201860654A664EBF
:1014A000664B012110603160196033688BB164486C
:1014B00010256C1E0023C25C02F00301012936D006
:1014C0000133122BF7D112382546002CF1D13460AC
:1014D0003FE0DFF868A1DAF8001000293ED0DFF81D
:1014E00074B1DBF80020002A3DD0564C564A2168E2
:1014F000106801EBC105554A00EB45050131575D08
:1015000001EBC10600EB4600514E27F0040757558A
:101510003668155CB14245F0040708BF45F0050583
:101520001754216004BF1554CBF8003011E047492F
:1015300004EBC40003EB400022F001020F2C0A541C
:1015400007D005EBC50503EB4503CA5C42F0010279
:10155000CA540520BDE8F00FFFF7A0BE01231360B9
:1015600097E7354EA1E740F27041C2F200010F68E3
:1015700040F2D43340F250313148C2F20003C2F29B
:101580000001D3F80090D1F8008094461026A0F511
:101590008775741ED30748D40023C25C02F0030190
:1015A000022905D00133122BF7D14B46002210E05F
:1015B000A4B112F0010216D006EBC60203EB420200
:1015C000A95CB04641F00401A9544FF0010C274634
:1015D0000122264612388CB19946DAE7EA5C42F0DD
:1015E0000502EA54F3E7BCF1000FF0D1E95C4FF0DB
:1015F000010C41F00401E9549046E8E740F27041E3
:10160000C2F200010F6040F2D431C2F200010B605F
:1016100040F25033C2F20003C3F80080CBF800C0A0
:10162000002A96D1CAF8002093E74B46D1E700BFC5
:1016300074040020843800204C040020480300205B
:101640009639002050030020D40300208838002061
:1016500070040020840400202DE9F843694B1A68C7
:1016600032B9694D2B68002B00F0A180BDE8F883EA
:1016700000201860654C644B206018604FEAC00C75
:101680000CEB00035B00624A1918C0F11206154604
:10169000F3188A18EF18A8461346197841F0040188
:1016A00003F8011BBB42F8D1C0F10F0E431C734578
:1016B00028BF4FEACE0C1BD20CEB0007C0F1110380
:1016C00000EB08014FEACE0C03EB470312390CEB99
:1016D0000E075B1901EB4707917C41F0040102F80A
:1016E000121F997CBA4241F0040103F8121FF3D192
:1016F0000CEB0E0205EB42020346D15C41F0040103
:10170000D1540133B342F8D3002848D0421EC0F16F
:101710001307BA420FD202EBC20149000B185B1942
:101720007E19013B761813F8011B21F00401B34226
:1017300003F8011CF7D1C0F11008404528BF4FEA5B
:10174000C8091DD200EBC0034FEAC80902EB4303EE
:10175000511909EB080CC0F112065B1901EB4C0C96
:1017600093F800E0991A2EF0040E83F800E011F8C7
:1017700006E012332EF0040E634501F806E0EFD1C7
:1017800009EB080300EB43035B19013B13F8011B52
:10179000013221F00401BA4203F8011CF6D30420FF
:1017A000FFF77CFD236801332360BDE8F883174C05
:1017B000206807287FF662AF08281CBF144B03F58A
:1017C000907404D119E0A34203F8010C0ED013F871
:1017D000012B02F00201C9B242F0040022F004021F
:1017E0000029F0D1A34203F8012CF0D10420FFF727
:1017F00055FD01232B60BDE8F88307220B27044D1C
:1018000089E700BF740400208438002050040020C1
:101810008838002070B5264A264813681BB903682B
:10182000002B3BD070BD00231360234D234A03607F
:101830002B6013602E6886B9214B03F590711A78DE
:1018400022F0040203F8012B8B42F8D10420FFF7A9
:1018500025FD2B6801332B6070BD184A13680133D6
:101860001360DA07DED5741EA4B2B4F5907F10D2EF
:1018700013490B5D03F00202D2B22AB110E00B5DF6
:1018800003F00202D2B25AB90134A4B2B4F5907F87
:10189000F5D10123036001362E6070BD064DC9E706
:1018A00043F0040304200B55661CFFF7F7FCF2E736
:1018B0007404002084380020580400204C030020C9
:1018C000883800202DE9F00F8D4A86B0136843B99F
:1018D0008C4B1A68002A00F0098106B0BDE8F00FB1
:1018E000704700231360884C864A2360136003937B
:1018F000864F002000EBC00207EB42020023117864
:10190000013321F00401122B02F8011BF7D1013041
:101910001028EFD1039B002003F10109C3F1080651
:10192000C4F800900196C21900231178013321F008
:101930000801122B02F8011BF7D11230B0F5907F8D
:10194000F1D1019A714D5342CDF8089093469A46D1
:1019500000269946BAF1080F2CBFD0464FF0080870
:101960004A4601990023BBF1070F34BFDC464FF014
:10197000070C17E0082934BF08460820082B6446E6
:1019800003D9092A2CBF1046092004EBC40400EB3C
:1019900044003C5C44F008043C5401330131013202
:1019A000122B15D0E85C00F00200C0B20028F4D081
:1019B000072EDFD9082B05D8082934BF0846082090
:1019C0004446E2E7082A8CBF104609204446DCE77B
:1019D00001361235102E0AF1010A0BF1010BB9D1B3
:1019E000039E002301936FF0110303FB0673DDF8E0
:1019F00008906FF0120C02936FF023030CFB06FCAF
:101A0000DDF80CB003FB06F65A46D2430596CA46EB
:101A10004FF000080492039E0BEBCB056D00049B76
:101A2000AA19019EED18F119D219ED194C4600239F
:101A30001DE0082B2ED8C14509D8994507D8059E29
:101A4000A81910F8126C46F0040600F8126C11F890
:101A5000010B00F00806F6B21EB140F0040001F8D8
:101A6000010C0133013201350134122B29D012F857
:101A70000C00C007EBD5B8F1070FDAD9082B16D840
:101A8000BAF10F0FE3D89945E1D8A87C40F00400E3
:101A9000A874DCE7C145DAD8112CD8D8029E3019D9
:101AA00010F8126C46F0040600F8126CCFE7BAF199
:101AB0000F0FCCD8112C9EBFD07C40F00400D07406
:101AC000C5E7019A029B08F1010812321233B8F1FE
:101AD000100F01920BF1010B02930AF1010A9AD146
:101AE000042006B0BDE8F00FFFF7D8BB064C226813
:101AF000082A03927FF6FCAE01221A60EDE600BFD1
:101B000074040020843800207C04002088380020E1
:101B10002DE9F84FA64C2368002B40F0A980A54B77
:101B20001B68032B12D8DFE803F076461302236804
:101B3000002B40F0CB80A04A13683BB99F490B684B
:101B4000B3F5907FC0F0C98001231360BDE8F88F22
:101B50002368002B00F0A280954900220A60984B70
:101B600095491A600A60974C02F1120504F11208B7
:101B70001D600021C2EB08088B1A1B1908EB01003D
:101B80000DE013F8126C16F0010F9E5C00F002815C
:101B900046F004069E540133984200F002818D42C3
:101BA000EFD993F80E6106F00206F6B2002E00F0AF
:101BB000F0809E5CECE72368002B7AD07C49002300
:101BC0000B60814A7C4913600B605F1C7D4C1E4694
:101BD000176003F5907C594203F1130033193A461C
:101BE0000DE05D7815F0010F5D5C00F0F28045F0CE
:101BF000040501325D540133824200F0F280112A63
:101C0000EFD913F8115C05F00205EDB2002D00F0DC
:101C1000DF805D5CEBE72368002B34D0644A002151
:101C200011606A4B644A19601160481C654C186069
:101C30004E42C1F59077331900220EE013F8015C93
:101C400015F0010F5D5C00F0978045F0040501324E
:101C50005D540133122A00F097809042EED95D7CEA
:101C600005F00205EDB2002D00F085805D5CECE72B
:101C700009F0A8FAC3179B0FC21802F00302D31A87
:101C80004C4A13604DE74C4A1368002B7FF45EAF5B
:101C90004E4B196811293FF657AFC6E746490B6806
:101CA000002B7FF453AF464B1A68B2F5907F09D2F0
:101CB00059E741490B68002B7FF448AF424A13684B
:101CC000112B82D901230B60BDE8F88F384A00231D
:101CD00013603A49384A0B6013603A4C4FF6EE7A7B
:101CE00003F11202CFF6FF7A0A6003F5997B04F143
:101CF0001208C3EB0A0A40F21F16A2F590710AEB14
:101D000002000919131902EB080518E091F8207177
:101D1000C2EB030CFF0755BFC2EB03071CF80070B2
:101D200017F800C047F0040756BF2CF0040C0CF85D
:101D3000007007F800C001330131AB4213D0B2424A
:101D4000E4D90F78C2EB030907F00207FFB2002FB6
:101D50004CD019F80070013347F004070131AB4251
:101D600009F80070EBD112325A45C6D10420BDE803
:101D7000F84FFFF793BA5D5C25F0040501325D541E
:101D80000133122A7FF469AF1236BE427FF453AF9B
:101D9000ECE79E5C26F004069E54013398427FF4E3
:101DA000FEAE1231B1F5907F7FF4E6AEDEE700BF04
:101DB00074040020680300208438002060030020A1
:101DC00064040020883800205404002038040020D7
:101DD0005D5C25F0040501325D54013382427FF4DD
:101DE0000EAF123666457FF4F9AEBFE719F8007002
:101DF00027F0040709F800709DE700BF2DE9F04FB8
:101E0000B24A85B01368B24E33B93368002B00F084
:101E1000968005B0BDE8F08F00231360AD4AAE4C4C
:101E20001360AE4AAE4D1360AE4A336023602B6040
:101E300013602368002B43D1AB4A11781F295FD967
:101E400051781F2900F2C6803F228DF808308DF8A6
:101E500009208DF80A30A54B03A802A91A689D4FE6
:101E6000FEF7D4FEA2492E689DF80C809DF80DC0A7
:101E70009DF80EE09F4B38689F4A31F8188031F882
:101E80001CC031F81EE006EBC60100EB4100002645
:101E9000194683F8008083F801C083F802E01670C9
:101EA00056709670FFF726F823682D6893493868B6
:101EB000CD5493495A1CC8542260FEF75BFEA8E734
:101EC0002A681C2A24D98F4B03F5907403E0A3429F
:101ED00003F8010C0ED013F8012B02F00201C9B275
:101EE00042F0040022F004020029F0D1A34203F8DA
:101EF000012CF0D10420FFF7D1F90123336088E7EA
:101F00003F228DF808208DF809308DF80A30A2E7BD
:101F1000DFF8C8E16F4FDEF80030D7F800C09A4212
:101F200077D0704B1B6802F00109B9F1000F4AD15C
:101F300063452DD90CF101033B602A682FE0664C04
:101F4000674D76E7BBF1110F19D85B4608EBC80067
:101F500043F6880C03EB4000C2F2000C1CF800C0F2
:101F60001CF0010FDDF800C004D0E0E0C85CC00741
:101F700000F1DD800133122BF8D1CDF800C008F15B
:101F800001081231B8F1100F65D11D23CEF80030D1
:101F9000DEF800309A4228D301232A6833600F2AE2
:101FA0002ED92368DFF854810D2B78D0544E296840
:101FB0003A680C2B08F80310F25401D8013323605F
:101FC000FEF7D8FD25E76345E2D20CF1FF333B6015
:101FD0002A68E4E792781F2A0AD88DF808308DF82D
:101FE00009303F238DF80A3035E701322A60D6E701
:101FF0003F228DF808308DF809208DF80A202AE755
:10200000386802EBC20200EB42003A49FEF772FF69
:10201000C7E740F23440C2F2000003689C4582D119
:1020200012F0010900F08B800CF1FF3B9246BCF1ED
:10203000000F02D102F1010AE346BAF10F0FA4D852
:1020400043F688030AEBCA01C2F2000303EB410125
:10205000D046CDF800C0D0455FD018F001033FF462
:1020600075AF112308EBC80043F6880CC2F2000CD0
:1020700003EB40001CF80000DDF800C0C00706D4E8
:10208000002B3FF47AAF013BC85CC007F8D540F2A3
:102090003440C2F20000CEF80080036045E798F8B3
:1020A0000030174E0F2B2FD90023013318F803E00F
:1020B000F15C08EB0300F2180C2B00F801EC02F8BD
:1020C000011CF2D12368013B236070E774040020F7
:1020D0008438002038030020540300201803002017
:1020E0007C030020340400205801002094010020CB
:1020F000ECC1000828040020300400202003002048
:102100003C04002088380020307803EBC3031049DA
:1021100000EB4300FEF7EEFEC6E718F0010F3FF4B8
:1021200011AFBBF1FF3F18BF5B469BD127E740F2E1
:102130003441C2F20001CEF800800B60F5E6BCF13C
:10214000100F9CBF0CF1010B92467FF676AF71E742
:10215000300400202DE9F04F7F4B85B01A687F4C8A
:10216000002A40F098802368002B57D1DFF800B296
:10217000DBF800202F2A54D8DFF8ECA1DFF8F88133
:102180009AF800009AF801109AF802208DF80C00D5
:102190008DF80D108DF80E20994658F8044B182C28
:1021A0002DD9A4F11805012D63D0A4F11A030F2B2A
:1021B00067D90F2D5DD904EBC407193CA9F5EA7363
:1021C0000126A51E0F2C03EB470709D90E2D45D973
:1021D0000136243F6B1C2C460FD0A51E0F2CF5D8C2
:1021E0009AF8013007F11200B3FBF6F303A98DF85A
:1021F0000D30FEF77FFE002CE8D158F8044C09F1B1
:1022000001090134B9F1120F48F8044CC5D1FEF7A9
:10221000B1FCDBF800300133CBF8003005B0BDE88D
:10222000F08F4F4B03F5907503E0AB4203F8010CC0
:102230000ED013F8012B02F00201C9B242F00400E3
:1022400022F004020029F0D1AB4203F8012CF0D1B6
:102250000420FFF723F801232360DFE79AF8013019
:102260003846B3FBF6F303A98DF80D30FEF742FEB6
:10227000AEE705EBC50009EB40003A49FEF73AFE30
:1022800099E705EBC500A9F1240303EB40003649AB
:10229000FEF730FE8DE7354A002617681E60344B86
:1022A0003F253A4602A869461E6010238DF8063085
:1022B0008DF800508DF801508DF8055026608DF88E
:1022C00002608DF80460FEF7A1FC3A4603A801A95C
:1022D000FEF79CFC274B9DF80E709DF808809DF83A
:1022E00009C09DF80AE09DF80C509DF80D001D49AD
:1022F0001D4A33F8155033F8188033F81CC033F8F2
:102300001EE033F8100033F8173015701A4F81F8BB
:10231000008081F801C081F802E05070937035466A
:102320000DE008F04FFFC3171B0FC01800F00F009F
:10233000C31ABB5101350436122D3FF414AFEA071E
:10234000EFD408F03FFFC3171B0FC01800F00F00B9
:10235000C31A0833BB51EDE7740400208438002011
:10236000883800206C0400206004002094010020C4
:1023700030030020ECC10008E003002010B582B05B
:10238000002914BFFF230023002814BFFF240024CA
:10239000002A14BFFF220022002001A98DF804406A
:1023A0008DF805308DF8062007F0B8FB012007F006
:1023B0002FFB02B010BD00BF074B012003F5907149
:1023C00013F8012B12F0020214BF03F8010C03F8FA
:1023D000012C8B42F4D17047883800202DE9F84F4A
:1023E0001746814688460AB9BDE8F88F0020FEF7F7
:1023F00097FD39077FD4FA0679D44B4A4B4B1268C4
:1024000003EBC20113F832B07B0791F801A0EBD5C2
:10241000474E4B224748002108F03FFC06F59075D7
:102420000122334613F8014B14F0020414BF03F8E1
:10243000012C03F8014CAB42F4D13F4B1B68002B3D
:1024400067D03E4B1B68D80767D53A4B01225A70BC
:102450009A703B4BCBEB0B1B08EB8B01354C03EB22
:10246000C10101200023CA185278013312B1072B91
:10247000A054F8D10B780AEB8A0A9944B9F1180FE5
:1024800088BFA9F119092F4B0AEB8A0A0AEB090444
:10249000284803EB840401210023E25C013312B1DC
:1024A000042B8154F9D1284CDFF8A8C0002504F191
:1024B0004B0714F8013F93B105EB0C03987815F81E
:1024C0000C205B7858B102EBC202181806EB4202EE
:1024D000D15C41F00201D15401338342F8D103357C
:1024E000BC42E6D1194B01221A60BDE8F88F0120E9
:1024F000FEF77CFB81E706F099FDC820FEF7A0FA05
:10250000134B1B68002B7FF478AF0120FEF74EFBC6
:1025100073E7F9067FF568AFE4E7B8F1000F18BF7D
:10252000B8F11E0F95D190E780030020A4DC0008CD
:1025300088380020880300205C01002074000020FF
:10254000F0C2000890D70008870300207404002020
:102550002C040020C0DB000840F27403C2F2000328
:102560001868704738B50B4B04461B680A4D032B9F
:1025700004D0830702D52B68980707D5FEF7B6FB72
:10258000064B01222C601A60204638BDFEF7C2FAC5
:10259000F4E700BF2C040020740000207404002025
:1025A00040F22C43C2F2000318687047032810B5AC
:1025B00009D8074C2368834203D02060FEF796FBBE
:1025C0002368184610BD024B1B68184610BD00BF9B
:1025D0002C04002040F26813C2F200031868704710
:1025E0003B28024B88BF3C201860704768010020E0
:1025F00040F26413C2F20003186870473A28024B95
:1026000088BF0020186070476401002040F28033CA
:10261000C2F20003186870471128044B04D81860F0
:10262000034B01221A60704718687047800300202E
:1026300074040020064B1868102805D90020186083
:10264000044B01221A60704701301860F8E700BFA0
:102650008003002074040020054B186828B101385D
:102660001860044B01221A60704711201860F8E7C7
:10267000800300207404002040F26843C2F200038B
:1026800018687047074B10B5186000B110BD064BB5
:102690000F241C60FEF7B6FC044B1C60BDE8104024
:1026A000FEF7F8BA680400209401002054010020CD
:1026B00040F29813C2F2000318687047024B0A28D0
:1026C0008CBF18681860704798010020044B186888
:1026D000092802D90020186070470130186070473F
:1026E00098010020044B186810B101381860704739
:1026F0000A201860704700BF98010020064B1B6835
:10270000012B00D07047054B00223F2119705A70F1
:102710009A70FEF777BC00BFD80300205801002054
:1027200040F2D833C2F2000318687047012810B590
:10273000034602D9054B186810BD044C2068984226
:1027400003D02360FFF7DAFF206810BDD803002014
:10275000F0B5584B83B01B680446012B42D0022BC6
:1027600001D003B0F0BD20B9534B1A68002A7AD0CB
:1027700018600020FEF73AFA504B1B683B2B2ED80E
:102780001D2B73D967081E254D4A4E4B1078517882
:10279000927833F8100033F8111033F81220464BBA
:1027A0008DF804001B688DF805108DF80620002BAD
:1027B00046D1AF423CBF444E3C4606D339E000F21E
:1027C000211007F0ABF9AC4233D2306801A92018D0
:1027D0000134A842F3D33C383B28F4D8EFE727462E
:1027E0003C25D1E70020FEF701FA344B1B683B2B58
:1027F00048D9354A3C231268A418314AA34298BFED
:10280000C3EB040411782F4B9078557833F81110EE
:1028100033F8152033F810303B2C8DF804108DF868
:1028200005208DF8063004D804F2211001A907F024
:1028300075F9264B1B68002B93D0FEF79FF990E7A4
:10284000214E002405E000F2211007F067F9BC4298
:10285000EFD8336801A9E0180134A842F3D33C381B
:102860003B28F4D8EFE701221A6082E7132B7FF6AA
:1028700078AF4AF6AB27CAF6AA27A7FB0437142578
:102880007F0881E71D2B0ED8132B7FF66AAF4AF61F
:10289000AB23CAF6AA23A3FB04240B4A1423126811
:1028A00002EB5404A9E7084A1E23126802EB540401
:1028B000A3E700BF2C04002078040020680100205A
:1028C00070000020ECC10008640100205C010020C1
:1028D00038B5874B1B680A2B1DD8864A864C126870
:1028E00092B9864D2A68DAB9042B00F0E280844A56
:1028F000844803EB8303116800EB8303986801317C
:102900008142116045D238BD7E4A03EB830302EB5E
:1029100083035B689847794B1B68002BF3D0764C98
:10292000794B1B68012B1FD0784B1B68032B06D0FB
:102930002368002BE7D1BDE8384006F093BB744B09
:1029400074491A68496B0132B2EB411F1A60EFD328
:10295000714A0020116818604B1E052B3AD8DFE839
:1029600003F050A19A938C856C4B6D491A684969A4
:102970000132B2EB411F1A60D6D36A4A00201168B7
:1029800018604B1E052B0CD8DFE803F069625B541E
:102990004D4400215B68116098472B68002BBED125
:1029A000B1E761490B680133072B00F09E800B6093
:1029B0005E4913600A685B4801320D2A0A6000F024
:1029C0008B800E2AB0D1013B08BF06230360002391
:1029D0000B60A9E756490B680133072B7AD00B60CF
:1029E000544913600A684C4801320D2A0A6068D0C5
:1029F0000E2A9DD1013B08BF0623036000230B6014
:102A000096E74D4B59783E29E4D801315970FEF7CD
:102A100041F98DE7494B99780029C2D00139997065
:102A2000FEF7F0FA80E7454B19783E29B9D8013115
:102A30001970F5E7414B59780029B2D00139597026
:102A4000EEE73E4B99783E29ABD801319970E7E724
:102A50003A4B19780029A4D001391970E0E7374BB7
:102A600059783E299DD801315970D9E7324B997870
:102A70000029AFD001399970C9E72F4B19783E2949
:102A8000A8D801311970C2E72B4B59780029A1D081
:102A900001395970BBE7284B99783E299AD8013102
:102AA0009970B4E7244B1978002993D00139197033
:102AB000ADE7144B5B6D98472B68002B7FF42FAF6D
:102AC00021E70133072B18BF03607FF431AF0123E7
:102AD00003602DE7012382E70133072B18BF036052
:102AE0007FF422AF012303601EE701235FE700BFED
:102AF00098010020740400205C010020843800202C
:102B00007403002078000020D80300202C0400204B
:102B1000140300202C000020DC0300205C030020B4
:102B200070010020580300201C03002090010020A9
:102B3000340300206C0100206C00002058010020AC
:102B4000064B1A783E2A07D803D13F221A70FEF7A7
:102B500059BA02321A70FAE7704700BF58010020D4
:102B6000064A137843B1012B03D100231370FEF7FB
:102B700049BA023B1370FAE7704700BF58010020C2
:102B8000064B5A783E2A07D803D13F225A70FEF7E7
:102B900039BA02325A70FAE7704700BF5801002074
:102BA000064A537843B1012B03D100235370FEF73B
:102BB00029BA023B5370FAE7704700BF5801002062
:102BC000064B9A783E2A07D803D13F229A70FEF727
:102BD00019BA02329A70FAE7704700BF5801002014
:102BE000064A937843B1012B03D100239370FEF77B
:102BF00009BA023B9370FAE7704700BF5801002002
:102C000040F25813C2F200031A7802705A784270E8
:102C10009B788370704700BF10B404784178827845
:102C200040F25813C2F200033F2C34BF20463F202D
:102C30003F2928BF3F213F2A28BF3F2218705970E3
:102C40009A7010BCFEF7DEB940F26C03C2F20003CA
:102C50001A7802705A7842709B788370704700BF70
:102C600010B404784178827840F26C03C2F2000319
:102C70003F2C34BF20463F203F2928BF3F213F2A19
:102C800028BF3F22187059709A7010BCFEF702B826
:102C900040F29413C2F20003186870470F2803D85B
:102CA000034B1860FEF7AEB9014B0F221A60F9E72B
:102CB00094010020034B1A6802B97047013A1A6068
:102CC000FEF7A0B994010020044B1A680E2A00D91F
:102CD000704701321A60FEF795B900BF94010020D9
:102CE00040F25413C2F20003186870470F2803D84B
:102CF000034B1860FDF7CEBF014B0F221A60F9E7B6
:102D00005401002070B5012682B040F25D1516F026
:102D1000010F0CBF0021392116F0020F0CBF002259
:102D2000392216F0040F0CBF002339238DF804104C
:102D30008DF805208DF806300024204601A90134C5
:102D400006F0ECFEAC42F8D1204606F061FE0136FA
:102D50000320FDF783FE082ED9D10020FEF7E0F80E
:102D6000002001460246FFF709FB02B070BD00BF1C
:102D70002A4B2DE9F04103F59071012413F8012B42
:102D800012F0020214BF03F8014C03F8012C8B422D
:102D9000F4D1017800293FD080460746082600205C
:102DA000C6F10802FEF718F898F80110013759B378
:102DB000112E16D83D46344601E0112C11D820467C
:102DC0000022FEF709F815F8011F09340029F4D193
:102DD00005E02046202100220934FDF7FDFF112CDB
:102DE000F7D90420FEF75AFA3220FDF729FE013EFA
:102DF0000CD017F8011C0020C6F10802FDF7ECFF0B
:102E000098F801100029D3D13446E8E718F8011FDB
:102E10000029C3D1BDE8F081BDE8F08188380020E9
:102E2000F8B5324B1B681BB1A0F114053B2D00D93E
:102E3000F8BD0020FEF774F82D4B2E4C93F8883027
:102E400004F59071C3EB031305EB83052A4B0120B6
:102E500003EBC505234613F8012B12F0020214BF41
:102E600003F8010C03F8012C8B42F4D1234E707946
:102E7000F278337958B102EBC202181804EB42021F
:102E8000D15C41F00201D15401338342F8D1307A50
:102E9000B279F37958B102EBC202181804EB42027E
:102EA000D15C41F00201D15401338342F8D10027B3
:102EB000EB195B78ABB103EB4303F1188878F25C54
:102EC0004B7858B102EBC202181804EB4202D15CF5
:102ED00041F00201D15401338342F8D10137072F69
:102EE000E6D1074B01221A60F8BD00BF5C0100204B
:102EF000A4DC000888380020F0C20008C0DB00080D
:102F0000740400202DE9F04FBA4B04461B6893B0BF
:102F1000184613B913B0BDE8F08F3F268DF8346022
:102F20003C2603258DF82360162600230CA92A468B
:102F3000A4208DF824600F268DF835308DF83630BA
:102F40008DF825308DF826308DF82B308DF82750F0
:102F50008DF8296000F0B0FB01220DF12101A720BE
:102F600000F0AAFB01220DF12501A82000F0A4FB2E
:102F700001220AA9BD2000F09FFBBE2001220DF115
:102F80002A0100F099FBB4F5843F80F0A4809DF8FD
:102F900021809DF822C0B8F1110F88BF4FF00008C2
:102FA0009DF825E088BF8DF82180BCF1030F84BF18
:102FB0004FF0000C8DF822C09DF82610BEF10A0FCC
:102FC00084BF4FF0000E8DF825E0012902D90021C1
:102FD0008DF826109DF828700F2F02D90F278DF835
:102FE00028709DF829600F2E71D89DF82A000128BD
:102FF00002D000208DF82A009DF823203C2A009260
:1030000003D93C258DF8235000959DF824303B2BA7
:1030100002D916238DF82430774C07932568774B17
:1030200001959DF827509DF834B002959DF83050D9
:103030009DF835A003959DF831509DF83690049584
:103040009DF8325083F800B005959DF82B5083F819
:1030500001A0069540F28035C2F20005C5F8008057
:10306000DFF8C481029DC8F800C0DFF8C0C183F852
:103070000290CCF80050DFF8B8C1614BCCF800E00A
:10308000DFF8B0E15F4ACEF800101F6003995E4B95
:103090001170049D05991E605C4B5570917018600D
:1030A000009A5B4B079D1A605A4B06991D605A4B5C
:1030B000196000232360FDF7EDFDFDF7A3FF019AE2
:1030C0002260FFF71BFBFDF711FE012022E70F2610
:1030D0008DF8296089E7A92001220DF1260100F071
:1030E000EBFA40F6FF03C0F201039C427FF64FAFBC
:1030F00001220DF12701BC2000F0DEFA0DA92A46BD
:10310000D72000F0D9FA01220DF12901DA2000F0D0
:10311000D3FADB2001220DF1220100F0CDFAB4F543
:10312000003FFFF434AF01220DF12301DC2000F059
:10313000C3FADD20012209A900F0BEFAFF23C0F284
:1031400002039C427FF623AF0DF12B010122E02008
:1031500000F0B2FA0FA90B22E52000F0ADFA0EAE96
:103160000BA9022240F2251000F0A6FA40F2351019
:103170003146042200F0A0FA0DF14605274B0DF16F
:103180003B0005E042F002021A611433A84212D05B
:1031900010F8012FFF2AF8D002F01001C9B202F096
:1031A0000F029A601A690029ECD122F002021A611A
:1031B0001433A842ECD19DF82C301948FF2B1EBFC8
:1031C000184A03F00F0353609DF82D30FF2B1EBFEC
:1031D000144A03F00F0353610023F25C00EB031168
:1031E0000133FF2A1CBF02F00F024A60042BF4D106
:1031F000CDE600BFA80400205C0100206C00002088
:10320000940100205801002054010020680400208F
:1032100068010020640100205C0400207800002088
:103220002C000020700100202C04002074000020DD
:1032300098010020D80300202DE9F04F854BA3B062
:103240001B68002B00F08C80834B844A93F800802D
:1032500093F801C093F802E0814B92F800B01F6828
:10326000804B92F801A01E687F4B92F802901D6877
:103270007E4B8DF819501C687D4B8DF81A401B68E9
:103280008DF820B000937B4B009C1B688DF81B4091
:103290000193794B019C1B688DF821A00293774B19
:1032A0008DF822901B688DF824800393744B8DF861
:1032B00025C01868734B8DF826E01968724B8DF89D
:1032C00015701A688DF816608DF81C40029C6F4BC3
:1032D0008DF81D40039C8DF817008DF81E408DF869
:1032E000181000208DF81F2012ACFF250A2888BF77
:1032F000255409D89A68196902F00F0289072254E7
:1033000044BF42F010022254013014334028EDD162
:103310005F4800230AAEFF22012B9BBF00EB031185
:103320004968F25401F00F0198BFF1540133102B9A
:10333000F2D1584800230EADFF21032B9BBF00EBB9
:1033400003125268E95402F00F0298BFEA540133A5
:10335000102BF2D1A42008A9032200F0C7F918B954
:10336000002023B0BDE8F08FA7200DF11501012248
:1033700000F0BCF90028F3D0BC200DF119010122A6
:1033800000F0B4F90028EBD0A8200DF11A010122B9
:1033900000F0ACF90028E3D0A9200DF11B010122B7
:1033A00000F0A4F90028DBD0BD2007A9012200F01D
:1033B0009DF90028D4D0BE200DF11E01012200F09D
:1033C00095F90028CCD0D72009A9032200F08EF966
:1033D0000028C5D0DA200DF11D01012200F086F988
:1033E0000028BDD0DB200DF11601012200F07EF98E
:1033F0000028B5D0DC200DF11701012200F076F98C
:103400000028ADD0DD2006A9012200F06FF90028C8
:10341000A6D0E0200DF11F01012200F067F900287D
:103420009ED0E5202146402200F060F9002897D088
:1034300040F225103146102200F058F900288FD0B4
:10344000102240F23510294600F050F9003018BF24
:10345000012086E7A80400206C000020580100200D
:10346000800300202C04002074000020980100201C
:10347000D80300209401002054010020680400209B
:1034800068010020640100205C0400207800002016
:10349000700100202C00002006F06ABB2DE9F843E3
:1034A00081468846174605F059FC10B90020BDE852
:1034B000F883552005F0FAFC2E48082105F032FD6E
:1034C000442005F0F3FC002443F2144505F0B0FC61
:1034D0000134AC4298BF002814BF00260126F5D065
:1034E00043F214439C4227D805F038FC0028DDD075
:1034F000552005F0DBFC204C08211E4805F012FD8C
:10350000BE2005F0D3FC0921204605F0C1FC05F0E2
:1035100025FC1A4B1B68222B13D0282B11D0092312
:10352000C9F8003094F901300120DB0FC8F80030F1
:1035300023783B60BDE8F88305F010FC3046BDE819
:10354000F88323796278C3F341132578093302F0B5
:103550000704C3F10C00191F45FA00F004FA01F149
:10356000D2090143C9F800300120C8F800203960B1
:10357000BDE8F8839C040020880400209804002003
:10358000F8B5A0F10905032D044602D900263046FE
:10359000F8BD05F0F7FC05F0E1FB0028F6D02E4F52
:1035A000384605F0CDFC3B782C4A012113602C4AAB
:1035B000222B0646116001D0282BE8D105F0CEFB66
:1035C0000028E4D0552005F071FC264F0821224840
:1035D00005F0A8FCBE2005F069FC0921384605F07D
:1035E00057FC3B79C3F341130933A342CFD005F015
:1035F000B5FB0028CBD0552005F058FC0821164813
:1036000005F090FC4E2005F051FC7F2005F04EFCAB
:10361000802005F04BFC680100F0E00005F046FC5E
:1036200005F09CFB05F09AFB0028B0D0552005F072
:103630003DFC0948082105F075FC482005F036FCE2
:10364000002405F0F5FB0134F92C98BF0028F8D0D0
:1036500005F084FB9BE700BF9C0400209804002039
:1036600094040020880400202DE9F04184B003F088
:1036700027F8DFF8408000240127650045F0A00509
:10368000012600972846002132460DF10F03A419A8
:10369000C8F8005003F04CF830B1082CEDD1044BC1
:1036A000186804B0BDE8F081014B30461E60F8E7B1
:1036B000A8040020A404002010B50A4B82B01C68A6
:1036C0000B4614B9204602B010BD0092064A0146CE
:1036D00012681046012203F02BF8D0F1010038BF28
:1036E0000020F0E7A8040020A40400202DE9F04702
:1036F000144B82B01B68174603B3EAB1DFF84CA045
:10370000114C0646C0EB01094FF001080025DAF81C
:103710000000CDF800803146012209EB060303F0DA
:1037200085F858B910202368002BFCD0013825609B
:10373000F9D10136013FEAD1012000E0002002B0BA
:10374000BDE8F087A8040020A8390020A4040020C8
:1037500030B53A4B87B01A68044682426BD068464F
:103760001C6006F021FD02A807F096F80420012154
:1037700006F0E6FE0420012106F0E2FE4FF40030E0
:10378000012106F0EBFE04234FF400600325C4F290
:1037900001006946ADF8003018238DF803308DF82C
:1037A000025006F09DFC08234FF40060C4F20100B3
:1037B0006946ADF8003048238DF803308DF802508B
:1037C00006F08EFC4FF48840C4F20000012107F09F
:1037D000A1F800234FF488401D46C4F2000002A95E
:1037E000ADF80C30ADF80E30ADF81030ADF8143047
:1037F0000C23ADF81230029406F0E8FF4FF4884035
:10380000C4F20000012107F053F84FF48840C4F2DD
:10381000000040F22551012207F058F826238DF8C8
:10382000043001A801238DF805508DF806508DF85D
:10383000073006F05FFA07B030BD00BFAC040020CF
:1038400030B40F4A13687F2BFCD80E490E4D0B681D
:103850005C1C7F2C45F8230098BF0C6001D9002325
:103860000B6072B613680133136062B64FF4884080
:10387000C4F2000040F22771012230BC07F026B8E4
:10388000BC060020C0060020B404002010B5044689
:10389000007828B1FFF7D4FF14F8010F0028F9D100
:1038A00010BD00BF40F2B043C2F200031868003000
:1038B00018BF0120704700BF30B40D4B1A6882B1A9
:1038C0000C490D4D0A68541C802C55F8225018BF25
:1038D0000C6009D072B61A68013A1A6062B6012209
:1038E0000560104630BC704700220A60F2E700BF56
:1038F000B0040020B4060020C4060020024A136869
:10390000002BFCD1704700BFBC0600204FF488405C
:1039100038B5C4F2000040F2255107F009F800283C
:103920002BD14FF48840C4F2000040F2277106F01A
:10393000FFFF00B938BD4FF48840C4F2000040F2E8
:10394000277107F01BF8234B1A68002A38D0224A47
:10395000224C1168481C802808BF002054F8211010
:1039600010601A684FF48840013AC4F2000089B22E
:103970001A60BDE8384006F0C5BF4FF48840C4F275
:10398000000040F2255106F0F9FF4FF48840C4F2E0
:10399000000006F0BBFF124B1A687F2AC1D81149FC
:1039A000114D0A68C0B2541C7F2C45F8220098BF04
:1039B0000C6001D900220A601A6801321A60B0E76F
:1039C0004FF48840C4F2000040F22771BDE838404F
:1039D00006F07CBFBC060020C4080020B404002010
:1039E000B0040020B8060020C4060020F0B583B063
:1039F00001A84FF40065C4F2010506F0D5FB0420D0
:103A0000012106F09DFD012402271026284601A968
:103A1000ADF804408DF806708DF8076006F060FB85
:103A20000420214606F08CFD284601A9ADF804705B
:103A30008DF806708DF8076006F052FB04202146D1
:103A400006F07EFD284601A9ADF804608DF80670E9
:103A50008DF8076006F044FB28462146224606F012
:103A6000B1FB28463946224606F0ACFB28463146D3
:103A7000224606F0A7FB03B0F0BD00BFF8B5094D24
:103A800004460F46002601E02B6833B92046FFF7B5
:103A900013FF0028F8D00120F8BD0136BE4228608F
:103AA000F4D3F8BDAC3900202DE9F04F85B00546C0
:103AB00003F004FDFFF722FFFFF7F4FE002843D0D8
:103AC0000024624FDFF888A10126A346294603A8F7
:103AD000FFF7D4FFDFF874914FF001080346002888
:103AE00035D0039B3E600A2B07D00D2BEED0FF2C68
:103AF000ECD80AF804300134E8E70AF804B0002CE6
:103B000032D103F0DBFCE1E7514852491A4607F095
:103B1000F0FB00284CD04E484F49032207F0E9FB48
:103B200000284FD04A484D49052207F0E2FB002803
:103B300055D14B484B49022207F0DBFB002849D105
:103B40000123C9F80830062005B0BDE8F08F4648CB
:103B5000019303F085FC454803F082FC444803F0E0
:103B60007FFC019B1846EFE73F48019303F078FC88
:103B7000374803F075FC3E4803F072FC34483D4979
:103B8000022207F0B6FB38B131483B49052207F065
:103B9000B0FB18B90220D7E74046D5E72C48374993
:103BA000022207F0A6FB019B0028ADD10320CBE742
:103BB00009F13C0032490F2207F0B4FBC9F8048038
:103BC0000420C1E709F11C002E491F2207F0AAFBBF
:103BD0000520B9E70023C9F808300620B4E71C48DF
:103BE0002949052207F085FB98B119482749092280
:103BF00007F07FFB10B316482549042207F079FB34
:103C0000A8B113482349092207F073FB40B1FF20F4
:103C10009AE7214812490F2207F084FB072093E717
:103C20001E481F49FF2207F07DFB0A208CE71D4834
:103C30001D491F2207F076FB092085E71B4818491C
:103C40000F2207F06FFB08207EE700BFC8080020A6
:103C5000980A002054DD000860DD000864DD0008DB
:103C60009D0A00206CDD000834DD000838DD000806
:103C700040DD000844DD000848DD000850DD000894
:103C8000A20A00209B0A002070DD000878DD0008F1
:103C900084DD00088CDD0008340A002014090020AF
:103CA000A10A0020140A00209C0A0020D408002049
:103CB000F0B583B0074607F014FB06461A4803F038
:103CC000CFFBBEB13C46F61904E0184603F0A2FB58
:103CD000B4420FD014F8013B6846A3F120055E2DD5
:103CE00012491A46F1D907F0B9FA684603F0B8FB51
:103CF000B442EFD10E4803F0B3FB03F0DFFB3846CC
:103D0000FFF7C4FD0B48FFF7C1FDFFF7F7FD02E029
:103D1000022807D020B10A20FFF7C6FE0128F7D1FC
:103D200003B0F0BD0020FBE798DD0008ACDD000823
:103D3000A0DD000874DF000838B539B10446451825
:103D400014F8010BFFF77CFDAC42F9D1BDE8384017
:103D5000FFF7D4BD40F6C800C2F20000704700BFB4
:103D600010B54FF40060C4F201000121002282B0BE
:103D700006F028FA0C4A0521144600201368002B8F
:103D8000FCD001392060F9D101214FF40060C4F268
:103D900001000A4606F016FA01A83221FFF76EFE6E
:103DA0000028F9D102B010BDAC39002008B5024698
:103DB0000B460748074907F051FA0548FFF778FF17
:103DC00020B1054B002283F83C205A6008BD00BF9B
:103DD000440A0020B4DD0008C808002008B50246E7
:103DE0000B460748074907F039FA0548FFF760FF17
:103DF00020B1054B002283F83C205A6008BD00BF6B
:103E0000440A0020C4DD0008C808002008B50246A6
:103E100008B1037823B90748BDE80840FFF748BF59
:103E20000549064807F01AFA0448BDE80840FFF7BC
:103E30003FBF00BFF0E30008D4DD0008440A0020C3
:103E400030B54FF4E13083B003F0D2FBFFF7CEFD85
:103E50004FF4E130FFF77CFC4FF40060C4F2010046
:103E60001021002206F0AEF91F4C4FF40060002232
:103E7000C4F20100012106F0A5F905252246002320
:103E800021680029FCD0013D1360F9D101214FF4D4
:103E900000600A46C4F2010006F094F91249322289
:103EA0002368002BFCD0013A0D60F9D14FF400607B
:103EB000C4F201001021012206F084F903E001A8F8
:103EC00003F0DAFA60B901A8FFF7F6FC0028F6D093
:103ED000019803F09FFA01A803F0CEFA0028F2D06F
:103EE0000198FFF7ADFCEEE7AC39002008B50B4BAD
:103EF0001A6802B108BD01224FF4E1301A6003F0E4
:103F000077FB074803F0ACFAFFF770FD4FF4E130A0
:103F1000FFF71EFCBDE80840FFF722BF940A00200F
:103F2000E0DD000810B403781649FBB100220860F8
:103F30001446013005E001300E2A14DC10F8013C73
:103F40008BB13D2B02BF01EBC20300F8014C58605E
:103F5000F1D0262BEFD1013200F8014C41F83200AC
:103F600001300E2AEADD531C0F2B08DC002201EB86
:103F7000C30011460133815008320F2BFADD10BC0B
:103F8000704700BF280C0020F8B50A4D06460024F3
:103F900055F83430E70031461846013423B107F0B4
:103FA0008EF918B1102CF3D10348F8BD014BDF197D
:103FB0007868F8BD280C0020FCDE000808B5FFF783
:103FC000E3FF4DF6D861C0F6000107F078F9D0F1B3
:103FD000010038BF002008BD00B50B4685B04DF686
:103FE000E0610246C0F60001684607F037F968460E
:103FF000FFF7CAFF05B000BD10B5044607F071F920
:10400000014600B910BD2046BDE81040FFF794BE40
:1040100010B504464DF6E860C0F60000FFF7ECFF6F
:104020004DF6F860C0F60000FFF7E6FF4DF60070B1
:10403000C0F60000FFF7E0FF4DF60C70C0F6000080
:10404000FFF7DAFF4DF61870C0F60000FFF7D4FF57
:104050002046FFF7D1FF4DF62070C0F60000FFF7B5
:10406000CBFF4DF62C70C0F60000FFF7C5FF4DF6F4
:104070003870C0F60000FFF7BFFF4DF64470C0F681
:104080000000FFF7B9FF2046FFF7B6FF4DF64C7072
:10409000C0F60000BDE81040FFF7AEBF38B50446DB
:1040A0004DF65470C0F600000D46FFF7A5FF204600
:1040B000FFF7A2FF4DF66070C0F60000FFF79CFF0F
:1040C0002846FFF799FF4DF66470C0F60000BDE882
:1040D0003840FFF791BF00BF4DF6FC604DF6787198
:1040E00008B5C0F60000C0F60001FFF7D7FF4DF697
:1040F00080704DF68871C0F60000C0F60001FFF731
:10410000CDFF4EF294704DF69071C0F60000C0F6EF
:104110000001FFF7C3FF4DF69C704DF6A071C0F68D
:104120000000C0F60001FFF7B9FF4EF610104DF683
:10413000A471C0F60000C0F60001FFF7AFFF4DF616
:10414000AC704DF6B871C0F60000C0F60001FFF784
:10415000A5FF4DF6C4704DF6D071C0F60000C0F654
:104160000001FFF79BFF4DF6DC704DF6E471C0F6E1
:104170000000C0F60001FFF791FF4DF6EC70C0F6AD
:104180000000BDE80840FFF737BF00BF054A1368CD
:1041900001331360DB0702D40348FFF72DBF034848
:1041A000FFF72ABFB40C002008E00008F0DF000889
:1041B00010B504464EF21000C0F60000FFF71CFFD9
:1041C0002046FFF719FF4EF21800C0F60000BDE8C8
:1041D0001040FFF711BF00BF70B584B00C46054614
:1041E0001B49164668461A4607F038F802A81849CF
:1041F000089A07F033F83CB123782BB12046FFF73B
:10420000FBFE1448FFF7F8FE1348FFF7F5FE2846BB
:10421000FFF7F2FE1148FFF7EFFE2846FFF7ECFE2E
:104220000F48FFF7E9FE3046FFF7E6FE0D48FFF7BF
:10423000E3FE6846FFF7E0FE0B48FFF7DDFE02A84D
:10424000FFF7DAFE0948FFF7D7FE04B070BD00BFE4
:104250002CEB0008C0E6000820E0000838E0000869
:1042600044E0000850E0000860E0000860DF00085B
:1042700010B504464EF26C00C0F60000FFF7BCFE1D
:104280002046FFF7B9FE4EF2A000C0F60000FFF78F
:10429000B3FE4EF2B000C0F60000BDE81040FFF7DC
:1042A000ABBE00BF70B505460F480E46FFF7A4FE33
:1042B0000E48FFF7A1FE002E0EDD043D00240C4841
:1042C000FFF79AFE55F8040FFFF796FE01340948F0
:1042D000FFF792FEB442F2D10748FFF78DFE074B7D
:1042E00000221A6070BD00BFB8E0000808E00008B6
:1042F000D4E00008ECE00008CCE00008B40C00209A
:104300004EF2FC00C0F60000FFF776BE38B504465A
:104310004EF20C10C0F600000D46FFF76DFE204671
:10432000FFF76AFE4DF66070C0F60000FFF764FE0E
:104330002846FFF761FE4EF23810C0F60000BDE8D7
:104340003840FFF759BE00BF4EF2481008B5C0F61E
:104350000000FFF751FE4EF25410C0F60000BDE819
:104360000840FFF749BE00BFF0B5044683B01F48C0
:104370001E460D461746FFF73FFE2046FFF73CFE60
:104380001B48FFF739FE2046FFF736FE1948FFF7B6
:1043900033FE002E24DD043D00240BE01648FFF719
:1043A0002BFE55F8040FFFF727FE1448FFF724FEF5
:1043B000B44215D02246124901A806F04FFF114819
:1043C000FFF71AFE01A8FFF717FE0F48FFF714FECC
:1043D000BC4204F10104E1D10C48FFF70DFEDDE71A
:1043E0000B48FFF709FE03B0F0BD00BF60E1000815
:1043F00038E0000870E100086CE20008A0E1000865
:104400002CEB000884E100084CE0000894E100086F
:1044100078E1000870B50E4605460E481446FFF7D1
:10442000EBFD3046FFF7E8FD0B48FFF7E5FD2846BA
:10443000FFF7E2FD0948FFF7DFFD14B10848FFF779
:10444000DBFD0848FFF7D8FD0748BDE87040FFF7DF
:10445000D3BD00BF10E00008ACE10008D0E10008C7
:10446000E4E100086CE2000818E000082DE9F041E2
:10447000069F044616469846079D11B10B78002BFF
:1044800049D12848FFF7B8FD2046FFF7B5FD26487B
:10449000FFF7B2FD2046FFF7AFFD2448FFF7ACFD64
:1044A0003046FFF7A9FD2248FFF7A6FD4046FFF77B
:1044B000A3FD2048FFF7A0FD3846FFF79DFD55B14D
:1044C0002B7843B11C48FFF797FD2846FFF794FD72
:1044D0001A48FFF791FD1A48FFF78EFD2046FFF7B7
:1044E0008BFD1848FFF788FD2046FFF785FD16482D
:1044F000FFF782FD1548FFF77FFD2046FFF77CFDA3
:104500001348FFF779FD3046FFF776FD1148BDE807
:10451000F041FFF771BD0846FFF76EFD0E48FFF74B
:104520006BFDAEE7ECE1000838E0000844E000086D
:1045300008E2000810E2000818E2000828E200087B
:104540002CE2000838E2000848E2000854E20008C3
:1045500064E2000870E20008C0E600084EF27C2029
:10456000C0F600000321FFF7E7BB00BF10B504460B
:104570004EF21000C0F60000FFF73EFD4EF2802123
:104580002046C0F60001FFF7C1FE4EF2B000C0F6B3
:104590000000BDE81040FFF72FBD00BF70B5064614
:1045A0004EF2100082B0C0F600000D461446FFF730
:1045B00023FD4DF6FC614EF28823C0F60001C0F6E3
:1045C00000033046009301912A462346FFF74EFF31
:1045D0004EF2B000C0F6000002B0BDE87040FFF738
:1045E0000BBD00BF38B505460C46FFF7CFFD28468A
:1045F000FFF7DEFD2046FFF7DBFD4DF6FC60C0F661
:104600000000FFF7D5FD4EF2CC00C0F60000BDE87B
:104610003840FFF7F1BC00BF10B504464EF28C20C5
:10462000C0F60000FFF7E8FC2046FFF7E5FC4EF27D
:104630007010C0F60000BDE81040FFF7DDBC00BF01
:1046400010B50446FFF7A2FD2046BDE81040FFF775
:10465000E3BF00BF4EF2AC20C0F60000FFF7CCBCB9
:1046600008B5FFF7F7FF4EF2CC00C0F60000BDE83A
:104670000840FFF7C1BC00BFF0B50E4683B014463A
:104680001F46089DFFF7DCFF3046FFF791FD4EF215
:104690001000C0F60000FFF7AFFC4DF6FC61C0F65D
:1046A00000013A462B4620460095FFF795FD4EF255
:1046B0001800C0F60000FFF79FFC2046FFF7D8FD6A
:1046C00003B0BDE8F040FFF7CBBF00BFF8B5069DD3
:1046D0000E4614461F46FFF7B3FF3046FFF768FD4E
:1046E000204639462A46FFF795FE2046FFF7C0FDD3
:1046F000BDE8F840FFF7B4BF2DE9F0410F4614467E
:104700009846069E079DFFF79BFF3846FFF750FD32
:104710004EF21000C0F60000FFF76EFC4146324634
:104720002B462046FFF720FE4EF21800C0F6000090
:10473000FFF762FC2046FFF79BFDBDE8F041FFF765
:104740008FBF00BF2DE9F04F83B08B46924699464C
:104750000C9D0D9FFFF774FF1148FFF729FD1148CD
:10476000FFF74AFCDFF8488000242E595BF804006C
:1047700033463E595AF8041059F804208DE8400198
:10478000FFF774FE04340848FFF736FC0C2CECD11C
:104790000648FFF76DFD03B0BDE8F04FFFF760BFBF
:1047A000B8E20008C0E20008CCE2000878E900089E
:1047B000C8E200082DE9F04F05460E46C5B0854811
:1047C0002946934602F004FF33781BB3741C4FF064
:1047D0002008002706E02B2B08BF04F8018C14F8F2
:1047E000013BBBB1252BF6D120460221FBF7BAFDD8
:1047F000A27804F8010C002A00F04485234603F84F
:10480000012B9A781946002AF9D10F7014F8013B50
:10481000002BE7D13146704802F0DAFE3046FFF750
:1048200081FB28466D4906F04AFD002842D0284603
:104830006B4906F044FD0446002800F0CF8328466B
:10484000684906F03CFD002800F07484284666495B
:1048500006F035FD0446002800F0868128466349AD
:1048600006F02DFD002800F06D852846604906F011
:1048700026FD002800F0F68728465E4906F01FFD59
:10488000002800F04D8228465B4906F018FD0028FC
:1048900000F00C875948FFF7AFFB5948FFF7ACFB16
:1048A0005848FFF7A9FB0026FFF758FE304645B0F1
:1048B000BDE8F08F544C18AF3CAD04F1080694E805
:1048C0000300039587E803000FCE0FC596E80300A9
:1048D00023AA04F12006914685E8030007920FCE33
:1048E000A9E80F00366828AD04F1480C06970DF1D1
:1048F000C8082DAFC9F80060049504F1340EE246F3
:104900002E4644463D46BEE80F000FC6BCE80F00E9
:104910000FC5BAE80F000FC4DCF80030DEF8002045
:1049200005942B6016AC059D13A90894326037944A
:1049300014AA12A81AAC0DF1440A2B603A913B92CA
:104940000594CDF8E0A0399002F096FF814602F080
:1049500099FF2E49C0F30742C0F30723059806F0DC
:104960007DFC02F095FF42690446002A54DB03698E
:10497000002B51DBC16800294EDB806800284BDB2F
:104980006568002D48DBB2F5966F45DC0C2B43DCE7
:104990001F2941DC17283FDC3B2D3DDC02F26C7205
:1049A00008981B4906F05AFC226950460132194901
:1049B00006F054FCE26812A8164906F04FFCA26803
:1049C00013A8144906F04AFC14A81249626806F0BC
:1049D00045FC2CE060E4000874E400088CE4000866
:1049E000B4E5000828E700080CE8000894E800088F
:1049F000CCE9000888EA000830EB00087CEB0008EE
:104A0000F8DE000894EB0008F4DD000890E40008EC
:104A10009CE40008A0E4000800238DF858308DF8CD
:104A200044308DF848308DF84C308DF85030964831
:104A3000FFF7AAFA0546002801F05F80934906F0C7
:104A40003EFC002841F02A80914C49269148FFF70E
:104A5000DFFADFF8C8A2FFF73FFB06980221FFF755
:104A600021FC8D484946FFF7BDFDDAF800308B4A3E
:104A70008B498C48002B18BF1146FFF7B3FDDAF8BD
:104A80000030002B41F00480FFF73AFC0398062128
:104A9000FFF708FC8448FFF7D3FD4FF000090595A8
:104AA000DDF820A00394079DDDF810B002E037ABDD
:104AB00059F803A07D48FFF79FFA58F8094055F8C8
:104AC00009005BF8091057F8093052460094FFF7C7
:104AD00083FB09F104097648FFF78EFAB9F1140F48
:104AE000E5D17448039C059DFFF7C2FBFFF7B8FDB5
:104AF000FFF706FC06980221FFF7D4FB6A481E2741
:104B000003466D4A6D490097FFF7B6FDFFF7F8FBC6
:104B10006548FFF781FD6A486A49FFF7F7FB6A4875
:104B20006A49FFF7F3FB59486949FFF7EFFB69480A
:104B30006949FFF7EBFBFFF78DFD44B16748FFF7CD
:104B40005BFA2046FFF758FA6548FFF755FA284602
:104B5000604906F0B4FB0446002800F0F884FFF733
:104B6000F3FBFFF7FBFCA1E65E4B3CAD93E80300D3
:104B7000039585E80300FDF77FFD80464248FFF777
:104B800003FA0546002801F00782574906F097FB13
:104B90000646002801F04E812846544906F08FFB56
:104BA0000646002801F029802846514906F087FB77
:104BB0000546002841F0EC814E48FFF7FFF910F15F
:104BC000000818BF4FF00108CBF800804C260023E6
:104BD0008DF8B4300A24FBF75DFB0DF13200FBF7D2
:104BE00069FB002841F010810A20FBF729FF013CF6
:104BF000F3D144AF3F2327F85C3D02F05DFA3E4914
:104C000082B232A806F02AFB02F05CFA3A4982B27C
:104C100037A806F023FB3948FFF7FAF9FFF75CFAEB
:104C200003980221FFF73EFB35483946FFF7DAFCCF
:104C3000344832A9FFF7D6FC334837A9FFF7D2FC36
:104C40002C4A324B2E493248CDF80080FFF73EFD0A
:104C5000FFF756FB2E48FFF7DFFC23482D49FFF7EF
:104C600055FB22482C49FFF751FBFFF7F3FC002DC1
:104C70003FF475AF1948FFF7BFF92846FFF7BCF9B5
:104C80001748FFF7B9F96AE7A8E40008B0E400089C
:104C9000E4E2000800E500080CE5000898F30008CD
:104CA00034E3000814E50008FCDE000810E000080A
:104CB00018E00008D0E40008F8E400082CE500083B
:104CC000B8E4000834E50008C0E4000840E5000846
:104CD0004CE5000864E5000870E500087CE5000884
:104CE0001CE70008F4DD000814E800081CE80008D0
:104CF00024E8000828E8000830E8000834E8000844
:104D0000A0DF000844E8000848E800084CE8000874
:104D10009CDF000864E800087CE80008A804002084
:104D20003CAD039523AD924A079528AD0495039DAC
:104D300002F150031EAC02F1180702F10C0E02F151
:104D4000240602F1300A07CA84E807000FCB85E881
:104D50000F009EE80700079DDFF878C285E807008E
:104D600097E80700049D0DF1C80885E8070096E85C
:104D7000070088E807009AE80700DCF800300DF12A
:104D8000DC0989E807007B4F53B97B4D3B6A3968E2
:104D90003A69386B85E80E000123E860CCF80030F2
:104DA000FDF7FEFB0690FDF715FC0590FDF720FCD6
:104DB0000890FDF7D1FB00F002000990FDF790FF8D
:104DC0008246FDF759FC0A900DA8FDF73DFF6B48A0
:104DD000FFF7DAF80546002800F01487684906F066
:104DE0006EFA0346002801F07E802846654906F0E9
:104DF00066FA0346002801F0F6802846624906F06C
:104E00005EFA0346002801F0B98128465F4906F0A2
:104E100056FA0646002801F0008328465C4906F051
:104E20004EFA0646002801F0DD822846594907223D
:104E300006F05FFA0646002801F0CB822846564964
:104E4000042206F056FA0646002801F05A83284646
:104E5000524906F034FA0026B34610B9DFF878B1AB
:104E600053267A6B4E4913A806F0F8F94C49059A77
:104E700014A806F0F3F94A49089A16A806F0EEF9C4
:104E8000524647490EA806F0E9F90DF1400A444997
:104E90009DF834200FA806F0E1F911AF40499DF8C4
:104EA0003520504606F0DAF99DF836203C49384660
:104EB00006F0D4F903250FA93A482D91CDF8B8A0F2
:104EC0002F97FFF7A5F8FFF707F920462946FFF7C8
:104ED000E9F935483549364A14AB0095FFF7CCFB64
:104EE000009531483349344A16ABFFF7C5FB099C9E
:104EF0005CB90A9D002D01F01B818DE800032A4852
:104F00000799049A2DABFFF71DFC069F04242B4A3A
:104F1000194B25482A4901940097FFF7EDFBFFF74D
:104F2000EFF921460398FFF7BDF9264D00242B68C1
:104F3000DA0700F1938601341035042CF7D1FFF71E
:104F4000DFF91948FFF768FB14481F49FFF7DEF93E
:104F5000FFF780FBBBF1000F3FF401AE1B48FFF7EA
:104F60004BF85846FFF748F81948FFF745F8F6E5BB
:104F700058DE00082C000020100C0020A8E40008D7
:104F8000BCE80008CCE8000894EA0008A4EA00089D
:104F9000B4EA0008C4EA0008D4EA000818E90008E6
:104FA0002CEB0008DCEA0008C4DF0008F0EA000887
:104FB000A8EA0008F8EA0008B8EA000898EA000839
:104FC00010EB000838000020C0E900087CE500086C
:104FD0001CE70008200C002040E40008AB4A3CAD70
:104FE00002F108030DF1DC0992E80300039589E85A
:104FF000030093E8070085E80700FEF7ABFE0546CF
:10500000A348FEF7C1FF05F10C088246AF680028EF
:1050100000F0E4879F4906F052F90646002800F0A8
:10502000488650469C4906F04AF90646002800F09A
:10503000F4865046994906F042F90646002800F0E9
:1050400008875046964906F03AF9002800F059853D
:105050002646B24604F040FC9249024632A806F0C9
:10506000FDF89148FEF7D4FFFFF736F803980321C7
:10507000FFF718F905F13C018C48FFF7B3FA4146F8
:105080008B48FFF7AFFA8B48FFF7DAFA8A48FFF749
:105090008FF88A48FEF7B0FF4FF00F08884849465E
:1050A0003A460223FFF760F905F11C0285492023E7
:1050B0008548CDF80080FFF78FF814258348FEF768
:1050C0009BFF8349834A402383480095FFF784F878
:1050D0008248FEF791FF8248FFF7CAF8FFF7C0FA4F
:1050E00004F01CFC032503467E4972487E4ACDF835
:1050F0000080FFF7C1FA7D497D4A32AB6D480095CB
:10510000FFF7BAFAFFF7FCF86A48FFF785FA644838
:105110007849FFF7FBF8FFF79DFA002C00F00882B2
:105120007548FEF769FF2046FEF766FF7348FEF7F5
:1051300063FF14E5724B0DF1C80893E8030088E89B
:1051400003005348FEF720FF0446002800F0EC84DB
:105150006C4906F0B4F80646002800F04B8620465D
:10516000694906F0ACF80646002800F09F86204604
:10517000664906F0A4F8002840F0D684644D57260E
:10518000644B1B68002B00F0608504F0C1FA0DF140
:10519000DC09044662084846424906F05FF8E70722
:1051A00000F1AF86484606F09CF85B4B09EB000225
:1051B00001469C8818689B7949F801009480937196
:1051C000564B1B68002B00F0378504F0C1FA3CAF4A
:1051D0000446620838463349039706F03FF8E4076F
:1051E00000F19C86039806F07CF8039C4A4B221839
:1051F000039F01469C8818689B797850948093712E
:1052000004F076FA0246002840F0758544AF07F8AE
:105210005C0D04F0EDFA0246002840F0648544ACD1
:1052200004F8700D04943E48FEF7F2FEFEF754FFBA
:1052300040460221FFF736F83A484946FFF7D2F9CF
:10524000022439480399FFF7CDF938483849394ADB
:105250003B460094FFF710FA3749384A049B33481D
:105260000094FFF709FAFFF74BF83048FFF7D4F93D
:1052700026483349FFF74AF8FFF7ECF9002D7FF491
:10528000F9AC6CE421460F70FFF7C0BA50DE00089D
:10529000A8E40008C0E500085CE600086CE6000829
:1052A0007CE600082CEB0008E0E5000884E6000836
:1052B00090E6000880DF0008A4E6000810E000087F
:1052C000CCE50008ACE60008D8E50008B4E6000824
:1052D000C8E60008FCDE0008A4F4000818E0000896
:1052E000C4E50008CCE6000860E60008D8E600083F
:1052F00070E60008ECE60008FCE6000818E7000885
:10530000F4DD000838E7000848E7000858E700081F
:10531000F8E300085813002070E700089404002008
:1053200078E7000890E70008A0E7000894E7000885
:10533000A8E700083CE70008D0E700084CE70008B1
:10534000F8E70008AF4B23AC07943CA803F10C0E20
:1053500003F1240503F13004039003F1180693E8E8
:10536000070028AF079B049783E807009EE8070023
:10537000049B2DAF0DF1DC0983E8070096E80700D8
:1053800087E8070095E8070089E8070094E8070028
:10539000039C84E80700FDF739F90990FDF7DCF874
:1053A0000546FDF7BDF90A90FDF772FC8046FDF752
:1053B00063F9954C0B9014A8FDF722FC236805F0C7
:1053C0000102C5F3400A069253B9904A9048191851
:1053D00049680833902B42F8041FF8D10123236059
:1053E0008C48FEF7D1FD0446002800F0EF858A497D
:1053F00005F065FF002800F05E832046874905F030
:105400005EFF002840F095858548FEF7D7FD00280F
:1054100000F00D86012045F002050590CBF8005004
:10542000472620467F4905F04AFF0546002800F040
:105430004E8520467C4905F042FF002840F09785C4
:10544000DFF860A2DFF860B2582616AC4246774912
:105450000DF16008204608941AAD05F0FFFE73496F
:105460009DF85020404605F0F9FE1CAC6F499DF8B0
:105470005120284605F0F2FE9DF8522020466B4947
:1054800005F0ECFEDBF80020CDF8C88033953494AD
:10549000002A40F0158544AC04F8982D6448FEF7C6
:1054A000B7FDFEF719FE07980321FEF7FBFE069DE8
:1054B00060486149614A624B0095FFF707F9099D11
:1054C0005C48009512255F495F4A604B0195FFF7E4
:1054D00013F9059D574800955D49514A5D4BFFF70B
:1054E000F5F80B9D002D00F0C3840A9D002D00F0FF
:1054F000D18423460224584A58494E480094FFF765
:10550000BBF8FEF7FDFE4B48FFF786F854485549B7
:10551000FEF7FCFE54485549FEF7F8FE4248544950
:10552000FEF7F4FE53485449FEF7F0FEFFF792F8F9
:10553000BAF1000F3FF413AB5048FEF75DFD504643
:10554000FEF75AFD4E48FEF757FDFFF708BB4D48E2
:10555000FEF752FDA0461CAD1EAC42464A49284605
:1055600005F07CFE2846FEF747FD4848FEF744FD5F
:10557000404621461022FEF79FF800283DD0002724
:105580000DE0E25D4249284605F068FE2846FEF738
:1055900033FD01373F48FEF72FFD102F0AD007EBF0
:1055A0000803B3F5A27F3C48EBD90137FEF724FD91
:1055B000102FF4D13748FEF71FFD002320212E20A5
:1055C00003EB0802B2F5A27F88BFE15404D8E25C85
:1055D000203A5E2A88BFE0540133102BF0D100231B
:1055E00020468DF8883008F11008FEF705FD2B489D
:1055F000FEF702FDB8F5A87FAFD12948FEF7FCFC05
:10560000FFF7ADBA58DE0008A80C0020C40B00203C
:10561000A4DC0008A8E40008A0E80008ACE8000842
:10562000B0E80008FCE800080CE900082CEB0008D2
:1056300020E9000810E9000834E90008A4E800089F
:105640003CE900085CE90008F0E80008C80B00200D
:10565000D0DF00086CE9000800E9000898E90008BC
:10566000B8E4000834E50008C0E4000840E500089C
:10567000B0E9000818E90008C0E900087CE5000866
:105680001CE7000894E500089CE50008A4E5000874
:1056900080F20008E0E10008B0E5000874DF0008CF
:1056A000A8E500082CE400085C040020B44D3CACE4
:1056B00003940FCD0FC495E80F0084E80F00B148A4
:1056C000FEF762FC044630B1AF49062205F011FE38
:1056D000002800F02D82DFF834B30DF1DC09AB486F
:1056E000FEF796FC23ACFEF7F7FC03980821FEF7C3
:1056F000D9FD18AD07941AAC4FF0000A0695059431
:1057000028AD1EAC049556462DAF0DF1C8081CAD52
:1057100003940BEB0A0CDCF8042048F68904C8F665
:105720008804A4FB02029A4952090598CDF808C0E2
:1057300005F094FDDDF808C09549DCF80420A4FBD1
:1057400002035B09C3EB0313A2EB8302284605F0B7
:1057500085FD9048FEF774FF32468F49069805F0A4
:105760007DFD32468D49039805F078FD32468C491F
:10577000079805F073FD32468A49049805F06EFDDE
:1057800032468949384605F069FD32468749404628
:1057900005F064FD0698FEF70BFD5BF80A200798FC
:1057A0008349C2F3C012FEF735FE5BF80A20804938
:1057B000C2F380120498FEF72DFE32467D4948461A
:1057C00005F04CFD5BF80A207B48C2F3C204FEF7EB
:1057D00013FC0723224679494846FEF7C5FD784861
:1057E000FEF70AFC32467749484605F037FD5BF87C
:1057F0000A20714802F00704FEF7FEFB2246072349
:105800006E494846FEF7B0FD6D48FEF7F5FB0224F1
:105810006948FEF7F1FB6649059A2346384600942D
:10582000FEF7DAFC6648FEF7E7FB6348FEF7E4FBA9
:105830005F492A46234640460094FEF7CDFC604867
:10584000FEF7DAFB01360398FEF712FDFEF708FFBC
:10585000082E0AF1080A7FF45CAFFEF751FD00261E
:10586000FFF77DB9DFF8A8E13CAF3E460EF13C04FE
:105870000DF1C8089EE8070088E807000FCC0FC6A6
:10588000514D039724682F680DF1DC090EF1500E7D
:105890009EE80F00346089E80F00002F00F01B81A4
:1058A0004A4EFCF705FF0746FCF73AFF0546354828
:1058B000FEF76AFB0446002800F0B683444905F071
:1058C000FEFC8246002800F0BA822046414905F0DD
:1058D000F6FC8246002800F0698320463E490322F8
:1058E00005F007FD8246002800F0668420463B490B
:1058F000062205F0FEFC8346002800F0A384204623
:105900003749072205F0F5FC0646002800F0908490
:1059100020463449042205F0ECFC0646002800F03D
:105920004A852046304905F0CAFC0026B24610B927
:10593000DFF8E0A053262D48FEF76AFB0B24FEF7A4
:10594000CBFB40460321FEF7ADFC294829492A4AF2
:105950002A4B019400970224FEF7CEFE2849294ADB
:10596000294B234800950194FEF7C6FEFEF7C8FCBC
:1059700003980521FEF796FC144D002451E000BF6A
:10598000B8DE0008A8E4000838EB000850EB000877
:10599000A0E40008DCDF00082CEB000864EB000842
:1059A0006CEB000870EB000874EB000878EB000863
:1059B000FCDE000848EB000810E0000800000020B2
:1059C00018E000084CEB0008240C002078000020B0
:1059D000D8E90008E8E90008FCE9000800EA000846
:1059E00018EA000828EA000818E9000830EA000868
:1059F000ACDF000848EA0008DCE900089C0B002046
:105A000054EA0008ECE90008AC0C0020D43900206E
:105A100058DE000840E40008013414350B2C00F077
:105A2000F5802B69D807F7D52246B64918A805F0A6
:105A300015FC2246B4491AA805F010FC2246B349C9
:105A40001CA805F00BFC2246B1491EA805F006FC77
:105A5000AA68B04916A805F001FCAF48FEF7F0FDB2
:105A60002868FEF7A5FB16A91AA8AC4AFEF796FD12
:105A70001CA8FEF77BFD2A69A949C2F340021EA8B3
:105A8000FEF7C8FC18A8FEF7F3FBFEF7E9FDC3E735
:105A9000A4480599FEF7A6FDFEF7F6BF2846A249E1
:105AA00005F00DFC002832D10123CBF80030502640
:105AB0009E4CFEF7CBBF9E48FEF780FA002800F010
:105AC0005282012345F001050693CBF80050CDF832
:105AD00014A04726A5E4974A974E3B46995914339C
:105AE000DC2B42F8041FF9D1944B95491A681B69C5
:105AF00081E80C0001232B60D3E606460446FEF73E
:105B0000A5BFDFF894A24E260446FFF7A3BA2846A5
:105B10008C4905F0D4FB002840F01C83CBF8000032
:105B20005026894CFEF792BF00263546FFF728BB6A
:105B3000A01D05F04DF8072804463FF6CCAD014600
:105B40008248FEF749FA824905F0B9FB002800F0C7
:105B50005983DFF848B25BF8343023F080034BF808
:105B6000343021467B48FEF737FA794905F0A7FB28
:105B7000002800F040835BF8343023F040034BF8FA
:105B800034300DF1DC0922467349484605F066FBC6
:105B90004846FEF7F9F905F01BF822466F4905461D
:105BA000484605F05BFB4846FEF7EEF905F010F8B5
:105BB0005BF83430ED0000F0070023F03F0340EACB
:105BC000030205F0380313434BF834302146644890
:105BD000FEF702FA04F0FCFF214605466148FEF795
:105BE000FBF904F0F5FFC5EB05150BEBC40400EB66
:105BF0008500606003F04AF871E501F085FA5A4DBE
:105C0000FEF7E5BF06468346FFF72BB9FEF778FBA4
:105C100048460421FEF746FB544D00242B68D90763
:105C200000F1BE8001341035022CF7D1FEF768FB7D
:105C30003948FEF7F1FC75E44D4B3CAC93E80300AA
:105C4000039484E80300FFF7DBBA494B0DF1DC094C
:105C500093E8030089E80300FFF7B2BA22464549FA
:105C600018A805F0FBFA224643491AA805F0F6FAEF
:105C7000224642491CA805F0F1FA55F8082C25499E
:105C800012A805F0EBFA3E48FEF7DAFC55F80C0CCA
:105C9000FEF78EFA12A93B4A1AA8FEF77FFC1CA851
:105CA000FEF764FC18A8FEF7E3FAFEF7D9FCFFF74D
:105CB00042B93548FEF768F904F08AFF07463348D1
:105CC000FEF762F982463248FEF75EF90446002F7D
:105CD00000F0B28105F005FB092800F2C7812D4CC8
:105CE000B246FFF7B7B928AC20460A49049405F03C
:105CF000B5FAFFF798BA2DAF3846064905F0AEFA67
:105D0000FFF787BA64EA000808EA00086CEA0008AE
:105D100010EA00082CEB0008ACDF000874EA000869
:105D2000FCDE00081CE50008B8E4000804E30008F5
:105D3000A4E80008980B00207800002070010020E3
:105D4000AC0C0020C0E400081CE3000840EB000895
:105D5000D8DE000844EB000848EB00084CEB0008D4
:105D6000E8E400087CEE000814E400087C01002050
:105D700034E3000820EB0008CCEA000828EB000818
:105D8000C4DF000894E90008CCE50008D8E5000865
:105D9000A4F400083CE30008E4E30008D439002040
:105DA0002246BF4923A805F059FA2246BD4928A832
:105DB00005F054FA2246BC492DA805F04FFA55F8D3
:105DC000082CBA4914A805F049FAB948FEF738FC7E
:105DD00055F80C0CFEF7ECF914A9B64A28A8FEF702
:105DE000DDFB2DA8FEF7C2FB23A8FEF741FAFEF764
:105DF00037FC17E7B048FEF7C7F804F0E9FE03F0F8
:105E00007DFC3546FFF7BCB92DAF3846AB49BDF830
:105E1000322005F023FAFEF7F0BEA948FEF7B4F8E9
:105E200003F082FD002800F0BB803446DFF8E8A2D2
:105E3000FFF710B901F04CF9A24DFEF7C8BEA24819
:105E4000FEF7A2F804F0C4FE41260746CBF8000096
:105E500071E59E48FEF798F804F0BAFE03F042FDA3
:105E6000002800F0AD803446DFF8B0A2FFF7F2B8AA
:105E70009748FEF7E5FB9748FEF79AF908998D4A8F
:105E80009548FEF78BFB9448FEF7F2F9FEF7E8FB26
:105E9000FFF72BBB039DCDF8009001958C4804992A
:105EA0003A4632ABFEF74EFCFFF723BB8B48FEF7BA
:105EB0006BF804F08DFE03F0A1FC3546FFF760B9E6
:105EC0001EAC2046794905F0C9F9FFF7E7BA8448C6
:105ED000FEF75AF804F07CFEDFF844B2AA46CBF88D
:105EE0000000FFF7B2BA7C480293FEF74DF804F0C9
:105EF0006FFECBF80000029B824662269B46FEF7AF
:105F0000B0BF484605F0EDF9764B09EB0002198861
:105F10009B7829F800109370FFF744B9039805F0B7
:105F2000E0F9704B3A1819889B7839529370FFF753
:105F300059B920466C4905F0C2F9002800F04E819D
:105F400020466A4905F0BBF9002800F0B2812046DE
:105F5000674905F0B4F9002800F05D81CDF814A080
:105F60000026FFF75EBA25F001050690ADE5204654
:105F7000604905F0A4F9002840F00E810123CBF818
:105F800000305026DFF89CA1DFF894B1FFF75DBA2E
:105F900026462546FEF71BBE06460546FEF717BEFB
:105FA00006460446DFF880A1FFF754B85248FDF7D3
:105FB000EBFF04F00DFE46260546CBF80000BAE4E0
:105FC00006460446DFF864A1FFF744B8CDF814A0F4
:105FD00006468246DFF848B1FFF737BA0646044660
:105FE0008246FFF737B845480293FDF7CDFF04F02E
:105FF000EFFD8DF834004248FDF7C6FF04F0E8FDE0
:106000008DF835003F48FDF7BFFF04F0E1FD8DF846
:1060100036000D9A6326110CABF800208BF80210A5
:10602000029B9B46FEF71DBF0646824683E425F091
:1060300002050590FFF7F2B93348FDF7E9FF334851
:10604000FDF7DAFFFEF780F9FEF788FA4FF4FA70F1
:10605000FAF7F6FC2E4B6F6085F83C7050462146EF
:106060001F603E46FDF7A2FEFEF720BC2648FDF766
:10607000CFFF2848FDF7C0FFFEF766F9FEF76EFA7E
:106080004FF4FA70FAF7DCFC214B6E6085F83C6047
:10609000504621461E60FDF7A1FEFEF707BC00BF7B
:1060A00078EA000820EA000880EA00082CEB0008E3
:1060B000ACDF000894E900083CE7000830E800087D
:1060C00060E6000814E40008DCE9000870E6000857
:1060D00010E9000880E90008E8F700084CE700082C
:1060E00000E900086CE70008BCE80008CCE80008FC
:1060F000ECE80008B8E40008ECE90008D8E800087B
:10610000DCE80008E4E80008E0E50008F4E5000841
:106110007812002028E600085CE30008A4E30008E9
:106120005C04002004E3000880E30008C4E30008E6
:10613000BF48FEF785FABF48FEF73AF80EA9BE4AF7
:10614000BE48FEF72BFABD48FEF792F8FEF788FA34
:10615000FEF7D3BE2846BA4905F0B1F809900028E9
:1061600000F0C7802846B74905F0A9F80446002882
:1061700000F0168100263446FEF768BCB248029350
:10618000FDF702FF04F024FDCBF80000029B06900F
:1061900064269B46FEF765BE2046AC4905F08FF8A5
:1061A000002840F02A81CBF800005026DFF8ECA24E
:1061B000DFF8ECB2FFF749B9E01C04F009FD0A284A
:1061C00084BF5646B2463FF6B6AB00EB800006EB06
:1061D0008003DA6856469A60FFF7ADBB9748FDF733
:1061E000D3FE04F0F5FC42268046CBF80000CDF843
:1061F00014A0FFF716B95BF8343043F040034BF8B6
:106200003430BEE4DFF89CB25BF8343043F08003F6
:106210004BF83430A5E48E48FDF7B6FE04F0D8FC08
:1062200044260990CBF80000CDF814A0FFF7F9B888
:10623000E01D04F0CDFC0128044640F24E81B24638
:10624000FFF779BBA01D04F0C3FC0A2888BF5E4697
:10625000824688BFB2463FF66EAB7E4952461EACC0
:106260001AA804F0FBFF52467B49204604F0F6FFD3
:106270001AA8FDF789FE04F0ABFC431E0E2B4FEA73
:106280008A0B9EBF0BEB0A0306EB83039860204644
:10629000FDF794FE0BEB0A0306EB83031A69002853
:1062A00000F00281002642F002021A61B246FFF7B6
:1062B00042BB6A48FDF768FE04F08AFC8DF8500086
:1062C0006748FDF761FE04F083FC8DF851006548D6
:1062D000FDF75AFE04F07CFC8DF85200149BCDF8BB
:1062E00014A01A0CABF800308BF802204326FFF7FD
:1062F00098B85D48FDF748FE04F06AFC06465B4826
:10630000FDF742FE04F064FC034659480293FDF792
:106310003BFE04F05DFC04465648FDF735FE04F0F4
:1063200057FC0A905448FDF72FFE04F051FC32460A
:106330000B905249089804F091FF029B50491A466D
:10634000504604F08BFF22464D4912A804F086FF08
:106350004B490A9A13A804F081FF49490B9A14A8E3
:1063600004F07CFF029BA6F26C715A1E0A98CBF8CF
:106370001C10CBF810200B99099ACBF80C40CBF8E5
:106380000800CBF80410CBF800202046324619460E
:10639000F9F7AEFF5426CBF81800099CFEF756BB60
:1063A0003848FDF7F1FD1E220146584604F0BAFFB9
:1063B0007026FEF74BBB201D04F00AFC01283FF6B7
:1063C0003EAF314BB24603EB00139A685A60FFF7B9
:1063D000B2BAE81D04F0FCFB032805466BD9B346AE
:1063E000FEF73FBD2948FDF7CFFD04F0F1FBFCF7B8
:1063F00005F9B3460890FEF734BD2046244904F061
:106400005EFF244B00280CBF9A464FF0000ADFF8CD
:1064100090B008BF5326FFF718B81F48FDF7B4FD2A
:1064200004F0D6FBFCF7DCF8B3460590FEF719BD87
:10643000C4DF000880E9000894E90008E8F70008D4
:10644000CCE40008F4E4000898EA0008C0E400087E
:10645000F0E8000808EA000810EA0008D8E8000898
:10646000DCE80008E4E80008DCE40008E4E40008F4
:10647000ECE4000894F70008F0E400089CE400084D
:10648000A0E40008F8E4000870010020B8EA000861
:1064900018E9000840E40008A8EA00081CE3000826
:1064A0005C040020D439002022F0020206461A6162
:1064B0008246FFF740BA024618491AA804F0CEFEF9
:1064C0001AA8FDF761FD04F083FB0F2887D807EBBE
:1064D00005156860B346FEF7C4BC0246104928A8FB
:1064E00004F0BCFE28A8FDF74FFD04F071FB0F2857
:1064F0003FF6A5AE0B4BB24603EB04146060FFF70A
:106500001ABA281D04F064FB03283FF668AF07EBB6
:1065100000139A68B3465A60FEF7A3BCCCEA0008A1
:1065200020EA00087001002030B585B04FF48044A7
:10653000684603F019FF0022200448F2A063C0F26D
:1065400001030121ADF80420ADF8082040F4A84073
:106550004FF480624BF6FF75ADF80650ADF80A2097
:10656000ADF80C40009303F00DFF200440F4A84068
:10657000694603F089FE05B030BD00BF10B54FF489
:10658000A844C4F200042046012103F017FF20466E
:10659000012103F03FFF2046002103F03BFF20468E
:1065A00003F052FEBDE81040FFF7BEBF70B50546D0
:1065B0000E4643F2010401E0013C13D04FF4A84021
:1065C0002946C4F2000003F033FF0028F4D04FF452
:1065D000A840C4F20000314603F02AFF0028EBD0A7
:1065E000012070BDFFF7CAFF204670BD38B50546D3
:1065F00019B1BDE83840FFF7D9BF43F2010401E00B
:10660000013C0AD04FF4A840C4F20000294603F030
:106610000FFF0028F4D0012038BDFFF7AFFF204660
:1066200038BD00BFF8B507464FF4A840C4F20000DB
:106630000E46012115461C4603F0B2FE0120C1F2B0
:1066400000000021FFF7D2FF002832D04FF4A8400D
:10665000C4F2000034BB012103F0BEFE4FF4A84495
:10666000C4F200042046F9B2002203F0C9FE022061
:10667000C1F200000021FFF7B9FFB8B18020C1F2DC
:1066800000000021238BFFF7B1FFA8B125B1C6F3AD
:106690000721204603F0AEFE2046F1B203F0AAFE29
:1066A0000020F8BD002103F097FED7E76FF001004E
:1066B000F8BD4FF0FF30F8BD6FF00200F8BD00BF2D
:1066C00030B51A4B83B01C680CB103B030BD012546
:1066D00001A81D6003F068FD29464FF4001003F087
:1066E0003DFF0820294603F02BFF0820294603F030
:1066F00027FF29464FF4001003F03EFF21464FF4D8
:10670000001003F039FFC023ADF804304FF44060AF
:106710001C23C4F2010001A98DF8073003238DF872
:10672000063003F0DDFCFFF7FFFECEE7B80C0020DB
:106730002DE9F041069D1E466F1E7B427B4180463F
:10674000FFF770FF074610B13846BDE8F0818020A2
:106750000421C1F20000C1F20001FFF727FF002869
:106760005BD04FF4A844C4F200042046012103F09A
:1067700017FE0120C1F200003946FFF737FF00285D
:106780004ED020465FFA88F1012203F039FE022044
:10679000C1F200003946FFF729FF002843D0238BC0
:1067A0008DB33C4611E040200021C1F20000FFF70C
:1067B0001DFF18B34FF4A840C4F2000003F01CFE04
:1067C0003219AC4202F8010C1DD00134AC42EAD1BE
:1067D0004FF4A840C4F20000002103F0FDFD4FF487
:1067E000A840C4F20000012103F0E8FD4020002190
:1067F000C1F20000FFF7FAFE0028DBD16FF00607B8
:106800003846BDE8F0814FF4A840C4F200000121F1
:1068100003F0E2FD3846BDE8F0816FF0030793E72F
:106820006FF0040790E76FF005078DE770B51C4621
:106830000023FFF7F7FE064608B1304670BD802002
:10684000C1F200003146FFF7D1FE28B3049BD3B15B
:10685000049BE51801E0AC4215D04FF4A84014F8B1
:10686000011BC4F2000003F0C5FD80200421C1F229
:106870000000C1F20001FFF799FE0028EBD16FF094
:106880000306304670BD4FF4A840C4F20000012159
:1068900003F094FD304670BD6FF00206CDE700BFF7
:1068A00070B43A4A3A49546A0B689C4215D8956AC2
:1068B000AB4212D2D56B002D52D01C1B00FA04F44F
:1068C000344D2E6826432E601268032A32D0052AE2
:1068D00015D001330B6070BC7047D46A2B4DA342B6
:1068E000F2D32E6BB342EFD2ED6B002D3ED01C1BCA
:1068F00000FA04F4284D2E6826432E60E4E7A3F145
:106900001402032A23D9A3F11804032C34D800FA63
:1069100002F2224C25681543256003F0070201248A
:1069200004FA02F458BB1E48DA08855C25EA040420
:106930008454CEE7102BCCD9142BCAD8A3F1110460
:1069400000FA04F0174A146804431460C1E7A3F185
:10695000080500FA05F5104A14682C431460DCE7BA
:106960000C4C256840EA45052560ADE70A4C2568D2
:1069700040EA45052560A7E72F2BAAD8CDE70848B0
:10698000DA08855C2C438454A3E700BFE80C0020A0
:10699000D00C00202C0D0020480D0020440D0020BC
:1069A000C00C00203C0D002000B583B001A803F00E
:1069B000FBFB0820012103F0C3FD0823ADF80430E0
:1069C0004FF4406002238DF80630C4F20100042326
:1069D00001A98DF8073003F083FB03B000BD00BFB1
:1069E000F0B4294A1368002B2BD028490B68022BDE
:1069F00017D0032B264B26D0264C0F682168264D36
:106A0000A0F801101E680021A0F803602E6807702E
:106A10001960467121600120296000231360F0BCD9
:106A200070471B4B1D681C68E443E4B2B4EB152FA0
:106A30001BD0184C48F2EE752668AE421AD00020E2
:106A4000EBE71846EBE71D681C68E443E4B2B4EBDF
:106A5000152FF4D11C68E4B21C60104C26681D6828
:106A60000C4C45EA06251D60C7E71D68094CEDB2D0
:106A70001D60C2E70B250D601D68C5F30725256065
:106A80001D68EDB21D60B8E74C0D0020E40C00203D
:106A9000CC0C0020340D0020380D0020D40C002038
:106AA0002DE9F0474FF440609E4CC4F201000821EC
:106AB00003F082FB236893B99B4E356895B99B4BD5
:106AC000002800F0C2801B68002B40F00C81984B1E
:106AD0004FF6FE711A688A4201D801321A602068A6
:106AE000BDE8F087934F3A68002A70D0002800F084
:106AF000B280914A11780131C9B2E929117000F2CE
:106B000006818E4B8E495A6B09688A42E7D1996B90
:106B10000029E4D1DFF868828A49D8F800C00D68FE
:106B2000AC4500F079818848002707601B68012B7D
:106B300000F06581052B00F07A810A2B18BF292B04
:106B400003D10068C00700F156810120022B2060AC
:106B500040F09C81002A40F0028275480368B3F53A
:106B6000E16F80F01682794D794FD5F800903B683F
:106B7000DFF8F4A149F00109C5F80090CAF8003027
:106B8000C1F800C002606546724A02201060724A75
:106B90003B601360714B1A68714B1D60714B1A603A
:106BA000236863B10B689C4500F0BA816E4A604867
:106BB0001568674FC8F8003000233D6003605B4AEA
:106BC000002313605C4A33600B60137087E7674FE4
:106BD0003B68002B00F08180584B002840F0D280A9
:106BE0001A68032A00F05581DFF84C81DFF83C91E8
:106BF0005A68D9F8001051488A420BD882689142ED
:106C000008D898F800C0C268944503D30269944537
:106C100040F2B3815B69494A99420BD39369994227
:106C200008D898F80010D369994203D3136A99429F
:106C300040F2A9810025356088F800500123C9F889
:106C40000030002D3FF44BAF5BE71A6801321A6049
:106C50002068BDE8F087DFF8D490DFF8DC80D9F851
:106C60000030A3F11F020A2A17D898F80020052A3D
:106C700013D90A2A11D83E493048442204F004F8B6
:106C80002F4A002313600122C9F8002088F8003041
:106C90003B60002D3FF423AF33E7A3F15E02532A9C
:106CA00008D898F800202D2A00F2A080162A01D9D1
:106CB0003049E1E7A3F13C020F2A40F28A80283BE9
:106CC000162B00F2908098F80030122B40F28B8047
:106CD0001F2B00F288802849CEE7E8B9134B1A68C9
:106CE00001321A600DE7134A012313601F4AFF2186
:106CF0001560144A336015601B4A15601F4A156001
:106D0000164A15600E4A11600B4A1370E7E60749F0
:106D100033600B601370E2E6074A01233B60137097
:106D2000EFE600BF4C0D0020C80C0020400D0020F5
:106D3000D80C0020BC0C0020DC0C0020E80C00204B
:106D4000D00C0020480D0020300D0020380D002010
:106D5000A0010020E40C0020340D00203C0D002098
:106D6000CC0C0020D40C00202C0D0020E00C0020C6
:106D700034EC000800ED000878EC0008440D002019
:106D80009C0100208B49D3F83490D1F800C0E14534
:106D900000F09080DFF850821A6898F800A0012A6D
:106DA0000AF1010A5FFA8AFA834888F800A000F025
:106DB0009980BAF1E90F7FF644AF09F1FF329445AB
:106DC00000F0C3807D4A00233360136088F80030F0
:106DD00085E698F800203B2A7FF671AF4B2A3FF6F4
:106DE0006EAF774948E70025356049E7592A3FF6F5
:106DF00061AF744940E7744800230360D0E602683D
:106E0000013A012A88BF2360F5D9704A7048126898
:106E10000360704B1A60BDE66B480068B0F5966F72
:106E2000BFF481AE6C480768013707607EE60368EF
:106E3000012BE0D001232360684B1F7858789A78A3
:106E400087EA000909F00F0989EA171787EA101085
:106E500002F00F09814501D000202060D8781F7909
:106E60004240587982EA0703984201D00023236008
:106E70005B4B5C4A1F681068544A38431860544B97
:106E8000052018601268534B1A6083E6052BD3D097
:106E9000BBE748490A68102A7FF4A6AEDFF81C91C8
:106EA000D9F80020053A072A79D94F4B306018707D
:106EB0000546C3E6986B01287FF46CAFDFF8FC90C1
:106EC0005869D9F80010884205D89869814298BF5E
:106ED0009A637FF6B6AE444A00233360C9F80030A7
:106EE0001370FCE5BAF10B0F7FF6ABAEBCF10A0FE5
:106EF0007FF65FAFDFF8D490C16AD9F80020ACF11B
:106F00000B0A614442EA0A220CF1010C0131C9F872
:106F100000200A22C0F834C0016388F8002065E62A
:106F20002A48324F05683A682748AA427FF442AEA1
:106F3000026840F6C90C62459FBF294AD2F800C0DA
:106F40004CF0010CC2F800C034E69B6B002B7FF4C0
:106F500039AFC1F80090002D3FF4C1ADD1E51B4B16
:106F6000224F1B6810E60A200F3A202118601020DB
:106F70000F2AD8621963596305D80120FFF790FCE6
:106F800000233B605AE60020FFF78AFC00233B60A9
:106F900054E6174B154F1A600C4B1B68F4E5124A68
:106FA00012783B2ADFD94B2ADDD800233B6011231E
:106FB0000B6043E6D00C0020E80C0020400D0020C0
:106FC00044ED0008BCEC0008D80C00202C0D00207B
:106FD000E40C0020340D0020300D0020C00C0020F7
:106FE000380D0020440D0020DC0C0020A001002002
:106FF0004C0D0020F9F74EB910B582B004460DF1E2
:107000000600F9F757F978B1084B09491B88BDF814
:1070100006200988D21AC2EB0212CB1A92FBF3F3B4
:107020000F2B28BF0F23236002B010BD500D00208E
:10703000520D002008B50F4B1B686BB1FF23C0F247
:10704000020398420AD80C4B00221A800B4B40F2E4
:10705000FF321A80012008BD184608BD02220649E9
:10706000E120FCF729FBE32004490222FCF724FB82
:10707000012008BDA8040020500D0020520D002062
:1070800008B50A4B1B680BB9002008BDE120084970
:107090000222FCF72BFB0028F6D00222E320054950
:1070A000FCF724FB003018BF012008BDA804002015
:1070B000500D0020520D002040F65053C2F2000344
:1070C0001888704740F65253C2F200031888704780
:1070D00010B582B0F9F7DEF80A240DF10600F9F7D1
:1070E000E9F840B90A20F9F7ABFC013CF5D1054CB1
:1070F000208802B010BD034CBDF806302380FFF796
:10710000BFFFF5E7500D002010B582B0F9F7C2F8C7
:107110000A240DF10600F9F7CDF840B90A20F9F775
:107120008FFC013CF5D1054C208802B010BD034C0A
:10713000BDF806302380FFF7A3FFF5E7520D0020CE
:10714000F9F738B8F0B507468DB00A20FCF7ACFC6B
:10715000092828D00A2813D0072803D00024204665
:107160000DB0F0BDFCF7F6FD0A2201A900F5B670DE
:1071700004F006FA0146384602F0E8FB7424EEE714
:10718000FCF7E8FD00F14C042021204604F08AF8C9
:10719000014610B1002301F8013B20463A46FDF7B5
:1071A00009FB0446DBE7FCF7D5FD01AE00F5A6744C
:1071B000002502E002340A2D12D023782046022155
:1071C000002B7BD06378002B78D0F9F7CBF8A3782D
:1071D0000135202B46F8040FECD103340A2DECD1F5
:1071E000029CA4F141032F2BB8D801A252F823F03E
:1071F000B1720008B17200080B730008B172000888
:107200005D710008B1720008B17200085D7100087C
:107210005D7100085D7100085D710008B1720008C1
:107220005D710008C57200085D710008B172000848
:107230005D7100085D710008C5720008E572000804
:107240005D7100085D710008C57200085D7100087D
:107250005D7100085D7100085D7100085D710008D6
:107260005D7100085D7100085D7100085D710008C6
:107270005D710008B17200080B730008B17200085C
:107280005D7100085D7100085D7100085D710008A6
:107290005D7100085D7100085D7100085D71000896
:1072A0005D7100085D7100085D710008CD72000815
:1072B000022D7FF453AF039B3B6050E7002D3FF45A
:1072C0004DAF8DE7012D7FF449AF48E720233846C5
:1072D00000F8013B0DF109011E2204F023F8002300
:1072E000FB773CE7072D7FF439AF039B03F1640282
:1072F000049B7A61013B3B61059BFB60069BBB6085
:10730000079B7B60089B3B6029E7042D7FF426AF39
:10731000039B3B70049B7B70059BBB701FE700BF0A
:1073200030B53B4B87B01A68044682426DD0684640
:107330001C6002F039FF02A803F0AEFA042001211C
:1073400003F0FEF80420012103F0FAF84FF4804026
:10735000012103F0F5F84FF400734FF400600325AA
:10736000C4F201006946ADF8003018238DF80330EF
:107370008DF8025002F0B4FE4FF480634FF40060C9
:10738000C4F201006946ADF8003048238DF803309F
:107390008DF8025002F0A4FE4FF46050C4F20100D8
:1073A000012103F0B7FA00234FF460501D46C4F2E8
:1073B000010002A9ADF80C30ADF80E30ADF8103078
:1073C000ADF814300C23ADF81230029403F0FEF93E
:1073D0004FF46050C4F20100012103F069FA4FF448
:1073E0006050C4F2010040F22551012203F06EFA10
:1073F00025238DF8043001A801238DF805508DF860
:1074000006508DF8073002F075FC07B030BD00BFA4
:10741000540D002030B40F4A13687F2BFCD80E495E
:107420000E4D0B685C1C7F2C45F8230098BF0C6048
:1074300001D900230B6072B613680133136062B682
:107440004FF46050C4F2010040F22771012230BCB9
:1074500003F03CBA640F0020680F00205C0D002090
:1074600010B50446007828B1FFF7D4FF14F8010FD7
:107470000028F9D110BD00BF30B40D4B1A6882B19D
:107480000C490D4D0A68541C802C55F8225018BF29
:107490000C6009D072B61A68013A1A6062B601220D
:1074A0000560104630BC704700220A60F2E700BF5A
:1074B000580D00205C0F00206C0F0020024A13685A
:1074C000002BFCD1704700BF640F00204FF46050C8
:1074D00038B5C4F2010040F2255103F029FA002822
:1074E0002BD14FF46050C4F2010040F2277103F039
:1074F0001FFA00B938BD4FF46050C4F2010040F2E9
:10750000277103F03BFA234B1A68002A38D0224A2D
:10751000224C1168481C802808BF002054F8211014
:1075200010601A684FF46050013AC4F2010089B249
:107530001A60BDE8384003F0E5B94FF46050C4F27A
:10754000010040F2255103F019FA4FF46050C4F2E3
:10755000010003F0DBF9124B1A687F2AC1D81149E8
:10756000114D0A68C0B2541C7F2C45F8220098BF08
:107570000C6001D900220A601A6801321A60B0E773
:107580004FF46050C4F2010040F22771BDE838406A
:1075900003F09CB9640F00206C1100205C0D0020EA
:1075A000580D0020600F00206C0F002010B541F234
:1075B0007014C2F2000402460B4620464FF480715C
:1075C00004F008FB2046BDE81040FFF749BF00BFAC
:1075D0000FB400B583B004AB53F8040B1946019304
:1075E000FFF7E4FF03B05DF804EB04B0704700BFA1
:1075F000FFF796BE10B584B001A803F087F801200C
:10760000014602F0ABFF0023ADF80A30ADF80630BA
:10761000052301A9ADF808304FF0804040F21F3338
:10762000ADF8043002F0B6FF01210A464FF0804069
:1076300003F09EF801240F2368461C228DF80020D9
:107640008DF803408DF801308DF8023002F052FBC6
:107650004FF08040214603F06DF804B010BD00BF2C
:1076600038B54FF08040012103F0ACF86A4B1C683C
:10767000002C34D0694B43F698211A6801328A42B3
:107680001A6000D038BD664A0120664910600C6857
:10769000654A24180C6014680021241814601468CA
:1076A00019603C2CEED1614B11601A6812181A60F7
:1076B0005F4A10601A683C2AE4D15E4A1960136878
:1076C0001B1813601368182BDCD15B4B11601A6810
:1076D00012181A601A68072AD4D1196038BDFFF74A
:1076E000DFF950490B68012B07D9544B40F6A660CF
:1076F0001A68013282421A6043D0514B1A68013233
:10770000EA2A1A6054D04F4B1A680132962A1A603E
:1077100048D04D4B1A680132962A1A603CD04B4B28
:107720001A6801320F2A1A6030D03C4B43F6982079
:107730001A68013282421A60A4D1394A01201060CD
:107740000C68394A24180C6011680024091811606B
:1077500011681C602D2931D01268334B3C2A38D077
:107760001B681E2B53D03A4B1A68002A8AD01A681D
:10777000013A1A601B68002B84D1364B01221A6033
:1077800080E7354A012010601C60B6E7334A0120CB
:10779000106000221A60C8E7314A01201060002200
:1077A0001A60BCE72F4A0120106000221A60B0E77F
:1077B0002D4A0120106000221A60A4E72B4B1B49C0
:1077C0001C680D68AC421FBF09681960284B18601F
:1077D000C2E7164A002119601368012001331360C3
:1077E000134B186013683C2BBDD1124B11601A6803
:1077F00012181A601A68182AB5D10F4A196013684E
:107800001B1813601368072B08BF1160ABE7194BF7
:1078100001221A60A7E700BFC012002070120020EA
:107820007C120020C81200208C120020D0120020F0
:1078300090120020B0120020801200209812002028
:10784000B41200209412002088120020AC120020F4
:10785000A401002074120020B8120020A8390020D2
:10786000AC390020A8120020CC120020AC0100206E
:107870009C120020BC1200204EF68850C0F600007A
:10788000704700BF40F2B013C2F20003186870479F
:1078900041F2B02141F2D02241F28C23C2F2000128
:1078A000C2F20002C2F20003096843F6B010126887
:1078B0001B68C2F20000816042600360704700BF35
:1078C0002DE9F04F9FB003F0BDF803F049F9012016
:1078D000014602F035FE4FF400700121C0F2300085
:1078E00002F076FC4FF4E130FFF782FEFFF75CF820
:1078F00001F074FB01F09AFBFFF77CFE0120F9F721
:10790000C3F8F8F76DFDF8F789FD01F04FFDFBF7BF
:10791000ABFEF8F79BFD002841F01B81BF48FFF745
:107920009FFDBF48FFF79CFDBE48FFF799FDBC488F
:10793000FFF796FDBC48FFF793FDDFF81CB3BB488B
:10794000FFF78EFDB648FFF78BFDDBF80030002B0C
:1079500001F0A680B648FFF783FDB148FFF780FD30
:10796000B44DFBF799FD2B68002B01F09080B248D5
:10797000FFF776FDAA48FFF773FD2B68002B41F057
:10798000C580AE4CAE482168FFF722FE226822F483
:107990007F0323F47F43EBB940F2FF43C0F20103BE
:1079A0009A4201F2F48040F2FF632268C0F20103C0
:1079B0009A4201F2E280A348FFF752FD9848FFF790
:1079C0004FFD206801F0DAFE206801F057FE2068C4
:1079D000FFF730FBFFF7B4FBF8F778FD01F0BCF9D7
:1079E00041F2C0200123C2F20000036001F010FF49
:1079F00041F2C021C2F2000100260E60FAF7DCFC61
:107A0000FAF704FE41F28422C2F200021060FAF793
:107A10004FFE41F2A423C2F200031860FAF780FE81
:107A200041F2A029C2F20009C9F80000FAF724FEC9
:107A300041F2C42C2B68C2F2000CCCF8000083B3D6
:107A40004FF480752368C0F20205AB427B4F28D00B
:107A50007D482946FFF7BCFD764B3D601B68002B37
:107A600041F0C8807948FFF7FBFC6D48FFF7F8FC50
:107A700001F052FC002801F0B580FBF7DDFB002887
:107A800001F0A88001F0FAFE002801F09B8001F0CF
:107A9000FDF8002801F069804FF48073C0F2020302
:107AA000236041F29C2E0120C2F2000E41F2C82157
:107AB000C2F20001CEF800000C6802460146033411
:107AC000FAF75CFC41F2C822C2F2000213680BA86C
:107AD0009C421ED9FEF784FF0028F3D000210A46FD
:107AE0000120FAF74BFC0120F8F7B8FF0BA8FEF7CE
:107AF00077FF002001460246FAF740FC5448FFF7A2
:107B0000AFFC4748FFF7ACFC01F00EFB08B101F0F9
:107B100003FC00200146024604460890FAF72EFCBA
:107B2000FCF7E4F9FCF716F9089E4FF0010900F1A3
:107B30003C0CDFF82881474F0694824604253446E2
:107B4000CDF81C90CDF824C0059615A8FFF7FAFAD9
:107B50008146002840F03081D8F8003043B141F22E
:107B6000C42EC2F2000EDEF80030002B40F03C863E
:107B7000069E002E40F09C83DAF80030002B40F087
:107B8000E0853448F8F770FC002840F0A58341F206
:107B90009C20C2F2000003685BB1DBF80030002BD0
:107BA00040F0D98541F29C2C0023C2F2000CCCF8A5
:107BB0000030D8F8003073B141F2C42EC2F2000E8A
:107BC000DEF800303BB141F2B820C2F20000036899
:107BD000002B40F09A8641F27421C2F200010B683A
:107BE0008BB1DAF80430002B40F03D8641F274226C
:107BF0000023C2F2000240F2A4161360C2F2000693
:107C000040F6D863336041F29029C2F20009D9F8F6
:107C10000030002B40F0A78322E000BF90ED000869
:107C200074DF0008B0ED0008D0ED000888ED000812
:107C3000DCED0008A8040020FCED0008B0010020E5
:107C400010EE0008C8EE000804EF000828EF000856
:107C5000E8EF0008B03900205813002084380020D5
:107C600041F2BC2CC2F2000CDCF80030002B00F01A
:107C7000758240F25C49C2F20009B04AD9F800307E
:107C800000211160002B00F0698241F2D02CC2F279
:107C9000000CDCF80020B2FBF3F103FB1123002BF6
:107CA00040F05C8240F2944EC2F2000EDEF80030EA
:107CB000002B40F0BB85DBF80030002B00F028855E
:107CC00001F026FD9E4B9F4A064610F0010F4FEA39
:107CD00056019D4818BF1A46FFF77AFCFF2E0AD0BE
:107CE0003046FBF79DF841F2C82CC2F2000CDCF8DC
:107CF000003006330893002D40F0448241F2CC203E
:107D0000C2F200000368002B40F0758241F27C2231
:107D1000C2F200021368002B40F07F8241F2A825D6
:107D2000C2F200052B68002B40F0898201F0B6F901
:107D3000FF28054600F08E82002101200A46FAF74E
:107D40001DFB132D00F2B486DFE815F0BC01E8013D
:107D5000D601F5018701B30199016C0133011401CA
:107D6000EA00DD00D000C300A900B60094007F0047
:107D7000B20614007548FFF773FB7548FFF770FBF8
:107D80000126322405960025069EDDF81C9016EA91
:107D9000090F52D1002C3FF4D8AE013C7FF4D5AE90
:107DA000204621462246FAF7E9FA15A8FFF7CAF954
:107DB000814600283FF4D0AE002101200A46A9F1F7
:107DC0004109FAF7DBFAB9F1330F00F21B83DFE860
:107DD00019F06904560451043B0419038504050491
:107DE00019030E0319031903E3031903A30319036A
:107DF0008A03190319037F03250319031903D80301
:107E0000CD031903190319031903190319031903DE
:107E100019031903C203B3037403190319031903E4
:107E20001903190319031903190319031903190372
:107E300069031903190319031C03F8F707FB00284A
:107E400040F01F8501260796A4E74248FFF708FB8C
:107E50003F48FFF705FB41F2C426C2F20006336833
:107E6000002B40F0DC850025FAF72EFF3224059523
:107E7000022589E73848FFF7F3FA3548FFF7F0FAAB
:107E800041F2C426C2F200063368002B40F0B885E8
:107E90000025FAF70FFF32240595022574E72F48D5
:107EA000FFF7DEFA2A48FFF7DBFA0025FAF798FE1B
:107EB00032240595022567E72948FFF7D1FA2448BF
:107EC000FFF7CEFA0026FAF77BFE3224059602254C
:107ED0005AE72448FFF7C4FA1D48FFF7C1FA002605
:107EE000FAF74EFE3224059602254DE71E48FFF7AD
:107EF000B7FA1748FFF7B4FA0025FAF751FE322413
:107F00000595022540E71948FFF7AAFA1048FFF740
:107F1000A7FA0026FAF714FE32240596022533E765
:107F20001348FFF79DFA0A48FFF79AFA0025FAF777
:107F300017FE32240595022526E700BFBC1200205B
:107F40006CE70008FCDE000848F4000898F600081A
:107F500074DF00087CF6000860F6000820F60008D0
:107F600040F60008FCF50008D8F50008B8F5000850
:107F700098F50008B948FFF773FAB948FFF770FAA7
:107F800041F2D023C2F200031A68B64B3A2A00F23B
:107F9000EB841A6801321A6041F28C240023C2F289
:107FA00000042360DBF80060FEB932240596042546
:107FB000EAE6AD48FFF754FAA948FFF751FA41F253
:107FC000D020C2F200000268A64B002A00F0D8843C
:107FD0001A68013A1A6041F28C21DBF80060002334
:107FE000C2F200010B60002EDFD041F2B02941F255
:107FF000D02C41F28C2EC2F2000CC2F2000EC2F262
:108000000009D9F80010DCF80020DEF80030002567
:108010009648B9607A603B60322401F023FA0595F6
:108020000425B1E69248FFF71BFA8D48FFF718FACE
:1080300041F2B02CC2F2000CDCF800208D4B162A65
:1080400000F296841A6801321A6041F28C2E0023E5
:10805000C2F2000ECEF80030A4E78748FFF700FA1E
:108060007F48FFF7FDF9FAF73DFB41F2A426002512
:10807000C2F20006059532243060042584E67F486C
:10808000FFF7EEF97648FFF7EBF941F2B026C2F2BE
:1080900000063268774B002A00F06E841A68013AB5
:1080A0001A6041F28C290023C2F20009C9F800309D
:1080B00078E77348FFF7D4F96948FFF7D1F9FAF781
:1080C00005FBD2E76F48FFF7CBF96548FFF7C8F922
:1080D00040F25C1CC2F2000CDCF800503224D5F1F6
:1080E000010538BF00250026CCF800500596B542A2
:1080F0000CBF14250C2547E66348FFF7B1F9584833
:10810000FFF7AEF9FAF7A8FA41F28425C2F20005AA
:108110000026286032240596042535E65B48FFF7E3
:108120009FF94F48FFF79CF900240594FBF784F86A
:108130003224059D28E65648FFF792F94848FFF794
:108140008FF9FAF777FA41F284290025C2F2000983
:1081500005953224C9F80000042515E6059E002E79
:108160007FF4A0AD089E002E3FF4C5AD41F2C829B2
:10817000C2F20009D9F80030B342FFF4BCAD059E4D
:1081800004250896434841F28429FFF769F9C2F2B1
:1081900000093348FFF764F9D9F80030112B40F09B
:1081A000BF8240F2944CC2F2000CDCF80030002B8D
:1081B00040F0BB83DBF80030002B00F0AD8301F012
:1081C000A7FA354B354A064610F0010F4FEA560123
:1081D000334818BF1A46FFF7FBF9A6F11401002037
:1081E0002A46FAF7FBF841F2CC20C2F200000368FD
:1081F000002B3FF48BAD40F25C112A4BC2F2000120
:10820000002208681A60FAF763FB41F27C22C2F28E
:1082100000021368002B3FF481AD234B00221A604B
:1082200041F28C23C2F2000341F2A8251868C2F281
:108230000005FAF78DFA2B68002B3FF477AD1B4B46
:1082400000221A60F8F778F900F028FFFF280546A9
:108250007FF472AD00260596354695E580F5000859
:1082600074DF0008D012002068F50008B039002043
:1082700050F50008B0120020F8F4000838F50008A6
:1082800018F5000898F40008B8F40008A8F40008ED
:10829000D8F4000888F400086CE70008FCDE000849
:1082A00048F40008CC1200207C120020A812002004
:1082B00041F27829C2F20009D9F8003023B9DAF87E
:1082C0000430002B40F003830126CA480696F8F7D5
:1082D000CBF800283FF45BAC012001460022FAF7FE
:1082E0004DF8DBF80030002B40F0C78241F2B02996
:1082F000C2F20009D9F80030BC68BE4A9C4200F0C6
:10830000DA82D2F804E00425D7F8189040F2000091
:10831000C2F2000050F829103E68F86841F2802C43
:10832000C2F2000C7A693B698DE811400396CCF8E3
:10833000009041F2B02941F2D02CC2F2000CC2F2FE
:108340000009C9F80040CCF800E041F28C2EC2F2DE
:10835000000EA94802F26C720133CEF80060FFF7FC
:1083600037F9322413E4A54B002241F2802C41F26C
:10837000B02E1A60C2F2000CC2F2000E41F2D02000
:10838000DCF80010C2F20000DEF8003040F25C15AC
:108390000268C2F20005C3EB0313286802EB8302F4
:1083A000974D00F09FFC002800F01B822B68DFF83F
:1083B00074C2D3F1010E38BF4FF0000E41F2B02667
:1083C00041F2D0298F49BEF1000FC2F20006C2F27D
:1083D000000932688C48D9F8003008BF6146C5F8FA
:1083E00000E00CBF14250C25FFF7F2F838E48748AD
:1083F000FFF736F88648FFF733F800F095FE0028BF
:1084000040F081813224FFF7A7BB159B40F2A412F4
:10841000C3F56E630233C2F200021360DBF8003072
:10842000002B40F00B8341F2B024C2F20004236819
:10843000DDF85CE09E4500F00583DDF858C00425BA
:108440001B9C40F20009C2F2000959F82410159E45
:10845000189B41F28029C2F20009CDF804E0009394
:10846000CDF808C00396C9F8004041F2B029C2F225
:108470000009C9F800E01A9A199B41F2D02E41F286
:108480008C29C2F2000EC2F20009CEF800C0614889
:1084900002F26C720133C9F800603224FFF798F8D9
:1084A000FFF75ABB15A8FAF763FC5B4815A9FFF75D
:1084B0008FF804253224FFF74FBB1598FAF776F8AA
:1084C00001465648FFF784F804253224FFF744BBE1
:1084D000FAF7B2FE5248FEF7C3FF4D48FEF7C0FF61
:1084E0003224FFF739BB40F25C1EC2F2000E159B2E
:1084F000DEF80020934285D04A4A4249002B08BF4B
:1085000011463F4A484814BF0C25142513603224F5
:10851000FFF75EF8FFF720BB41F2742C0123C2F293
:10852000000C4248CCF80030FEF79AFF3848FEF7BE
:1085300097FF3224FFF710BB15A8FAF791FB3C48D0
:108540009DF854109DF855209DF85630FFF740F8DF
:108550003224FFF701BB1598FAF7C8FB3548159987
:10856000FFF736F802253224FFF7F6BA3248FEF755
:1085700077FF2748FEF774FF3224FAF7C3FBFFF7B3
:10858000EBBA2E48FEF76CFF01242148FEF768FF86
:1085900005943224FFF7E0BA159B002B00F05D82B2
:1085A00041F2C42926480123C2F20009C9F800306B
:1085B000FEF756FF1648FEF753FF41F2C42EC2F2F3
:1085C000000E40F2A811FF23C2F20001DEF8000005
:1085D0000B603224FAF756F8FFF7BEBA1598F9F790
:1085E000C1FF18481599FEF7F3FF04253224FFF761
:1085F000B3BA00BFB0390020A8F3000890120020E1
:108600005C010020D4F6000800F40008FCF2000829
:1086100074DF0008A4F2000834F30008ECF000084E
:1086200014F30008E8F60008B0F00008DCF20008D7
:1086300084F00008D4F1000888F2000860F1000816
:1086400000F2000860F2000841F28421C2F2000149
:1086500015980B6898423FF4D5AEF9F7DDFFD04A84
:1086600003460146CF4813600425FEF7B1FF3224CC
:10867000FFF772BA15A8FAF7CFFACB4860E741F2D4
:10868000C425C2F200052B68002B40F0F381159839
:10869000FAF704FBC5481599FEF79AFF0225322424
:1086A000FFF75ABA41F2A422C2F2000215981368E9
:1086B00098423FF4A7AEFAF701F8BD4A034641F2EB
:1086C000CC2419461360C2F200040023B948236089
:1086D0000425FEF77DFF3224FFF73EBA41F2A026C3
:1086E000C2F200061598336898423FF48BAEFAF751
:1086F0001DF8B14A03460146B04813603224FEF724
:1087000067FFFFF729BA00F007FE3224FFF724BA0B
:10871000AB48FEF7A5FEAB48FEF7A2FEFFF7EBBAAB
:1087200041F2B02C41F2D02EC2F2000CC2F2000E87
:10873000DCF800002A46DEF80010F9F74FFEFFF7DC
:10874000DDBAA148FEF78CFE01269E48FEF788FEA2
:108750000696FFF716BADFF88892484600F016FF33
:1087600000283FF41FAA41F2B021C2F200010B68B9
:10877000D9F808E09E4500F00781D9F804C0042527
:10878000BE69F86840F20003C2F2000353F82610F5
:108790007A693B698DE80140CDF808C0386841F23C
:1087A0008029C2F200090390C9F8006041F2B026A6
:1087B00041F2D029C2F20006C2F20009C6F800E078
:1087C000C9F800C03E6841F28C29C2F200097F4816
:1087D00002F26C720133C9F80060FEF7F9FEFFF790
:1087E000E1B90425FFF73CBA0AA8FEF705FC00280A
:1087F0003FF4BEA940F2A8100A9AC2F20000016834
:10880000531C8B4203D34B1C9A427FF6B1A970488C
:10881000FEF7DEFE0A9B40F2A811C2F200011846E4
:1088200002250B60FAF73AFAFFF7A2B941F2C0202D
:108830000123C2F20000036000F08AFF654B664A24
:1088400010F0010F064641F2C02918BF1A46C2F2C5
:108850000009002361484FEA5601C9F80030FEF7CD
:10886000B7FEFFF73BBA002001460122F9F786FD6B
:10887000322401F065F8FFF7B9B9594800F0F2FD6C
:1088800034E55848FEF7ECFD4E48FEF7E9FD4FF0A1
:10889000000941F2782CC2F2000CCAF804908AF860
:1088A0003C9051495148CCF80090CDF81C90FBF712
:1088B00095FAFFF76FBA41F2D02CC2F2000CDCF847
:1088C0000030D2F804E09E457FF41DAD1CE5484B16
:1088D0004FF001094748C3F80090FEF7C1FD394841
:1088E000FEF7BEFD4449099A0DA802F0B7FC0DA899
:1088F000FAF73EFA41F2742CC2F2000C0425CCF8CF
:108900000090CDF81890FFF73CB9FEF773FB3B4B96
:1089100000221A60FFF75FB92948FEF7A1FD294838
:10892000FEF79EFD6FF0130159E441F2C02E0123C2
:10893000C2F2000ECEF8003000F00AFF254B264AA6
:1089400010F0010F064641F2C0294FEA560118BF48
:108950001A4622480023C2F20009C9F80030FEF787
:1089600037FEA6F114013AE400221A60FFF714BBA7
:1089700000221A60FFF769BB17221A60FFF791BB4C
:108980003B221A60FFF727BB41F2D022C2F200025D
:108990001368D9F804C09C457FF4F1AEF0E600BF3F
:1089A00084120020C8F0000858F000087CF100088C
:1089B000A412002010F10008A012002034F10008D9
:1089C0006CF4000874DF00087CF30008D4F300089E
:1089D00050F300086CE70008FCDE000820F40008F3
:1089E000B039002004F000084CF0000840F0000806
:1089F000781200208CF30008A0F30008B8120020C1
:108A0000814A002340F2A81918461360C2F20009F7
:108A1000FF23C9F80030F9F735FEFFF739BA7A4A73
:108A2000002340F2A81918461360C2F20009FF2380
:108A3000C9F80030F9F726FEFFF715BA15A800F0BF
:108A400011FDF0E441F2D026C2F200063368DDF8F1
:108A500058C09C457FF4F3ACF2E441F2C42CC2F25E
:108A6000000C6A48CCF80030FEF7FAFC6848FEF7C4
:108A7000F7FCA2E5644A002340F2A81618461360EA
:108A8000C2F20006FF233360F9F7FCFDFFE5614801
:108A9000FEF7E6FC5E48FEF7E3FC5F4CFEF79ABF8C
:108AA0005E48FEF7DDFC5A48FEF7DAFCFEF758BFD9
:108AB000132D54D80FF2040959F825F0D18000087D
:108AC00029810008058100084381000867800008AB
:108AD000BF8000088B80000831800008BF7F00083D
:108AE000817F00082D7F0008137F0008F97E0008B1
:108AF000DF7E0008AB7E0008C57E0008817E00088E
:108B0000577E00081B8B0008817D00080020424929
:108B10000422FAF7D1FDFEF734BF41F2C429C2F2B4
:108B20000009D9F8003040F2A81CD3F1010338BF86
:108B300000231846C9F80030C2F2000CFF230025BC
:108B4000CCF800303224F9F79DFD05950225FFF79A
:108B50001BB9F7F731FCFBF773F9FEF7DFBE002412
:108B6000059400253224FFF70FB92D48FEF778FC55
:108B70002748FEF775FCFEF78FBF2A48FEF770FC0A
:108B80002348FEF76DFC00F05BF8FEF714BF2648A3
:108B9000FEF766FC1E48FEF763FC00F093FB2348DB
:108BA000FEF75EFC1A48FEF75BFC2068FAF7AAF9AC
:108BB0001F48FEF755FC1648FEF752FC00F02CFE4D
:108BC000FEF7F1BE1B48FEF74BFC1148FEF748FCD0
:108BD000FEF75DBF1848FEF743FC0D48FEF740FC6A
:108BE000FEF750BF1548FEF73BFC0948FEF738FC7E
:108BF000FEF743BF304639460422FAF777FD0028D6
:108C00007EF436AFFEF72EBFC412002030F200080B
:108C100074DF0008F0EE0008B0010020ECED000861
:108C2000BCEF0008A4EE000834EE000854EE000883
:108C300080EE000890EF000870EF00084CEF00088D
:108C400030B5104B87B01B6813B9002007B030BD9A
:108C5000BF2069461822FAF72FFD0028F5D00A48F0
:108C60006A4600231478517895781C50C1EB0111A5
:108C70001C18083305EB81010332402B6160F1D1F0
:108C80000120E3E7A8040020D4390020F0B548F61D
:108C9000890787B0114C6A460023C8F6880719195E
:108CA00048681D59A7FB00614909C1EB0116A0EBFB
:108CB000860008331570517090700332402BEED14E
:108CC000074B186838B1BF2018226946FAF70EFD25
:108CD000003018BF012007B0F0BD00BFD43900201C
:108CE000A8040020F0B400231A4D02E00833402B02
:108CF00021D05C595E1914F0800FF7D07668964247
:108D0000F4D1C4F3C20604F0070704F0400418B11C
:108D1000D4F1010438BF0024002CE7D0BE420DD8A6
:108D2000B14234BF00260126B94288BF0026002E7A
:108D3000DCD0012000E00020F0BC7047B9428CBFBD
:108D400000270127B14234BF3E4647F00106002EFE
:108D5000CCD0EEE7D4390020704700BF70B5642056
:108D6000F7F75AFE4FF4406020210022C4F20100C0
:108D700001F028FA4FF40C70F7F74EFE4FF4406004
:108D8000C4F201002021012201F01CFA274D142019
:108D9000F7F742FE00264FF496732B60344603E04B
:108DA00004B92C682B68ABB14FF440602021C4F2A9
:108DB000010001F001FAD6F1010338BF0023002CB5
:108DC00008BF00230028EBD0002BEBD02E682B68C7
:108DD000002BE9D13220002E18BF002C0CBF00253B
:108DE000012515D0F7F718FE4FF440602021C4F29A
:108DF000010001F0E1F905467820F7F70DFE6B1E42
:108E00005842C6EB040458411E2C98BF002070BD88
:108E1000F7F702FE4FF440602021C4F2010001F098
:108E2000CBF97820F7F7F8FD284670BD8038002090
:108E300010B54FF44064C4F2010420210022204602
:108E400001F0C0F90520F7F7E7FD012220212046B7
:108E500001F0B8F90A20F7F7DFFD2021204601F0E4
:108E6000ABF904463220F7F7D7FD621E504250415D
:108E700010BD00BF70B5082401250026FFF7D8FFFC
:108E80006B0000B12E43013CDDB2F7D1304670BD1E
:108E900038B54D1E0446EDB239B101354519FFF71D
:108EA000E9FF04F8010BAC42F9D138BD70B50646B4
:108EB0000825012418E04FF440600022C4F20100AC
:108EC00001F080F90520F7F7A7FD4FF4406020215D
:108ED0000122C4F2010001F075F950206400F7F797
:108EE0009BFD013DE4B21BD04FF44060202114EA09
:108EF0000602C4F20100DED101F064F95020F7F758
:108F00008BFD4FF4406020210122C4F2010001F0EA
:108F100059F905206400F7F77FFD013DE4B2E3D184
:108F200070BD00BF38B54D1E0446EDB239B10135F4
:108F3000451914F8010BFFF7B9FFAC42F9D138BD60
:108F400010B50446FFF70AFF80B9234603F8010B6A
:108F50000133607003F8010B03F8010B03F8010BF8
:108F600003F8010B03F8010B187010BD3320FFF755
:108F70009DFF20460821FFF78BFFFFF7EFFE012042
:108F800010BD00BF30B5144B83B01A680AB103B0EE
:108F900030BD012401A81C6001F006F92020214603
:108FA00001F0CEFA14234FF44060202501A98DF87A
:108FB0000730C4F201000323ADF804508DF80630E9
:108FC00001F08EF84FF44060C4F2010029462246B9
:108FD00001F0F8F8DBE700BFD412002000B583B041
:108FE00001A801F0E1F80820012101F0A9FA01230C
:108FF000ADF804304FF44060022301A98DF806302B
:10900000C4F2010010238DF8073001F069F84FF227
:10901000B060C0F60000FEF723FA4DF67470C0F69B
:109020000000FEF71DFA03B000BD00BF10B50A4CEA
:109030002368012B0FD001214FF440600A46C4F28F
:10904000010001F0BFF80548FEF70AFA0448FEF7F0
:1090500007FA0123236010BDB4010020C4F6000804
:1090600074DF000810B50A4C23687BB14FF44060F0
:1090700001210022C4F2010001F0A4F80548FEF726
:10908000EFF90548FEF7ECF90023236010BD00BF9F
:10909000B4010020D8F6000874DF0008F0B583B0F2
:1090A0006846FDF79DFC68B31C4B1D4A18681168A3
:1090B00001301860002928D09DF8050000F001005B
:1090C00018490023BDF80170BDF803C09DF80040A9
:1090D00010600E46184602E00130782B12D0CA5CB0
:1090E0000633A242F8D100EB400206EB4202B2F88E
:1090F0000150BD42F0D1B2F80320624503D00130E7
:10910000782BECD1FF2003B0F0BD9DF8053013F0B3
:109110000100D5D001231360F4E700BFD81200206E
:10912000DC120020E01200202DE9F04FDFF89081E2
:1091300000274D4D83B001263C46C2462846F9F72C
:1091400017FE2846FEF78CF94848FEF789F968466D
:10915000FDF746FC04EB440908EB49090AEB070557
:109160004846FDF73DFC0028FAD06A7912F001026A
:10917000F6D1C4B399F80010134602E00133A342BC
:109180002FD018F8020006328842F7D103EB430CC7
:109190000AEB4C0CB9F80100BCF801E08645EDD1B2
:1091A000B9F803E0BCF803C0F445E7D1FF2B18D0B1
:1091B0000022134602E00133A342D1D018F802C0C6
:1091C00006328C45F7D103EB430C0AEB4C0CBCF890
:1091D00001B08345EFD1BCF803C0F445EBD1002BBF
:1091E000BED1142E37D0731E122B3BD8DFE803F00C
:1091F0002F2D2B29272523211F1D1B19171513116F
:109200000F0A31001A4D01340136063796E7194D21
:10921000F9E7194DF7E7194DF5E7194DF3E7194D42
:10922000F1E7194DEFE7194DEDE7194DEBE7194D52
:10923000E9E7194DE7E7194DE5E7194DE3E7194D62
:10924000E1E7194DDFE7194DDDE7194DDBE7194D72
:10925000D9E7194DD7E71948F9F78AFD012003B07E
:10926000BDE8F08F004DCEE700F7000874DF00087E
:10927000C8F80008A8F8000888F800086CF800088A
:1092800050F8000830F8000810F80008F4F700085B
:10929000D8F70008C4F70008B0F700089CF70008EA
:1092A00088F700086CF7000850F7000834F700084A
:1092B00018F7000810F70008ECF60008E4F80008BA
:1092C000E0120020F0B5124B83B01868E8B1002519
:1092D000104F04262C46052230466946FAF7ECF971
:1092E0009DF800C0BDF80110BDF8032004EB440355
:1092F000013407F805C007EB430305360635142C87
:10930000A3F80110A3F80320E5D103B0F0BD00BF1E
:10931000A8040020E0120020F0B5124B83B01868BA
:10932000E8B10025104F04262C4604EB440307EB5C
:10933000430317F805C0B3F801E0B3F80330052282
:109340003046694601348DF800C0ADF801E0ADF853
:109350000330B6180635FAF7C9F9142CE5D103B075
:10936000F0BD00BFA8040020E012002010B50446A4
:1093700082B00B460092D02000222146FDF7D8F99A
:10938000D0F1010038BF002002B010BD10B5044676
:1093900082B00B460092D02000222146FDF746FA0B
:1093A000D0F1010038BF002002B010BD30B583B04D
:1093B000FDF786F93F200DF107010122FFF7D6FFE7
:1093C000054620B301240720244B0DEB0001224663
:1093D0001C60FFF7CBFF10B39DF80730002B29D19D
:1093E00000200DF107010122FFF7C0FF0446B0B1D4
:1093F0009DF807301A0619D503F07F0300200DF100
:10940000070101228DF80730FFF7C0FF0EE00E20A4
:109410000DF107010122FFF7A9FF044618B9002446
:10942000204603B030BD9DF807306BB90C4B0122CC
:109430001A60F5E7072000230DEB000122468DF8A6
:109440000730FFF7A3FFCBE70E200DF10701012244
:109450008DF80750FFF79AFFE8E700BF6013002080
:10946000581300202DE9F04F474B89B01B681BB9FA
:10947000184609B0BDE8F08F836802690193C3689C
:1094800041690293D0F800E0013246F26763C6F208
:10949000666303926439049183FB0EBA0199DDF887
:1094A0000CB0476883FB0118029A83FB0B1B83FBFC
:1094B00007C983FB022C049ACDF800B083FB02B2EB
:1094C00001990592039B029ADDF810B04FEAEE76FF
:1094D000C6EBAA06DDF814A0FD17CC178069D117DA
:1094E000DA174FEAEB73C5EBA905C1EBAC01C3EB8F
:1094F000AA03DDF800C0059005EB850A03EB8300A5
:10950000C4EBA8040090C2EBAC020198A7EB4A0799
:10951000DDF80CA006EB860B04EB840902EB820C51
:10952000AEEB4B0EA0EB4909DDF810B00298AAEBA8
:109530004C0CDDF800A009EB041901EB8108059C37
:10954000A0EB4808ABEB4A0008EB01180CEB021C3F
:1095500000EB03130EEB061E07EB0517013400208A
:1095600006A907228DF818E08DF819708DF81A9069
:109570008DF81B408DF81C808DF81DC08DF81E30B5
:10958000FFF704FF75E700BF581300202DE9F04FE7
:10959000394B8BB01B6804461BB900200BB0BDE8EB
:1095A000F08F002008A90722FFF7E0FE0028F4D082
:1095B0009DF825A09DF820709DF826804FEA1A1B83
:1095C0009DF824304FEA171C0BEB8B0B4FEA181950
:1095D000CDF81CB00CEB8C0C05939DF822209DF867
:1095E000233009EB890908F00F08CDF800C0DDF839
:1095F0001CC00AF00F0ACDF80890CDF804809DF841
:10960000215011090693DDF81490DDF80480059BC4
:10961000CDF80CA00AEB4C0ADDF808C002F00F02EE
:1096200001EB81012E091B0909F00F0B02EB41012F
:1096300008EB4C09069ADDF8008005F00F0504934D
:1096400007F00F0706EB860603EB830305EB4606E0
:1096500002F1FF3C07EB48070BEB43030AF1FF3530
:1096600009F1640227606660A160C4F818C0E36075
:109670002561626192E700BF5813002000B50E4BD0
:1096800083B01B6853B1FF23C0F20203984207D88E
:1096900000220120094B1A6003B000BD1846FBE709
:1096A0000122DF200DF10701FAF706F89DF80720E7
:1096B0000A2A88BF0022EDE7A80400205C130020DE
:1096C00000B5094B094A1B68106883B08DF8073054
:1096D00040B1DF2001220DF10701FAF707F8003051
:1096E00018BF012003B000BD5C130020A8040020B7
:1096F00041F25C33C2F200031868704710B541F2C2
:109700005C34C2F200042060FFF7DAFF206810BD6D
:1097100000B50D4B83B01B68FF200BB903B000BD33
:10972000112001A90222FFF721FE0028F6D09DF8A2
:109730000500064B9DF80420C0F340001B6840EA7A
:109740004200C01AEAE700BF581300205C13002053
:1097500000B585B001A802A903AAF9F79FFE10B9C8
:10976000FF2005B000BD029B002BF9D1024B186809
:10977000039B181AF5E700BF6413002000B50E4BD9
:1097800083B01B6853B1FF23C0F20203984207D88D
:1097900000220120094B1A6003B000BD1846FBE708
:1097A0000122DF200DF10701F9F786FF9DF8072060
:1097B0000A2A88BF0022EDE7A804002064130020D5
:1097C00000B5094B094A1B68106883B08DF8073053
:1097D00040B1DF2001220DF10701F9F787FF0030CA
:1097E00018BF012003B000BD64130020A8040020AE
:1097F00041F26433C2F200031868704710B541F2B9
:109800006434C2F200042060FFF7DAFF206810BD64
:109810000920F9F7B5BE00BF00B5144B83B01B6833
:109820002BB1AA2012491022F9F746FF50B9102295
:109830000F48104901F076FD0F4B01221A600020FD
:1098400003B000BDBA2001A90222F9F735FF0028B4
:10985000EDD09DF804109DF80520074B01202D291F
:109860001A60EDD152421A600120E9E7A8040020F5
:10987000BC010020F4F80008B801002000B5134B2B
:1098800083B01B68002B1ADB2B228DF804208DF887
:1098900005300F4B1B6813B9002003B000BDAA2090
:1098A0000C491022F9F722FF0028F5D0BA20022235
:1098B00001A9F9F71BFF003018BF0120EDE75B425B
:1098C0002D228DF804208DF80530E2E7B801002044
:1098D000A8040020BC01002040F2B813C2F200032B
:1098E0001868704710B5014604460A48FDF770FE37
:1098F00004F10C03182B0AD8074B1A68A24204D0B3
:109900001C60FFF7BBFF012010BD012010BD00202F
:1099100010BD00BF04F90008B801002040F2BC10DF
:10992000C2F20000704700BF014640F2BC1008B50B
:10993000C2F2000001F0CDFCBDE80840FFF79EBF79
:1099400040F2BC10C2F20000FAF760BA70B5284AC3
:1099500048F280131268C7F65543CB184FF4616183
:1099600001FB023382B002AE46F8043D05463046A4
:1099700001F06CF903690446DA1E052A0CD9022BA2
:109980002BD0092B10D18369C268D21A182A03DDA3
:1099900053B98368022B07DC019B304603F56163F2
:1099A000019301F053F90446636904F10C006B6103
:1099B00023692B61E368EB6007C8013102F26C7226
:1099C000F6F796FCA861236A2B62A368AB60636814
:1099D0006B6023682B6002B070BD8369C268D21AC5
:1099E000182AE1DD002BD7D18368012BD4DCDBE71B
:1099F000B801002008B5202000F05AFB28B1202033
:109A000000F064FB014B00221A6008BD68130020BF
:109A10002DE9F843DFF800E10646DEF80030002BC0
:109A2000FBD1002E6FD03A48770007EB060C39497E
:109A30008444182510F8029CA5F11803A5F110081C
:109A4000802212EA090F0CBF22243A24CC5401339D
:109A500052084345F5D110F8039CA5F1080880226F
:109A600012EA090F0CBF22243A24CC5401335208C5
:109A70004345F5D110F8018C802212EA080F0CBF83
:109A800022243A24CC54013352089D42F5D10330AC
:109A900018356045CED10022CB18104698540132BB
:109AA000302AFBD14FF4305001240021C4F20100D0
:109AB000CEF8004000F03EFE1C200021C4F202005F
:109AC00000F0DEFABB19DB0030331C204FF6F871D2
:109AD0001940C4F2020000F0E9FA1C2002212246DB
:109AE000C4F2020000F0D8FA1C202146C4F20200A1
:109AF00000F0C6FA4FF43050C4F201002146BDE830
:109B0000F84300F017BE334602493746C3E700BFAB
:109B10006F1300208417002068130020B0F5AE7F7B
:109B200009D80A78044B00EB40001A544A781818F8
:109B300042708B78837070476C130020F0B469B169
:109B40000A4D01EB410700230678EC18EE544678E5
:109B5000033366708678BB42A670F5D10AB9F0BCB3
:109B600070470846F0BCFFF753BF00BF6C130020DE
:109B70002DE9F0415D4D94B0002468462C6000F062
:109B800013FB0420012100F0DBFC18234FF40060DC
:109B90004FF48078C4F2010069468DF80330032346
:109BA0008DF80230ADF8008000F09AFA4FF40060B2
:109BB00022464146C4F2010000F004FB02A800F076
:109BC000A5FD05A800F0ACFD01214FF4006000F0F8
:109BD000B7FC0120014600F0A5FC4FF430505B2398
:109BE000C4F2010002A9ADF80C30ADF80840ADF8A0
:109BF0000E40ADF80A4000F0CDFC4FF43050602329
:109C00000126C4F2010005A9ADF81430ADF81660C4
:109C1000ADF81A40ADF81C4000F01CFD4FF4305078
:109C20000821C4F2010000F0C5FD4FF43050C4F229
:109C30000100314600F0B0FD4FF43050C4F2010095
:109C4000314600F085FD4FF4305032464FF400713C
:109C5000C4F2010000F096FD0C2301A88DF8043039
:109C60008DF805408DF806408DF8076000F042F849
:109C700009A800F0F7F91C202146C4F2020000F008
:109C8000FFF91C20C4F2020000F020F942F6344330
:109C9000C4F20103099342F2E8031C200C938023D1
:109CA0000E934FF44053129310230B93104BC4F2B6
:109CB000020009A91194CDF83C8010940D941394DE
:109CC0000A93274600F0AEF98DF824408DF8254020
:109CD0008DF826402B68002BFCD109A840F25D11BD
:109CE0000122FFF72BFF14B0BDE8F08168130020BC
:109CF00084170020C37830B47BB90378012103F0C6
:109D00001F0201FA02F15A094FF46143CEF2000337
:109D1000203243F8221030BC70474FF46D43CEF22E
:109D20000003DB684478DB43C3F302230F22C3F153
:109D3000040122FA03F304FA01F48578017803EAB6
:109D40000502224301F160431201D2B203F56143DF
:109D500083F800230278012102F01F0301FA03F1C6
:109D60004FF46143CEF20003520943F82210D2E7C8
:109D700042680B6822F4702270B422F480720C796D
:109D8000134343EA0423436086688C68CA684FF231
:109D9000FD73CFF6F1734D7922433340134343EA09
:109DA000450383600B7CC26A013B22F47002DBB284
:109DB00042EA0353C36270BC704700BF00230360D4
:109DC000037143718360C36001230374704700BF54
:109DD000836819B923F001038360704743F00103DE
:109DE00083607047836843F008038360704700BF57
:109DF0008068C0F3C0007047836843F00403836049
:109E0000704700BF8068C0F380007047836819B94D
:109E100023F4A0038360704743F4A003836070477A
:109E2000092970B401EB41041ED91E3C072606FA2D
:109E300004F603FA04F4C568062A25EA060343EA91
:109E40000403C3601DD90C2A02EB820227D9413AD0
:109E50001F2404FA02F401FA02F1C36A23EA04029D
:109E60000A43C26270BC7047072606FA04F603FA7A
:109E700004F40569062A25EA060343EA040303619C
:109E8000E1D8013A02EB82021F2404FA02F401FA3B
:109E900002F1436B23EA04020A434263E2E7233AF6
:109EA0001F2404FA02F401FA02F1036B23EA04020C
:109EB0000A430263D6E700BFC06C80B2704700BFA0
:109EC000036819420CBF002001207047082110B41C
:109ED00004684FF6FE72C4F2020100232240884259
:109EE0000260036043608360C36050D01C23C4F2EF
:109EF0000203984252D03023C4F20203984255D054
:109F00004423C4F20203984258D05823C4F20203F7
:109F100098425BD06C23C4F2020398425ED0802347
:109F2000C4F20203984228D04FF48163C4F20203C2
:109F300098422AD040F21C43C4F20203984255D002
:109F40004FF48663C4F20203984258D040F244436F
:109F5000C4F2020398425BD04FF48B63C4F2020355
:109F6000984201BF4FF48063C4F202035A6842F47E
:109F7000702208BF5A6010BC70470023C4F202036D
:109F80005A6842F070625A60F5E74FF48063C4F299
:109F900002035A6842F00F025A60ECE70023C4F251
:109FA00002035A6842F0F0025A60E4E70023C4F268
:109FB00002035A6842F470625A60DCE70023C4F27C
:109FC00002035A6842F470425A60D4E70023C4F294
:109FD00002035A6842F470225A60CCE70023C4F2AC
:109FE00002035A6842F470025A60C4E74FF4806377
:109FF000C4F202035A6842F0F0025A60BBE74FF421
:10A000008063C4F202035A6842F470625A60B2E795
:10A010004FF48063C4F202035A6842F470425A60FB
:10A02000A9E700BF8B68F0B40D6A0C694A691D434B
:10A030002C438B691443CA6905684F6A23438E6AAF
:10A0400013431F4325F4FF4525F070053E432E437F
:10A050000660CB6843600B6883604B68C360F0BCEC
:10A06000704700BF0023036043608360C3600361E7
:10A0700043618361C361036243628362704700BFCF
:10A0800029B902684FF6FE731340036070470368F6
:10A0900043F001030360704703681AB923EA010122
:10A0A0000160704719430160704700BF416070470D
:10A0B000C1004CBF4FF480630023C4F202031B684D
:10A0C00003420CBF00200120704700BFC3004CBFFB
:10A0D0004FF480630023C4F202035860704700BF4E
:10A0E000CB782DE9F00303F00F06DB0648BF8B7831
:10A0F0000A8848BF1E4312F0FF0F27D007680023CD
:10A1000001254FF00F0803E00133082B1CD00A880B
:10A1100005FA03F42240A242F6D19C0008FA04F9A1
:10A1200006FA04F491F803C027EA0907BCF1280FE6
:10A1300047EA040708BF4261E6D0BCF1480F08BFF8
:10A1400002610133082BE2D107600A88FF2A28D96F
:10A150004768002301254FF00F0803E00133082B67
:10A160001ED00A8803F1080405FA04F42240A24232
:10A17000F4D19C0008FA04F906FA04F491F803C03B
:10A1800027EA0907BCF1280F04BF426191F803C018
:10A190002743BCF1480F08BF02610133082BE0D10F
:10A1A0004760BDE8F00370474FF6FF73038002235A
:10A1B00083700423C3707047836819420CBF00206A
:10A1C000012070470AB9416170470161704700BFC3
:10A1D00030B400230028C4F2010300F44012B4BFDD
:10A1E000DB695B68B2F5401F84B222D0C20217D58A
:10A1F000C0F30342032505FA02F223EA020343F007
:10A20000706321B1420D120104FA02F423430022CB
:10A21000C4F201020028B4BFD361536030BC704760
:10A22000420D120104FA02F223EA020343F07063C2
:10A23000E7E70022C4F20102556823F0706325F0BD
:10A2400070655560DDE700BF08B54FF4A843C4F260
:10A25000000398420BD001214FF4800000F08CF9EC
:10A260004FF480000021BDE8084000F085B90121CD
:10A270004FF4001000F080F94FF400100021BDE809
:10A28000084000F079B900BFF0B587B00446868871
:10A2900001A80D4600F0F2F8039A4DF68363C4F26C
:10A2A0001B33A3FB021326F03F06980C3604360C32
:10A2B00087B23E43A680238848F2A06123F00103C1
:10A2C0001B041B0C23802B68C0F201018B4222D897
:10A2D0005B00B2FBF3F292B201372784032A98BFE6
:10A2E0000422A28323889BB243F0010323802388A6
:10A2F000698923F48163AA8823F002031B040A43BB
:10A300001B0C13439BB223802A89AB8913439BB256
:10A31000238107B0F0BDEE884BF6FF718E421DBF62
:10A3200003EB830303EB8303B2FBF3F203EB43037F
:10A330000CBFB2FBF3F242F4804292B213051B0D44
:10A340000BB942F001024FF4967101FB00F044F6A4
:10A35000D351C1F2620181FB00318909013142F41C
:10A3600000422184BDE700BF002341F28832026031
:10A3700083804BF6FF72038143814FF48043C28098
:10A3800083817047038829B923F001031B041B0C48
:10A39000038070479BB243F001030380704700BF06
:10A3A000038829B923F480731B041B0C03807047B6
:10A3B0009BB243F480730380704700BF038829B9C0
:10A3C00023F400731B041B0C038070479BB243F4FF
:10A3D00000730380704700BF038829B923F48063AA
:10A3E0001B041B0C038070479BB243F48063038003
:10A3F000704700BF01827047008AC0B2704700BF3B
:10A400001AB901F0FE010182704741F00101018299
:10A41000704700BF038819B95B045B0C0380704769
:10A420006FEA43436FEA53439BB20380704700BF18
:10A4300082B000230A0F0093019301900092009BC9
:10A4400021F07F4153B1019B14330193019B1B68A1
:10A4500019420CBF0020012002B07047019B090C7B
:10A4600018330193F2E700BF4FF48053C4F20203A4
:10A470005A6822F4404210435860704710B44FF4B9
:10A480008053C4F202035A6802F00C02042A01D07D
:10A49000082A28D04FF49052C0F27A0202604FF49A
:10A4A0008053C4F202035C681C49C4F303140C5DBE
:10A4B00022FA04F242605C68C4F302240C5D22FAC2
:10A4C00004F484605C68C4F3C224095D22FA01F2DA
:10A4D000C2605B681249C3F38133CB5CB2FBF3F219
:10A4E000026110BC70475A685968C2F38342023255
:10A4F000CC030AD55B68990307D44FF49053C0F29C
:10A500007A0303FB02F20260C9E74FF41063C0F262
:10A510003D0303FB02F20260C1E700BFD40100204B
:10A52000D00100204FF48053C4F202035A6919B9D4
:10A5300022EA00005861704710435861704700BF1D
:10A540004FF48053C4F202039A6919B922EA000059
:10A550009861704710439861704700BF4FF4805373
:10A56000C4F20203DA6919B922EA0000D86170471F
:10A570001043D861704700BF4FF48053C4F2020308
:10A580001A6919B922EA000018617047104318616E
:10A59000704700BF70B44FF430524FF45054C4F2BF
:10A5A00001020388C4F20104904218BFA0429BB28A
:10A5B00014BF0022012208D04FF48064C4F20004CA
:10A5C000B0F1804F18BFA04236D14FF68F754C883E
:10A5D0001D4045EA04034FF4A0564FF48055C4F2E1
:10A5E0000005C4F20006B04218BFA8421FBFCD88C4
:10A5F0004FF6FF441C4044EA050303808B888385A3
:10A600000B8803855AB94FF488424FF48043C4F253
:10A610000102C4F20103984218BF904205D10B7A9F
:10A6200003860123838270BC70474FF49043C4F2C9
:10A6300001039842F5D1F2E74FF440654FF400640E
:10A64000C4F20005C4F20004A04218BFA842C2D15F
:10A65000BBE700BF038C2DE9F00123F001031B04CD
:10A660001B0C0384038C0D8984884F88028B2F4335
:10A6700022F0730223F002034FF450564FF430558A
:10A6800012041B04B1F800C0C4F20106C4F20105B3
:10A69000120C1B0CBFB2A84218BFB042A4B242EACF
:10A6A0000C0247EA03030BD04FF488464FF4804571
:10A6B000C4F20106C4F20105A84218BFB0421ED17F
:10A6C0004FF6F775B1F80AC0B1F80E808F891D40BA
:10A6D00045EA0C0C4FF6FB738E884FF6FF4548EAAF
:10A6E000070725400CEA0303BCB233432C438480A4
:10A6F0000283CA8882860384BDE8F00170474FF464
:10A700009045C4F20105A842F1D1D9E700234FF6E4
:10A71000FF7181800380C38043800372704700BF54
:10A720000023038043808380C3800381438183812E
:10A73000C3817047038829B923F001031B041B0C54
:10A74000038070479BB243F001030380704700BF52
:10A75000B0F8443021B95B045B0CA0F8443070477A
:10A760006FEA43436FEA53439BB2A0F8443070470B
:10A7700083899BB21AB923EA010181817047194389
:10A780008181704783899BB21AB923EA01018181D3
:10A790007047194381817047038829B923F08003EA
:10A7A0001B041B0C038070479BB243F080030380A3
:10A7B000704700BF038B23F008031B041B0C1943D5
:10A7C00001837047C94389B20182704770B5038A1B
:10A7D000CA8823F440531B041B0C13430382838950
:10A7E00004468A88088923F4B0530D4623F00C03ED
:10A7F000498902431B040A431B0C13439BB2A381E8
:10A80000A38AAA8923F440731B041B0C86B013434C
:10A81000A38201A8FFF732FE4FF46053A289C4F26D
:10A8200001039C4212B20CBF049B039B002A21DB54
:10A83000286803EB830303EB83038000B3FBF0F191
:10A8400048F21F53C5F2EB13A3FB0102A089520982
:10A8500000B216016425002802FB151213DB120159
:10A860003232A3FB0203C3F3431333439BB223816E
:10A8700006B070BD2A6803EB830303EB8303520029
:10A88000B3FBF2F1DCE7D2003232A3FB0213C3F3D5
:10A8900042133343EAE700BF4FF41652002302602D
:10A8A0000C228380C380038142818381704700BF73
:10A8B000838929B923F400531B041B0C838170473F
:10A8C0009BB243F400538381704700BF01F01F0324
:10A8D00010B4C1F342110124A14204FA03F30DD0D4
:10A8E00002290DD014302AB9026822EA030303605A
:10A8F00010BC7047026813430360F9E70C30F2E7BD
:10A900001030F0E7C905C90D818070478088C00507
:10A91000C00D7047838919B95B045B0C8381704754
:10A920006FEA43436FEA53439BB28381704700BF92
:10A93000C1F3421310B401F01F020124012B04FAE9
:10A9400002F416D0022B0CBF028A828A92B22240F5
:10A950000123090A03FA01F103889BB219420CBFD3
:10A9600000200120002A0CBF002000F0010010BCD4
:10A970007047828992B22240EAE700BF090A0123A8
:10A9800003FA01F3DB439BB2038070470649074A91
:10A99000074B9A42BEBF51F8040B42F8040BF8E78C
:10A9A0000448804704480047C8FA00080000002017
:10A9B000A802002045AA0008410100081F49204ABA
:10A9C000002301E041F8043B9142FBD3FCF778FF00
:10A9D000FEE7FEE7FEE7FEE7FEE7FEE7FEE7FEE74F
:10A9E000FEE7FEE7FEE7FEE7FEE7FEE7FEE7FEE73F
:10A9F000FEE7FEE7FEE7FEE7FEE7FEE7FEE7FEE72F
:10AA0000FEE7FEE7FEE7FEE7FEE7FEE7FEE7FEE71E
:10AA1000FEE7FEE7FEE7FEE7FEE7FEE7FEE7FEE70E
:10AA2000FEE7FEE7FEE7FEE7FEE7FEE7FEE7FEE7FE
:10AA3000FEE7FEE7FEE7FEE7FEE7FEE7A8020020EE
:10AA4000183A00204FF48053C4F202031968002220
:10AA500041F0010119605968CFF6FF020A405A60BF
:10AA60001A68002122F0847222F480321A601A6877
:10AA700082B022F480221A6058681A4620F4FE0040
:10AA800058604FF41F00986000910191196841F4DB
:10AA90008031196003E0009BB3F5A06F09D0136803
:10AAA00003F400330193009B01330093019B002BBF
:10AAB000F1D04FF48053C4F202031B6813F4003347
:10AAC00008BF019301D001230193019B012B08D002
:10AAD0004FF46D43CEF200034FF000629A6002B073
:10AAE00070474FF40052C4F2020211684FF48053D1
:10AAF00041F0100111601168C4F2020321F003015A
:10AB000011601068194640F0020010605A685A60DF
:10AB10005A685A605A6842F480625A605A6822F44D
:10AB20007C125A605A6842F4E8125A601A6842F07D
:10AB300080721A600A684FF480539201C4F20203D3
:10AB4000F8D559681A4621F003015960596841F057
:10AB500002015960536803F00C03082BFAD1B7E7E0
:10AB60004FF48053C4F202035A6802F00C02082A20
:10AB70001CBF4FF49052C0F27A020DD04FF48053B4
:10AB8000C4F202035B681049C3F30313CB5C22FADF
:10AB900003F20E4B1A6070475A685968C2F3834239
:10ABA0000232C80309D55B68990306D44FF4905369
:10ABB000C0F27A0303FB02F2E0E74FF41063C0F245
:10ABC0003D0303FB02F2D9E7E4010020F401002079
:10ABD00000210A2200F046BC08B5074B044613B119
:10ABE0000021AFF30080054B1868836A03B19847D2
:10ABF000204601F071F800BF000000001CF90008B9
:10AC000070B50E4B0E4D0024ED1AAD101E4603E03C
:10AC100056F8242090470134AC42F9D101F05EF897
:10AC2000084D094B0024ED1AAD101E4603E056F8FE
:10AC3000242090470134AC42F9D170BDA00200201D
:10AC4000A0020020A4020020A002002038B5074B7B
:10AC500005461C68E36B1BB9242000F00DF8E06387
:10AC6000E16B2846BDE8384000F002B858020020E9
:10AC7000002200F0C3B80000024B0146186800F043
:10AC800047BA00BF5802002010B5002302E0CC5C98
:10AC9000C45401339342FAD110BD8218034601E037
:10ACA00003F8011B9342FBD1704700002DE9F74FD9
:10ACB000064600F09FFF40F2B1739E42024640F309
:10ACC00096806FF4F663F318A6F2B2719B1040F20F
:10ACD0006D1505FB0135A6F26D716FF0630391FBF5
:10ACE000F3F36FF4C861ED1871184FF4C87391FB5A
:10ACF000F3F16D18642196FBF1FC01FB1C6C96FBD3
:10AD0000F3F103FB11614660D1F1010106F0030686
:10AD100038BF002101960346022407261F7A4A2FD6
:10AD200011D15F69019805EB070810B9BCF1000F5C
:10AD300000D121B13B2FD4BF0027012700E00F46EF
:10AD40004744013F3FE0442F02D15F69EF193AE0E9
:10AD5000019F37B9BCF1000F0CBF89464FF00109C4
:10AD600000E0894623484FF0300808FB0909D3F872
:10AD70000CA0A846012705E009EB870B5BF804BC93
:10AD80000137D8445745F7DB08F1040797FBF6FB7A
:10AD900006FB1B7B5F691869BAF1010FB8BF4FF062
:10ADA000010AB7EB0B0748BF073700F1FF3B0AF179
:10ADB000FF3A072000FB0B7759F82A9000E0073F85
:10ADC0004F45FCDA47449869DFF82C80013C08FBCA
:10ADD0000707186A074443F81C7F9FD1936BD1691A
:10ADE0009942ACBF002301231360012000E0002042
:10ADF000BDE8FE8F20F90008805101002DE9F843DD
:10AE000080460C46174600F0F5FED8F800109B4A25
:10AE1000064691FBF2F302FB131104E001F5A831A1
:10AE200001F5C071013B0029F8DB4FF4616091FB33
:10AE3000F0F200FB12113C20A26091FBF0F200FB4B
:10AE40001211626021601A1D072192FBF1F001FBD3
:10AE50001022002AB8BF0732002BA26140F2B2755F
:10AE60004FF4C8704FF0640CDFF81C9217DBA90791
:10AE700004D195FBFCF20CFB125242B995FBF0F1A8
:10AE800000FB1151D1F1010138BF002100E0012187
:10AE900059F82120934218DB01359B1AE7E7013D61
:10AEA000AA0704D195FBFCF20CFB125242B995FBA8
:10AEB000F0F100FB1151D1F1010138BF002100E098
:10AEC000012159F821209B18E9D4A5F26C72626126
:10AED0006B4A4FF0300909FB01290022E36122612E
:10AEE00002E001319B1A2161216959F82120934226
:10AEF000F7DA0133E360002F40F0BB8000F0A6FCDE
:10AF0000604B1B681BB373689D4205D13168D8F84C
:10AF10000030F26931B90CE02846FFF7C7FE00287F
:10AF2000F4D110E093420CDBB26B934209DA0123B7
:10AF30000BE09342FBDAB26B9342ACBF00230123D8
:10AF400003E0002301E04FF0FF33236200E02762BB
:10AF5000236A4FF46160012B0CBFF36B336A2568E1
:10AF600093FBF0F200FB12333C2093FBF0F100FB6B
:10AF700011336068EB1A411AA0683B2BC2EB000248
:10AF800023606160A26003DD013161603C3B04E04D
:10AF9000002B03DA013961603C33236063683B2B8B
:10AFA00003DD0132A2603C3B04E0002B03DA013AEE
:10AFB000A2603C336360A368172B1FDDE269013296
:10AFC000E261A2690132062AC8BF0022A261E268DA
:10AFD000183B0132A3602369E26059F823108A42CA
:10AFE00044DD0133521A0C2BE26023613ED16269C9
:10AFF0000023013223616261E36137E0002B35DA1F
:10B00000E269013AE261A269013A48BF0622A261FF
:10B01000E2681833013AE260A3603ABB2369013B5E
:10B0200001D423611EE00B23236163695A1E12F0D1
:10B03000030F626103F26B7305D1642293FBF2F19B
:10B0400002FB113252B94FF4C87293FBF2F102FBCA
:10B050001133D3F1010338BF002300E0012303F5CE
:10B06000B673E361236959F82330E36000F0EFFB26
:10B0700001E0002323622046BDE8F88380510100EF
:10B0800020F900087438002080F9000830B5002944
:10B090003BD051F8042C0B1F1C49002AB8BF9B1849
:10B0A0000A6812B95A600B6030BD93420CD219681D
:10B0B0005818904203D15A588918426819605A604A
:10B0C000124A136030BD0A46516809B19942FAD953
:10B0D000146815199D420AD11B68E318D0188842DC
:10B0E000136012D108681B1813604B680CE002D97A
:10B0F0000C23036030BD18681C188C4203D10C6807
:10B100004968001918605960536030BD70380020DC
:10B11000F8B5CD1C25F0030508350C2D38BF0C25DE
:10B12000002D064645DB8D4200D242E0234B1B68D2
:10B130001C4612E02268521B0DD40B2A02D9226051
:10B14000A4181EE0A34203D163681C4A136021E0E7
:10B1500062685A601EE023466468002CEAD123E04E
:10B160003046214600F06AF838602946304600F043
:10B1700065F8431C01461CD0C41C24F0030484421F
:10B1800001D1256006E03046611A00F057F8013021
:10B19000F7D10EE004F10B00231D20F00700C31AC5
:10B1A0000AD05A42E250F8BD054F3B68002BDCD173
:10B1B000D6E70C2333600020F8BD00BF70380020B4
:10B1C0006C3800201A4B10B51C68A36BD3B918203B
:10B1D000FFF752FD43F20E33A06303804AF6CD33EE
:10B1E000438041F2342383804EF26D63C3804DF679
:10B1F000EC630381052343810B2383810122002318
:10B20000C0E90423A46B0B492069626941430A4BDE
:10B2100003FB0212A0FB03015118012200231218A4
:10B2200043EB0103C4E9042323F0004010BD00BF39
:10B23000580200202DF451582D7F954C38B5064CFE
:10B24000002305460846236000F02CFD431C02D174
:10B25000236803B12B6038BD143A00200EB400B54A
:10B260004FF402719CB0ADF814106FF000410491DE
:10B2700007914FF6FF711DABADF81610084953F852
:10B28000042B02900690086802A9019300F0E6F9E9
:10B29000029B00221A701CB05DF804EB03B07047EB
:10B2A00058020020C9B2034610F8012B12B18A429D
:10B2B000F9D102E0002918BF00231846704710F8A2
:10B2C000012B11F8013B012A28BF9A42F7D0D01A6E
:10B2D0007047034611F8012B03F8012B002AF9D11E
:10B2E0007047034613F8012B002AFBD1181A0138C6
:10B2F000704770B5A2B108E0012A03D128781B7805
:10B30000C01A70BD013A002CF8D00B460546002A41
:10B31000F4D010F8016B1C780131B442ECD0EDE7A9
:10B32000104670BD30B50139034609E011F8015FE0
:10B33000013A03F8015B1C4615B99B18002205E091
:10B340001C46002AF2D1F8E704F8012B9C42FBD1FD
:10B3500030BD00002DE9F74F01904148D0F8009032
:10B360000846044614F8015B09EB05067778204689
:10B3700007F00807FFB2002FF3D12D2D03D114F8E9
:10B38000015B012704E02B2D04BF244614F8015B68
:10B39000002B5ED0102B08D158E02078782801D0FF
:10B3A00058284ED1657810230234002F0CBF6FF05F
:10B3B00000404FF00040B0FBF3FA002603FB1A08F0
:10B3C000304609EB050C9CF801C00CF0040B5FFA49
:10B3D0008BFBBBF1000F01D0303D0BE01CF0030CE8
:10B3E0001BD0BCF1010F14BF4FF0570C4FF0370CBE
:10B3F000CCEB05059D4210DAB6F1FF3F0AD050456F
:10B4000006D801D1454503DC03FB0050012601E0CD
:10B410004FF0FF3614F8015BD3E7731C0AD1002FFD
:10B4200001990CBF6FF000404FF0004022230B60E9
:10B4300022B912E007B140427AB106B1611E116033
:10B440000BE03025002BB0D10823AEE7302DACD176
:10B45000A3E7302DA1D00A23A7E7BDE8FE8F00BFE8
:10B460005C02002030B51346044A05460C461068BD
:10B4700029462246BDE83040FFF76CBF5802002045
:10B480002DE9F74F01903D48D0F80090084604465A
:10B4900014F8015B09EB05067778204607F00807EA
:10B4A000FFB2002FF3D12D2D03D114F8015B01273A
:10B4B00004E02B2D04BF244614F8015B002B57D069
:10B4C000102B08D151E02078782801D0582847D196
:10B4D0006578102302344FF0FF3ABAFBF3FA03FB0E
:10B4E0000AF000266FEA0008304609EB050C9CF8CC
:10B4F00001C00CF0040B5FFA8BFBBBF1000F01D015
:10B50000303D0BE01CF0030C1BD0BCF1010F14BF4D
:10B510004FF0570C4FF0370CCCEB05059D4210DA7D
:10B52000B6F1FF3F0AD0504506D801D1454503DCAE
:10B5300003FB0050012601E04FF0FF3614F8015BD9
:10B54000D3E7731C05D1019922230B60304622B941
:10B5500012E007B140427AB106B1611E11600BE002
:10B560003025002BB7D10823B5E7302DB3D1AAE79A
:10B57000302DA8D00A23AEE7BDE8FE8F5C02002084
:10B5800030B51346044A05460C4610682946224643
:10B59000BDE83040FFF774BF580200202DE9F047A6
:10B5A0008D688146AB420C4692461F463FD38A893E
:10B5B00012F4906F39D0266809696369C1EB0608F7
:10B5C00003265E43022508F1010302F4806296FB24
:10B5D000F5F6DB1912B29E4238BF1E4682B13146E3
:10B5E000FFF796FD054600B913E021694246FFF7D3
:10B5F0004BFBA38923F4906343F08003A3810CE009
:10B60000324600F022FB054638B948462169FFF76B
:10B610003DFD0C23C9F8003018E025616661454402
:10B62000C8EB06062560A6603D46AF4200D23D4607
:10B630002A462068514600F0EFFAA36800205B1B01
:10B64000A36023685D192560BDE8F087A3894FF0EA
:10B65000FF3043F04003A381BDE8F0872DE9F04FB0
:10B660009DB003938B89064603F080031BB20D4601
:10B67000144663B10B6953B94021FFF749FD2860B7
:10B68000286110B90C233360D0E040236B610023A4
:10B69000099320238DF82930DFF89C813023DFF8CF
:10B6A0009C918DF82A3023469A4613F8012B1AB93B
:10B6B000BAEB040B0FD002E0252AF5D1F8E73046AB
:10B6C000294622465B46FFF769FF013000F0A7805C
:10B6D000099B5B4409939AF80030002B00F09F808F
:10B6E00000234FF0FF3204930793059206938DF8E1
:10B6F00053301A930AF1010A4FF0010B05E0C8EB31
:10B7000000000BFA00F00343049354464A482178A2
:10B71000052200F073FA0AF1010A049B0028EED119
:10B72000D90602D520228DF853201A0702D52B22E4
:10B730008DF8532022782A2A03D0079B21460A201D
:10B7400010E0039A111D12680391002A01DB079291
:10B7500004E0524243F0020307920493013408E0EC
:10B7600000FB03230C4622780131303A092AF7D92D
:10B77000079323782E2B19D163782A2B09D1039BA9
:10B7800002341A1D1B680392002BB8BF4FF0FF3321
:10B790000BE0611C00230A2001E000FB03230C46A0
:10B7A00022780131303A092AF7D9059323482178C4
:10B7B000032200F023FA40B14023C9EB000003FA52
:10B7C00000F0049B01340343049314F8011B1C484C
:10B7D00006228DF8281000F011FA88B1194B33B900
:10B7E000039B073323F007030833039313E003ABF2
:10B7F0000093304604A92A46134BAFF3008007E0BC
:10B8000003AB0093304604A92A460F4B00F092F890
:10B81000431C074603D0099BDB19099343E7AB8917
:10B8200003F040031BB20BB9099801E04FF0FF3061
:10B830001DB0BDE8F08F00BF88F900088EF9000840
:10B8400092F90008000000009DB50008704770479D
:10B850002DE9F04715461F468A680B6906469A424D
:10B86000A8BF13462B6091F843200C46DDF82080DA
:10B870000AB101332B602368990602D52B68023385
:10B880002B60236813F0060916D094F84330226821
:10B89000003318BF0123920616D41EE00123304660
:10B8A00039465246C047013003D14FF0FF30BDE862
:10B8B000F08709F1010901E004F1190AE1682B6838
:10B8C000CB1A9945EADBE0E7E218302182F8431011
:10B8D00094F84510023382F844103046394604F19A
:10B8E0004302C0470130E0D023682A68E16803F0D2
:10B8F0000603042B08BFC2EB01052369A2680CBF35
:10B9000025EAE57500259A42C4BFC3EB0203ED1892
:10B910004FF000091A3408E0012330463946224628
:10B92000C0470130C1D009F10109A945F4DB00206D
:10B93000BDE8F0872DE9FF470E7E91466E2E8046CA
:10B940000C469A460C9D01F1430200F0AF800FD8DF
:10B95000632E1DD006D8002E00F0C080582E40F077
:10B96000D0804FE0642E1CD0692E40F0CA8018E0D1
:10B97000732E00F0B78005D86F2E2BD0702E40F0BC
:10B98000C08043E0752E25D0782E40F0BA8041E08B
:10B990002B6801F142071A1D1B682A6081F84230AA
:10B9A000B3E021682B6811F0800F02D0191D2960C7
:10B9B00008E011F0400F03F10401296002D0B3F94F
:10B9C000005000E01D68002D45DA2D236D4284F8FB
:10B9D000433040E021682B6811F0800F02D0191D20
:10B9E000296007E011F0400F03F10401296001D044
:10B9F0001D8800E01D68237E5F486F2B14BF0A235B
:10BA0000082324E081F845605B4807E00B6843F0B9
:10BA100020030B607823594884F8453021682B684F
:10BA200011F0800F03F104062E6000D003E04F06F2
:10BA300001D51D8800E01D68CE0744BF41F02001FC
:10BA400021601DB9236823F0200323601023002107
:10BA500084F8431001E048480A236668002EA66077
:10BA600003DB216821F00401216005B96EB104F106
:10BA70004201B5FBF3F603FB1655455D0F4601F891
:10BA800001593546002EF4D100E01746082B0AD1A3
:10BA90002368DB0707D561682369994203DC3023FB
:10BAA00007F8013C013FD21B226133E009682B6893
:10BAB00011F0800F05D0191D2960196863690B60AA
:10BAC0000CE011F0400F03F10401296003D0196864
:10BAD00063690B8002E061691B68196000232361C0
:10BAE000174617E02B681A1D2A601F683846FFF7B3
:10BAF000F8FB63682061984288BF23612369636013
:10BB000005E004F1420784F8426001232361002329
:10BB100084F84330CDF800A04046214603AA4B46A6
:10BB2000FFF796FE013002D14FF0FF3021E0404692
:10BB300049463A462369D0470130F5D02368980733
:10BB40000ED4E068039B9842B8BF184611E0012369
:10BB5000404649463246D0470130E5D0013502E043
:10BB6000002504F11906E168039BCB1A9D42EEDB28
:10BB7000E7E704B0BDE8F08799F90008AAF90008E2
:10BB800030B5141E9BB0054604DA8B2303604FF0DA
:10BB9000FF301DE04FF40272ADF80C2000910491CB
:10BBA00001D0611E00E021464FF6FF72029105911F
:10BBB000ADF80E2028461A4669461E9BFFF74EFD3B
:10BBC000431C01DA8B232B6014B1009B00221A70F6
:10BBD0001BB030BD73B50093054B06460D461446A9
:10BBE000186831462A462346FFF7CAFF7CBD00BFCE
:10BBF00058020020004870476002002010B5C9B20A
:10BC00000346821803E0047801338C4203D0934248
:10BC10001846F8D1002010BD814210B511D28C1801
:10BC2000A0420ED253428118E418CB1801E0A15C67
:10BC3000995412F1FF32FAD210BDCC5CC4540133D6
:10BC400000E000239342F8D110BDF8B50646154632
:10BC50000C4621B91146BDE8F840FFF759BA1AB9A8
:10BC6000FFF714FA2C4612E000F013F8A8420ED2A7
:10BC700030462946FFF74CFA074638B121462A4696
:10BC8000FFF702F830462146FFF700FA3C4620460F
:10BC9000F8BD51F8040C002802DA04390B58C0181A
:10BCA00004387047094A136863B118186946884216
:10BCB00098BF106004D9064B0C221A604FF0FF3376
:10BCC00018467047034B1360EFE700BF7838002039
:10BCD000143A0020183A0020FEE700BFF8B500BF74
:10BCE000F8BC08BC9E467047F8B500BFF8BC08BC5D
:10BCF0009E46704765617374657220646174653A2D
:10BD000020253034642D253032642D253032640DE9
:10BD10000A000000536F00004D6F000044690000EE
:10BD20004D690000446F000046720000536100003E
:10BD300053750000547500005765000054680000FA
:10BD40004443463737204572726F723A204869671C
:10BD5000682070756C7365203C3D20350000000044
:10BD60004443463737204572726F723A20486967FC
:10BD7000682070756C7365203E3D203235000000F0
:10BD80004443463737204572726F723A20706172B1
:10BD900069747920503120696E636F7272656374C3
:10BDA000000000004443463737204572726F723AF4
:10BDB0002070617269747920503220696E636F72ED
:10BDC00072656374000000004443463737204572B3
:10BDD000726F723A207061726974792050332069F1
:10BDE0006E636F72726563740000000000000000F3
:10BDF000000000003C42423C0000000024182442A5
:10BE00007E42420024003C4242423C002400424226
:10BE100042423C007C427C427C40400000000000EA
:10BE20000000000000000000000000000000000012
:10BE30000000000000000000000000000000000002
:10BE400000000000000000000000000000000000F2
:10BE500000000000000000000000000000000000E2
:10BE600000000000000000000000000000000000D2
:10BE700000000000000000000000000000000000C2
:10BE800000000000000000000000000000000000B2
:10BE900000000000000000000000000000000000A2
:10BEA0000000000000000000000000000000000092
:10BEB0000000000000000000000000000000000082
:10BEC0000000000000000000000000000000000072
:10BED0000000000000000000000000000000000062
:10BEE0000000000000000000000000000000000052
:10BEF000000000003838381000383800EEEE4400FA
:10BF0000000000002828FE28FE2828007C92907C53
:10BF100012927C00E2A4E8102E4A8E003048307065
:10BF20008A847A0038381020000000001820404031
:10BF3000402018003008040404083000004428EEB3
:10BF4000284400000010107C101000000000003891
:10BF5000381020000000007C0000000000000000FD
:10BF60003838380002040810204080003844A2927B
:10BF70008A4438001030501010107C007C82027C03
:10BF80008080FE007C82027C02827C00808484FEB1
:10BF900004040400FE80807C02827C007C8280FCA1
:10BFA00082827C00FE840810202020007C82827C1B
:10BFB00082827C007C82827E02827C0010281000BB
:10BFC00010281000383800383810200008102040A1
:10BFD0002010080000007C007C00000020100804F5
:10BFE000081020007C82020C100010007C82BAAA8B
:10BFF000BC827C0010284482FE828200FC8282FC8B
:10C000008282FC007C82808080827C00FC82828232
:10C010008282FC00FE8080F88080FE00FE8080F836
:10C02000808080007C82809E82827C00828282FE70
:10C0300082828200381010101010380002020202B2
:10C0400082827C00848890E0908884008080808058
:10C050008080FE0082C6AA928282820082C2A29260
:10C060008A8682007C82828282827C00FC8282FCC0
:10C07000808080007C8282828A847A00FC8282FCBA
:10C08000888482007C82807C02827C00FE101010FA
:10C09000101010008282828282827C0082828282E0
:10C0A000442810008292929292926C00824428104E
:10C0B000284482008244281010101000FE0408104A
:10C0C0002040FE007C40404040407C0080402010EA
:10C0D000080402007C04040404047C0010284400CA
:10C0E00000000000000000000000FE0038381008CA
:10C0F00000000000001824427E424200007C427C86
:10C1000042427C00003C424040423C00007C4242B3
:10C1100042427C00007E407C40407E00007E407CAD
:10C1200040404000003C42404E423C000042427EC3
:10C130004242420000080808080808000002020203
:10C1400002423C00004244784844420000404040E3
:10C1500040407E000042665A424242000042625223
:10C160004A464200003C424242423C00007C42427D
:10C170007C404000003C42424A443A00007C42423B
:10C180007C444200003C403C02423C00003E080827
:10C19000080808000042424242423C00004242423B
:10C1A00042241800004242425A66420000422418CB
:10C1B000182442000022140808080800007E040821
:10C1C00010207E00384040C0404038001010100061
:10C1D00010101000380404060404380060920C00AB
:10C1E000000000000000000000000000000001004E
:10C1F0000100020002000300030004000400050027
:10C20000050006000700080009000B000D000E00E5
:10C21000100012001400170019001C001F0021005C
:10C22000240028002B002E003200360039003D008B
:10C23000420046004A004F00540059005E0063006F
:10C2400069006E0074007A00800086008C00930004
:10C250009900A000A700AE00B600BD00C500CD004B
:10C26000D500DD00E500EE00F600FF004E6F6E65C4
:10C27000000000005261696E626F7700466164657C
:10C2800000000000526F6C6C000000004578706C7C
:10C290006F64650052616E646F6D0000536E616B78
:10C2A0006500000054656C657479706500000000DD
:10C2B00043756265000000004D617472697800008A
:10C2C00044726F700000000053717565657A6500F7
:10C2D0004E6F726D616C0000436C6F636B320000D7
:10C2E000080809090A0A0B0B0C0C0D0D0E0E0F00A5
:10C2F0000000000000000000000522000000000017
:10C3000000152200000000000007220000000000CD
:10C3100000122200000000000010220000000000B7
:10C32000000C220000000000000E220000000000AF
:10C330000013220000000000001122000000000095
:10C340000017220000000000000F22000000000083
:10C350000016220000000000000717220000000065
:10C360000012172200000000001017220000000039
:10C37000000B172200000000000D17220000000033
:10C380000013172200000000001117220000000017
:10C39000001922000000000000041819220000000B
:10C3A00000151819220000000007181922000000CB
:10C3B00000121819220000000010181922000000B5
:10C3C000000C181922000000000E181922000000AD
:10C3D0000013181922000000001118192200000093
:10C3E000001B2200000000000004181B22000000B7
:10C3F0000015181B220000000007181B2200000077
:10C400000012181B220000000010181B2200000060
:10C41000000C181B22000000000E181B2200000058
:10C420000013181B220000000011181B220000003E
:10C43000001A2200000000000004181A2200000068
:10C440000015181A220000000007181A2200000028
:10C450000012181A220000000010181A2200000012
:10C46000000C181A22000000000E181A220000000A
:10C470000013181A220000000011181A22000000F0
:10C48000001C2200000000000004181C2200000014
:10C490000015181C220000000007181C22000000D4
:10C4A0000012181C220000000010181C22000000BE
:10C4B000000C181C22000000000E181C22000000B6
:10C4C0000013181C220000000011181C220000009C
:10C4D000000000000000000000091E220000000013
:10C4E00000151F220000000000071F2200000000AE
:10C4F00000121F220000000000101F220000000098
:10C50000000C1F2200000000000E1F22000000008F
:10C5100000131F220000000000111F220000000075
:10C5200000171F2200000000000F1F220000000063
:10C5300000161F22000000000007171F2200000045
:10C540000012171F220000000010171F2200000019
:10C55000000B171F22000000000D171F2200000013
:10C560000013171F220000000011171F22000000F7
:10C5700000191F2200000000000418191F220000EB
:10C58000001518191F220000000718191F220000AB
:10C59000001218191F220000001018191F22000095
:10C5A000000C18191F220000000E18191F2200008D
:10C5B000001318191F220000001118191F22000073
:10C5C000001B1F22000000000004181B1F22000097
:10C5D0000015181B1F2200000007181B1F22000057
:10C5E0000012181B1F2200000010181B1F22000041
:10C5F000000C181B1F220000000E181B1F22000039
:10C600000013181B1F2200000011181B1F2200001E
:10C61000001A1F22000000000004181A1F22000048
:10C620000015181A1F2200000007181A1F22000008
:10C630000012181A1F2200000010181A1F220000F2
:10C64000000C181A1F220000000E181A1F220000EA
:10C650000013181A1F2200000011181A1F220000D0
:10C66000001C1F22000000000004181C1F220000F4
:10C670000015181C1F2200000007181C1F220000B4
:10C680000012181C1F2200000010181C1F2200009E
:10C69000000C181C1F220000000E181C1F22000096
:10C6A0000013181C1F2200000011181C1F2200007C
:10C6B000004100000000000000091E2200000000F0
:10C6C00000151F220000000000071F2200000000CC
:10C6D00000121F220000000000101F2200000000B6
:10C6E000000C1F2200000000000E1F2200000000AE
:10C6F00000131F220000000000111F220000000094
:10C7000000171F2200000000000F1F220000000081
:10C7100000161F22000000000007171F2200000063
:10C720000012171F2200000001030000000000009B
:10C73000000B171F22000000000D171F2200000031
:10C740000013171F220000000011171F2200000015
:10C7500001171F202600000001111F2026000000E5
:10C7600001131F2026000000010E1F2026000000DC
:10C77000010C1F202600000001101F2026000000D1
:10C7800001121F202600000001071F2026000000C4
:10C7900001151F202600000001091F2026000000AF
:10C7A000012600000000000001091E2226000000F2
:10C7B00001151F222600000001071F22260000008D
:10C7C00001121F222600000001101F222600000077
:10C7D000010C1F2226000000010E1F22260000006F
:10C7E00001131F222600000001111F222600000055
:10C7F00001171F2226000000010F1F222600000043
:10C8000001161F22260000000107171F2226000024
:10C810000112171F22260000012400000000000062
:10C820000112171F200000000107171F2000000041
:10C8300001161F2000000000010F1F200000000053
:10C8400001171F200000000001111F200000000040
:10C8500001131F2000000000010E1F200000000037
:10C86000010C1F200000000001101F20000000002C
:10C8700001121F200000000001071F20000000001F
:10C8800001151F200000000001091E20000000000B
:10C89000004100000000000000091E22000000000E
:10C8A00000151F220000000000071F2200000000EA
:10C8B00000121F220000000000101F2200000000D4
:10C8C000000C1F2200000000000E1F2200000000CC
:10C8D00000131F220000000000111F2200000000B2
:10C8E00000171F2200000000000F1F2200000000A0
:10C8F00000161F22000000000007171F2200000082
:10C900000012171F22000000000322000000000098
:10C91000000B171F22000000000D171F220000004F
:10C920000013171F220000000011171F2200000033
:10C9300000191F220000000001111F202600000026
:10C9400001131F2026000000010E1F2026000000FA
:10C95000010C1F202600000001101F2026000000EF
:10C9600001121F202600000001071F2026000000E2
:10C9700001151F202600000001091E2026000000CE
:10C98000012600000000000001091E222600000010
:10C9900001151F222600000001071F2226000000AB
:10C9A00001121F222600000001101F222600000095
:10C9B000010C1F2226000000010E1F22260000008D
:10C9C00001131F222600000001111F222600000073
:10C9D00001191F20000000000111171F2000000096
:10C9E0000113171F20000000010D171F2000000079
:10C9F000010B171F200000000124000000000000B0
:10CA00000112171F200000000107171F200000005F
:10CA100001161F2000000000010F1F200000000071
:10CA200001171F200000000001111F20000000005E
:10CA300001131F2000000000010E1F200000000055
:10CA4000010C1F200000000001101F20000000004A
:10CA500001121F200000000001071F20000000003D
:10CA600001151F200000000001091E200000000029
:10CA7000004100000000000000091E22000000002C
:10CA800000151F220000000000071F220000000008
:10CA900000121F220000000000101F2200000000F2
:10CAA000000C1F2200000000000E1F2200000000EA
:10CAB00000131F220000000000111F2200000000D0
:10CAC00000171F2200000000000F1F2200000000BE
:10CAD00000161F22000000000007171F22000000A0
:10CAE0000012171F220000000003220000000000B7
:10CAF000000B171F22000000000D171F220000006E
:10CB00000013171F220000000011171F2200000051
:10CB100000191F220000000001111F202600000044
:10CB200001131F2026000000010E1F202600000018
:10CB3000010C1F202600000001101F20260000000D
:10CB400001121F202600000001071F202600000000
:10CB500001151F202600000001091E2026000000EC
:10CB6000012600000000000001091E22260000002E
:10CB700001151F222600000001071F2226000000C9
:10CB800001121F222600000001101F2226000000B3
:10CB9000010C1F2226000000010E1F2226000000AB
:10CBA00001131F222600000001111F222600000091
:10CBB00001191F20000000000111171F20000000B4
:10CBC0000113171F20000000010D171F2000000097
:10CBD000010B171F200000000103200000000000CF
:10CBE0000112171F200000000107171F200000007E
:10CBF00001161F2000000000010F1F200000000090
:10CC000001171F200000000001111F20000000007C
:10CC100001131F2000000000010E1F200000000073
:10CC2000010C1F200000000001101F200000000068
:10CC300001121F200000000001071F20000000005B
:10CC400001151F200000000001091E200000000047
:10CC5000004100000000000000091E22000000004A
:10CC600000151F220000000000071F220000000026
:10CC700000121F220000000000101F220000000010
:10CC8000000C1F2200000000000E1F220000000008
:10CC900000131F220000000000111F2200000000EE
:10CCA00000171F2200000000000F1F2200000000DC
:10CCB00000161F22000000000007171F22000000BE
:10CCC0000012171F220000000103000000000000F6
:10CCD000000B171F22000000000D171F220000008C
:10CCE0000013171F220000000011171F2200000070
:10CCF00000191F220000000001111F202600000063
:10CD000001131F2026000000010E1F202600000036
:10CD1000010C1F202600000001101F20260000002B
:10CD200001121F202600000001071F20260000001E
:10CD300001151F202600000001091E20260000000A
:10CD4000012600000000000001091E22260000004C
:10CD500001151F222600000001071F2226000000E7
:10CD600001121F222600000001101F2226000000D1
:10CD7000010C1F2226000000010E1F2226000000C9
:10CD800001131F222600000001111F2226000000AF
:10CD900001191F20000000000111171F20000000D2
:10CDA0000113171F20000000010D171F20000000B5
:10CDB000010B171F200000000124000000000000EC
:10CDC0000112171F200000000107171F200000009C
:10CDD00001161F2000000000010F1F2000000000AE
:10CDE00001171F200000000001111F20000000009B
:10CDF00001131F2000000000010E1F200000000092
:10CE0000010C1F200000000001101F200000000086
:10CE100001121F200000000001071F200000000079
:10CE200001151F200000000001091E200000000065
:10CE3000004100000000000000091E220000000068
:10CE400000151F220000000000071F220000000044
:10CE500000121F220000000000101F22000000002E
:10CE6000000C1F2200000000000E1F220000000026
:10CE700000131F220000000000111F22000000000C
:10CE800000171F2200000000000F1F2200000000FA
:10CE900000161F22000000000007171F22000000DC
:10CEA0000012171F220000000003220000000000F3
:10CEB000000B171F22000000000D171F22000000AA
:10CEC0000013171F220000000011171F220000008E
:10CED00001171F202600000001111F20260000005E
:10CEE00001131F2026000000010E1F202600000055
:10CEF000010C1F202600000001101F20260000004A
:10CF000001121F202600000001071F20260000003C
:10CF100001151F202600000001091E202600000028
:10CF2000012600000000000001091E22260000006A
:10CF300001151F222600000001071F222600000005
:10CF400001121F222600000001101F2226000000EF
:10CF5000010C1F2226000000010E1F2226000000E7
:10CF600001131F222600000001111F2226000000CD
:10CF700001171F2226000000010F1F2226000000BB
:10CF800001161F22260000000107171F222600009D
:10CF90000112171F222600000103200000000000DC
:10CFA0000112171F200000000107171F20000000BA
:10CFB00001161F2000000000010F1F2000000000CC
:10CFC00001171F200000000001111F2000000000B9
:10CFD00001131F2000000000010E1F2000000000B0
:10CFE000010C1F200000000001101F2000000000A5
:10CFF00001121F200000000001071F200000000098
:10D0000001151F200000000001091E200000000083
:10D0100000000000000000000035000000000000DB
:10D02000002B0000000000000033000000000000A2
:10D030000032000000000000002E00000000000090
:10D040000030000000000000002800000000000088
:10D050000031000000000000002900000000000076
:10D060000038000000000000003700000000000051
:10D07000003D000000000000003338000000000008
:10D080000032380000000000002E380000000000D0
:10D09000002F3800000000000027380000000000CA
:10D0A00000313800000000000029380000000000B6
:10D0B0000039000000000000002C3639000000009C
:10D0C000002B363900000000003336390000000024
:10D0D0000032363900000000002E36390000000012
:10D0E000003036390000000000283639000000000A
:10D0F00000313639000000000029363900000000F8
:10D10000003B000000000000002C363B0000000047
:10D11000002B363B000000000033363B00000000CF
:10D120000032363B00000000002E363B00000000BD
:10D130000030363B000000000028363B00000000B5
:10D140000031363B000000000029363B00000000A3
:10D15000003C000000000000002C363C00000000F5
:10D16000002B363C000000000033363C000000007D
:10D170000032363C00000000002E363C000000006B
:10D180000030363C000000000028363C0000000063
:10D190000031363C000000000029363C0000000051
:10D1A000003E000000000000002C363E00000000A1
:10D1B000002B363E000000000033363E0000000029
:10D1C0000032363E00000000002E363E0000000017
:10D1D0000030363E000000000028363E000000000F
:10D1E0000031363E000000000029363E00000000FD
:10D1F000000000000000000000212D3F00000000A2
:10D2000000212B40000000000021334000000000FE
:10D21000002132400000000000212E4000000000EC
:10D2200000213040000000000021284000000000E4
:10D2300000213140000000000021294000000000D2
:10D2400000213840000000000021374000000000AD
:10D2500000213D4000000000002133384000000064
:10D26000002132384000000000212E38400000002C
:10D2700000212F3840000000002127384000000026
:10D280000021313840000000002129384000000012
:10D29000002139400000000000212C3639400000F8
:10D2A00000212B3639400000002133363940000080
:10D2B000002132363940000000212E36394000006E
:10D2C0000021303639400000002128363940000066
:10D2D0000021313639400000002129363940000054
:10D2E00000213B400000000000212C363B400000A4
:10D2F00000212B363B400000002133363B4000002C
:10D30000002132363B40000000212E363B40000019
:10D31000002130363B400000002128363B40000011
:10D32000002131363B400000002129363B400000FF
:10D3300000213C400000000000212C363C40000051
:10D3400000212B363C400000002133363C400000D9
:10D35000002132363C40000000212E363C400000C7
:10D36000002130363C400000002128363C400000BF
:10D37000002131363C400000002129363C400000AD
:10D3800000213E400000000000212C363E400000FD
:10D3900000212B363E400000002133363E40000085
:10D3A000002132363E40000000212E363E40000073
:10D3B000002130363E400000002128363E4000006B
:10D3C000002131363E400000002129363E40000059
:10D3D00000000000000000000111181C1F200000C8
:10D3E0000113181C1F200000010E181C1F20000034
:10D3F000010C181C1F2000000110181C1F20000029
:10D400000112181C1F2000000107181C1F2000001B
:10D410000115181C1F2000000104181C1F2000000B
:10D42000011C1F20000000000111181A1F2000001D
:10D430000113181A1F200000010E181A1F200000E7
:10D44000010C181A1F2000000110181A1F200000DC
:10D450000112181A1F2000000107181A1F200000CF
:10D460000115181A1F2000000104181A1F200000BF
:10D4700001191F20000000000111181B1F200000CF
:10D480000113181B1F200000010E181B1F20000095
:10D49000010C181B1F2000000110181B1F2000008A
:10D4A0000112181B1F2000000107181B1F2000007D
:10D4B0000115181B1F2000000104181B1F2000006D
:10D4C000011B1F2000000000011118191F2000007F
:10D4D000011318191F200000010E18191F20000049
:10D4E000010C18191F200000011018191F2000003E
:10D4F000011218191F200000010718191F20000031
:10D50000011518191F200000010418191F20000020
:10D5100001191F20000000000111171F200000004A
:10D520000113171F20000000010D171F200000002D
:10D53000010C171F200000000110171F2000000021
:10D540000112171F200000000107171F2000000014
:10D5500001161F2000000000010F1F200000000026
:10D5600001171F200000000001111F200000000013
:10D5700001131F2000000000010E1F20000000000A
:10D58000010C1F200000000001101F2000000000FF
:10D5900001121F200000000001071F2000000000F2
:10D5A00001151F200000000001091E2000000000DE
:10D5B00000173A0000000000001723263A00000080
:10D5C000000F3A0000000000000F23263A00000080
:10D5D00000163A0000000000001623263A00000062
:10D5E0000007173A0000000000071723263A000042
:10D5F0000012173A0000000000121723263A00001C
:10D600000010173A0000000000101723263A00000F
:10D61000000B173A00000000000B1723263A000009
:10D62000000D173A00000000000D1723263A0000F5
:10D630000013173A0000000000131723263A0000D9
:10D640000011173A0000000000111723263A0000CD
:10D6500000193A0000000000001923263A000000DB
:10D66000000418193A0000000004181923263A0093
:10D67000001518193A4900000015181923263A49CF
:10D68000000718193A4900000007181923263A49DB
:10D69000001218193A4900000012181923263A49B5
:10D6A000001018193A4900000010181923263A49A9
:10D6B000000C18193A490000000C181923263A49A1
:10D6C000000E18193A490000000E181923263A498D
:10D6D000001318193A4900000013181923263A4973
:10D6E000001118193A4900000011181923263A4967
:10D6F000001B3A4900000000001B23263A490000A5
:10D700000004181B3A4900000004181B23263A495C
:10D710000015181B3A4900000015181B23263A492A
:10D720000007181B3A4900000007181B23263A4936
:10D730000012181B3A4900000012181B23263A4910
:10D740000010181B3A4900000010181B23263A4904
:10D75000000C181B3A490000000C181B23263A49FC
:10D76000000E181B3A490000000E181B23263A49E8
:10D770000013181B3A4900000013181B23263A49CE
:10D780000011181B3A4900000011181B23263A49C2
:10D790000000000000000000000000000000000089
:10D7A0000000000000000000000000000000000079
:10D7B0000000000000000000000000000000000069
:10D7C0000000000000000000000000000000000059
:10D7D0000000000000000000000000000000000049
:10D7E0000000000000000000000000000000000039
:10D7F000000000003D000000350000002B0000008C
:10D8000033000000320000002E0000003000000055
:10D81000280000003100000029000000380000004E
:10D82000370000003D000000350000002B00000024
:10D8300033000000320000002E0000003000000025
:10D84000280000003100000029000000380000001E
:10D85000370000003D0000003D4100002C41000069
:10D860002B41000033410000324100002E410000F6
:10D8700030410000284100003141000029410000F2
:10D8800038410000374100003D4100002C410000BC
:10D890002B41000033410000324100002E410000C6
:10D8A00030410000284100003141000029410000C2
:10D8B00038410000374100003D4100003D41470034
:10D8C0002C4147002B414700334147003241424839
:10D8D0002E4142483041480028414800314148002B
:10D8E000294148003841434A3741434A3D414A00B3
:10D8F0002C414A002B41464A3341464A3241464A6E
:10D900002E41464A30414400284144003141440000
:10D910002941440038414400374147003D41470018
:10D920002A4100002C4100002B410000334100003F
:10D93000324100002E41000030410000284100002B
:10D94000314100002941000038410000374100000A
:10D950003D41000033384100323841002E3841004B
:10D960002F38410027384100313841002938410023
:10D97000394100002C3639412B3639413336394193
:10D9800032363941141D0000041D0000151D000031
:10D99000071D0000121D0000101D00000C1D0000DE
:10D9A0000E1D0000131D0000111D0000171D0000BA
:10D9B0000F1D0000161D0000041D0000151D0000B5
:10D9C000071D0000121D0000101D00000C1D0000AE
:10D9D0000E1D0000131D0000111D0000171D00008A
:10D9E0000F1D0000161D0000141D0000041D000086
:10D9F000151D0000071D0000121D0000101D000075
:10DA00000C1D00000E1D0000131D0000111D000064
:10DA1000171D00000F1D0000161D000007171D0038
:10DA200012171D0010171D000B171D000D171D00EC
:10DA300013171D0011171D00191D00000418191DD2
:10DA40001518191D0718191D1218191D4500000079
:10DA500000000000000000000000000000000000C6
:10DA600000000000000000000000000000000000B6
:10DA700000000000000000000000000000000000A6
:10DA80000000000000000000000000000000000096
:10DA90000000000000000000000000000000000086
:10DAA0000000000000000000000000004500000031
:10DAB0006868206D6D202831322900006868206D6B
:10DAC0006D20283234290000686820756E64206D4E
:10DAD0006D20283132290000686820756E64206D41
:10DAE0006D202832342900006D6D206E616368203E
:10DAF0006868202831322B29000000006D6D206EEF
:10DB00006163682068682028323429004F73736984
:10DB10002F4265726C696E202831322900000000A6
:10DB20004F7373692F4265726C696E202831322BF6
:10DB3000290000004F657369202831322900000058
:10DB40004F657369202831322B29000052686569BE
:10DB50006E2F52756872202831322900526865692B
:10DB60006E2F52756872202831322B290000000078
:10DB7000536368776162656E2028313229000000A6
:10DB8000536368776162656E202831322B2900006B
:10DB90005765737369202831322900005765737304
:10DBA00069202831322B2900436F756E74646F77BA
:10DBB0006E00000054656D706572617475720000CE
:10DBC000000000000002000303000707000E03002E
:10DBD0000E04000F0201000401020301020401020D
:10DBE00005010704010705010B04010B06020003F0
:10DBF000020204020604020A04020E0403000403E3
:10DC00000404030905030E04040003040407040BC1
:10DC100007050008050807050F03060006060007AC
:10DC2000060803060B03060E0407000307030B0791
:10DC30000707070E04080004080006080504080882
:10DC400004080C04080E03080E0409000409040467
:10DC5000090405090A04090E040A00040A02030A59
:10DC600002040A06030A0A030A0E040B00070B0744
:10DC7000040B0A080C00070C07050C0B070D000627
:10DC80000D00070D07030D0B040D0F030E00060E0C
:10DC9000060B0E0C040E0C060F00070F07040F0BEB
:10DCA0000700000007050000B0DA000807060000C2
:10DCB000BCDA000808050000C8DA00080806000001
:10DCC000D8DA000801030000E8DA000801040000C7
:10DCD000FCDA0008020100000CDB0008020300006F
:10DCE00020DB00080301000034DB00080303000010
:10DCF00040DB0008040100004CDB000804030000C6
:10DD00005CDB00080502000070DB00080503000072
:10DD100080DB00080601000090DB0008060300001D
:10DD20009CDB000809070000A8DB00080A000000CF
:10DD3000B4DB00082800000054696D656F7574003D
:10DD4000290D0A004F4B00004552524F520000006F
:10DD50002D200000495041444452455353200000B7
:10DD6000415020004D4F44452000000061700000EC
:10DD700054494D45200000004649524D57415245F7
:10DD800020000000434D442000000000485454503F
:10DD900020474554200000002D2D3E2000000000AB
:10DDA0003C30643E3C30613E0D0A00003C25303280
:10DDB000783E000063617020222573222C22257397
:10DDC00022000000617020222573222C222573225C
:10DDD0000000000074696D65202225732200000098
:10DDE00045535038323636204C4F474745520D0A7E
:10DDF00000000000A4EB0008ACEB0008B4EB000846
:10DE0000BCEB0008C0EB0008C4EB0008C8EB00083E
:10DE1000CCEB0008DCE40008E4E40008ECE40008D3
:10DE200094F70008F0E40008FCDE0008FCDE0008BF
:10DE3000FCDE0008FCDE0008FCDE00080400000038
:10DE400002000000020000000200000002000000CA
:10DE5000D4EB0008E0EB0008A4EB0008ACEB0008F2
:10DE6000CCEB0008D8E80008DCE80008E4E800088B
:10DE700040E80008E4EB0008E8EB000894E900083B
:10DE800094E9000894E90008ECEB0008ECEB0008CA
:10DE9000ECEB0008A4EB0008F0EB000880E20008BF
:10DEA00000EC0008CCEB0008A4EB0008F0EB000845
:10DEB00080E20008CCEB00080CEC000814EC000831
:10DEC0001CEC000820EC000828EC00082CEC0008F2
:10DED00044E80008CCEB00086163746976650000D3
:10DEE0002573256400000000485454502F312E3013
:10DEF00020323030204F4B000D0A0D0A0000000088
:10DF00003C68746D6C3E0D0A000000003C68656161
:10DF1000643E0D0A000000003C7469746C653E00AC
:10DF20003C2F7469746C653E0D0A00003C2F6865D7
:10DF300061643E0D0A0000003C626F64793E0D0A88
:10DF4000000000003C48313E0D0A00003C2F4831E3
:10DF50003E0D0A003C6120687265663D222F00007C
:10DF6000223E00003C2F613E266E6273703B266E9F
:10DF70006273703B0D0A00004D61696E0000000085
:10DF80006E6574776F726B004E6574776F726B009D
:10DF900054656D7065726174757265006C647200B1
:10DFA0004C445200446973706C617900616E696D14
:10DFB0006174696F6E730000416E696D6174696FA1
:10DFC0006E730000616D62696C69676874000000BF
:10DFD000416D62696C6967687400000074696D6501
:10DFE0007273000054696D65727300003C503E000E
:10DFF0003C7472206267636F6C6F723D236630669B
:10E000003066303E0D0A00003C74723E0D0A00007E
:10E010003C74643E000000003C2F74643E0000002D
:10E020003C696E70757420747970653D22746578F2
:10E0300074222069643D220022206E616D653D22BC
:10E0400000000000222076616C75653D2200000012
:10E0500022206D61786C656E6774683D2200000057
:10E06000222073697A653D22000000003C74643E02
:10E070003C627574746F6E20747970653D2273759F
:10E08000626D697422206E616D653D226163746901
:10E090006F6E222076616C75653D22736176650036
:10E0A000223E5365743C2F627574746F6E3E00009F
:10E0B0003C2F74643E0D0A003C7461626C65206202
:10E0C0006F726465723D303E0D0A00003C2F747221
:10E0D0003E0D0A003C74683E3C666F6E7420636FB0
:10E0E0006C6F723D626C75653E0000003C2F666F80
:10E0F0006E743E3C2F74683E0D0A00003C2F746124
:10E10000626C653E3C503E0D0A0000003C62757436
:10E11000746F6E20747970653D227375626D6974D9
:10E1200022206E616D653D22616374696F6E2220ED
:10E1300076616C75653D22003C2F627574746F6E5C
:10E140003E266E6273703B003C2F626F64793E0D19
:10E150000A0000003C2F68746D6C3E0D0A00000040
:10E160003C73656C6563742069643D2200000000A7
:10E17000223E0D0A000000003C2F73656C6563743D
:10E180003E0D0A003C6F7074696F6E2076616C758D
:10E19000653D22002073656C656374656400000052
:10E1A0003C2F6F7074696F6E3E0D0A00266E6273AD
:10E1B000703B3C696E70757420747970653D2263A4
:10E1C0006865636B626F7822206E616D653D220029
:10E1D000222076616C75653D2261637469766522E3
:10E1E00020000000636865636B6564003C696E70C5
:10E1F000757420747970653D2272616E67652220A6
:10E2000069643D220000000022206D696E3D2200FD
:10E2100022206D61783D220022207374796C653D67
:10E220002277696474683A0070783B0022206F6E30
:10E23000696E7075743D22005F6F75747075742E11
:10E2400076616C75653D00002E76616C7565223EC9
:10E25000000000003C6F7574707574206E616D6510
:10E260003D2200005F6F7574707574223E000000DF
:10E270003C2F6F75747075743E0000002E0D0A00FF
:10E2800044656661756C7400313500003C666F72E0
:10E290006D206D6574686F643D224745542220618E
:10E2A0006374696F6E3D222F000000003C2F666F83
:10E2B000726D3E0D0A000000436F6C6F72730000B8
:10E2C0003C74643E0D0A000036340000266E627312
:10E2D000703B266E6273703B266E6273703B0D0A54
:10E2E000000000004C6561726E696E672049522023
:10E2F00072656D6F746520636F6E74726F6C2E2E15
:10E300002E000000537769746368696E6720706F30
:10E31000776572206F6E2E2E2E0000005377697481
:10E320006368696E6720706F776572206F66662E0E
:10E330002E2E00006F66666C696E65004D696E6911
:10E340006D756D206C656E677468206F66206B65F7
:10E3500079206973203130210000000054696D6517
:10E360007365727665722073756363657373667522
:10E370006C6C79206368616E6765642E0000000034
:10E3800053657474696E67206F66206E65772074BC
:10E39000696D65736572766572206661696C656426
:10E3A0002E00000054696D657A6F6E652073756389
:10E3B0006365737366756C6C79206368616E6765FD
:10E3C000642E000053657474696E67206F66206E5A
:10E3D00065772074696D657A6F6E65206661696C1A
:10E3E00065642E0047657474696E67206E657420DD
:10E3F00074696D6500000000446973706C6179692F
:10E400006E672074656D70657261747572652E2E0D
:10E410002E00000053746F726564206D696E696D23
:10E42000756D2076616C756500000000546573742D
:10E43000696E6720646973706C61792E2E2E0000FE
:10E44000536176696E672073657474696E677320B3
:10E450007065726D616E656E746C792E2E2E000083
:10E460006874747020706174683A20272573270DD2
:10E470000A0000006874747020706172616D6574C8
:10E480006572733A20272573270D0A002F000000BC
:10E49000253032642E2530326400000025346400BB
:10E4A0002530326400000000616374696F6E000003
:10E4B0006C6561726E697200706F7765726F6E0065
:10E4C000706F7765726F6666000000007361766535
:10E4D0006461746574696D6500000000796561723E
:10E4E000000000006D6F6E746800000064617900C8
:10E4F0006D696E00736176657469636B65720000A7
:10E50000576F7264436C6F636B00000056657273E3
:10E51000696F6E00454550524F4D000045455052C1
:10E520004F4D2056657273696F6E00005469636BBE
:10E5300065720000506F776572204F6E000000001A
:10E54000506F776572204F66660000004C656172FF
:10E550006E2049522072656D6F746520636F6E7412
:10E56000726F6C00656570726F6D64756D70000020
:10E57000454550524F4D2064756D70003C503E0D26
:10E580000A3C666F6E7420636F6C6F723D677265D4
:10E59000656E3E003C5052453E0000002530347808
:10E5A00000000000202000003C2F5052453E00009B
:10E5B000202020002F6E6574776F726B00000000C2
:10E5C00073617665776C616E00000000776C616E38
:10E5D0006D6F6465000000007373696400000000E3
:10E5E000576F7264436C6F636B204E6574776F7204
:10E5F0006B0000003C423E436F6E6E656374696E53
:10E600006720746F2041636365737320506F696E78
:10E61000742C2074727920616761696E206C61745A
:10E6200065722E3C2F423E003C423E537461746939
:10E630006E672061732041636365737320506F6957
:10E640006E742C2074727920616761696E206C6130
:10E650007465722E3C2F423E0000000073617665A7
:10E6600074696D65736572766572000073617665B5
:10E6700074696D657A6F6E65000000006E65747474
:10E68000696D6500495020616464726573730000B0
:10E6900045535038323636206669726D776172653F
:10E6A00000000000574C414E000000005353494405
:10E6B00000000000266E6273703B266E6273703B32
:10E6C000266E6273703B00004B65790054696D657E
:10E6D000207365727665720054696D65207A6F6E7D
:10E6E000652028474D54202B2900000047657420E1
:10E6F0006E65742074696D65000000003C503E0D2D
:10E700000A3C666F6E7420636F6C6F723D72656455
:10E710003E3C423E000000003C2F423E3C2F666FD4
:10E720006E743E0D0A0000002F74656D7065726195
:10E7300074757265000000007361766574636F72B2
:10E7400072727463000000007361766574636F72A7
:10E750007264733138787800646973706C617974AD
:10E76000656D706572617475726500002E3500000C
:10E77000266465673B430000576F7264436C6F63A8
:10E780006B2054656D706572617475726500000070
:10E790005254432074656D706572617475726500C2
:10E7A000445331387878000054656D7020636F727F
:10E7B00072656374696F6E205254432028756E69C8
:10E7C0007473206F6620302E35B04329000000009E
:10E7D00054656D7020636F7272656374696F6E202B
:10E7E0004453313878782028756E697473206F66C9
:10E7F00020302E35B0432900446973706C61792054
:10E8000074656D7065726174757265002F6C6472E9
:10E81000000000006C64726D696E00006C64726DC3
:10E8200061780000736176656175746F00000000A7
:10E8300025750000576F7264436C6F636B204C4406
:10E84000520000004D696E004D6178004175746F93
:10E850006D61746963206272696768746E65737351
:10E8600000000000536574206173206D696E696D4E
:10E87000756D2076616C756500000000536574202D
:10E880006173206D6178696D756D2076616C756559
:10E89000000000002F646973706C61790000000053
:10E8A0007361766569746973000000007361766551
:10E8B00073796E63616D6269000000007361766553
:10E8C0006272696768746E65737300007361766560
:10E8D000636F6C6F727300007265640067726565C8
:10E8E0006E000000626C7565000000007361766563
:10E8F000646973706C61796D6F64650073617665CE
:10E9000074696E74657276616C000000746573746E
:10E91000646973706C61790073617665616C6C0019
:10E92000576F7264436C6F636B20446973706C61E2
:10E930007900000045532049535400005065726D22
:10E94000616E656E7420646973706C6179206F66A6
:10E95000202245532049535422000000446973701B
:10E960006C6179204D6F646500000000557365206F
:10E97000646973706C617920636F6C6F72730000EF
:10E980004272696768746E6573732028312D313562
:10E99000290000003000000054656D702064697328
:10E9A000706C617920696E74657276616C0000002C
:10E9B0005465737420646973706C617900000000A1
:10E9C0005361766520616C6C000000002F616E69F8
:10E9D0006D6174696F6E730073617665616E696DE8
:10E9E0006174696F6E00000073617665636F6C6FB0
:10E9F00072616E696D6174696F6E000064656600B6
:10EA000073617665616E000073702564000000001C
:10EA100066617625640000007361766563616E004F
:10EA20006373702564000000636465660000000085
:10EA3000576F7264436C6F636B20416E696D6174D4
:10EA4000696F6E7300000000416E696D6174696FDB
:10EA50006E000000436F6C6F7220416E696D6174CF
:10EA6000696F6E00616E25640000000064656625B4
:10EA7000640000003100000063616E256400000046
:10EA800063646566256400002F616D62696C696767
:10EA90006874000073617665616D62696D6F6465AD
:10EAA0000000000073617665616D62696C65647376
:10EAB0000000000073617665616D62696F66667360
:10EAC000657400007361766561616E006173702525
:10EAD000640000006164656600000000576F7264A6
:10EAE000436C6F636B20416D62696C696768740089
:10EAF000234C4544730000004F6666736574206FB5
:10EB000066207365636F6E64203D20300000000056
:10EB1000416D62696C69676874204D6F64650000BF
:10EB200061616E2564000000616465662564000013
:10EB30002F74696D65727300736176656964000096
:10EB4000610000006F000000662564007425640009
:10EB5000576F7264436C6F636B2054696D65727399
:10EB60000000000069642564000000006125640065
:10EB70006F256400682564006D2564004854545076
:10EB80002F312E3020343034204E6F7420466F7574
:10EB90006E640000343034204E6F7420466F756E02
:10EBA000640D0A004E616D650000000056616C75D1
:10EBB0006500000059595959000000004D4D0000F2
:10EBC00044440000686800006D6D00004163746992
:10EBD0006F6E0000574C414E20436C69656E7400A7
:10EBE00041500000470000004200000036330000A2
:10EBF000446563656C65726174696F6E0000000046
:10EC00004661766F7572697465000000536C6F74AD
:10EC10000000000041637469766500004F6E0000DB
:10EC200046726F6D00000000546F0000486F7572EF
:10EC300000000000010000000F00000015000000AF
:10EC4000070000000B000000070000000B000000A0
:10EC5000070000000B0000000F000000140000007F
:10EC6000000000000F000000140000000000000081
:10EC7000010000000000000005000000020000008C
:10EC80000B0000000C0000001A0000000200000051
:10EC90000B000000020000000B000000000000005C
:10ECA000100000001C0000002800000030000000E0
:10ECB0000100000001000000000000000200000050
:10ECC000050000000C000000110000002200000000
:10ECD000050000000C000000050000000C00000012
:10ECE00000000000100000001000000020000000E4
:10ECF00020000000010000000100000000000000F2
:10ED000002000000050000000C00000011000000DF
:10ED100022000000050000000C00000005000000BB
:10ED20000C000000000000000000000000000000D7
:10ED300000000000000000000100000001000000D1
:10ED40000000000003000000050000000C000000AF
:10ED50000F0000001E000000050000000C00000075
:10ED6000040000000B000000000000001000000084
:10ED70001500000025000000250000000100000033
:10ED80000100000000000000322E302E370000008D
:10ED90000D0A57656C636F6D6520746F20576F7235
:10EDA00064436C6F636B204C6F6767657221000072
:10EDB0002D2D2D2D2D2D2D2D2D2D2D2D2D2D2D2D83
:10EDC0002D2D2D2D2D2D2D2D2D2D2D2D0000000027
:10EDD00056657273696F6E3A20000000727463208A
:10EDE0006973206F6E6C696E650000007274632039
:10EDF0006973206F66666C696E6500006565707288
:10EE00006F6D206973206F6E6C696E650000000085
:10EE100063757272656E7420656570726F6D2076B1
:10EE2000657273696F6E3A203078253038780D0A34
:10EE30000000000072656164696E6720697220637A
:10EE40006F6465732066726F6D20656570726F6D9B
:10EE50000000000072656164696E67206469737008
:10EE60006C617920636F6E66696775726174696F32
:10EE70006E2066726F6D20656570726F6D000000A8
:10EE800072656164696E672074696D657365727619
:10EE9000657220646174612066726F6D20656570B3
:10EEA000726F6D0072656164696E67206E69676874
:10EEB000742074696D6572732066726F6D2065656C
:10EEC00070726F6D0000000072656164696E67208A
:10EED00074656D7020636F6E6669677572617469C1
:10EEE0006F6E2066726F6D20656570726F6D0000C9
:10EEF000656570726F6D206973206F66666C696EF0
:10EF0000650000007570646174696E672045455046
:10EF1000524F4D20746F2076657273696F6E20308A
:10EF200078253038780D0A0077726974696E672029
:10EF300076657273696F6E20746F20454550524F2D
:10EF40004D206661696C6564000000007772697429
:10EF5000696E6720495220636F64657320746F2067
:10EF6000454550524F4D206661696C656400000054
:10EF700077726974696E6720636F6E666967207463
:10EF80006F20454550524F4D206661696C656400A5
:10EF900077726974696E672074696D6573657276DE
:10EFA0006572206461746120746F20454550524F32
:10EFB0004D206661696C65640000000077726974B9
:10EFC000696E67206E696768742074696D65206476
:10EFD00061746120746F20454550524F4D20666129
:10EFE000696C65640000000063616C6C696E672089
:10EFF0004952206C6561726E2066756E6374696F2C
:10F000006E0000007573657220627574746F6E20F7
:10F01000707265737365643A20636F6E66696775B5
:10F0200072696E67206573703832363620617320DE
:10F0300061636365737320706F696E740000000014
:10F04000776F7264636C6F636B000000313233342E
:10F050003536373839300000636F6D6D616E643A54
:10F060002073657420646973706C617920636F6CC0
:10F070006F727320746F2025642025642025640D31
:10F080000A000000636F6D6D616E643A20736574F1
:10F0900020616D62696C6967687420636F6C6F7260
:10F0A0007320746F2025642025642025640D0A00D8
:10F0B000636F6D6D616E643A2073657420706F7755
:10F0C0006572202573000000636F6D6D616E643A98
:10F0D0002073657420646973706C6179206D6F644E
:10F0E0006520746F2025640D0A000000636F6D6D4C
:10F0F000616E643A2073657420616D62696C696742
:10F100006874206D6F646520746F2025640D0A009B
:10F11000636F6D6D616E643A2073657420616E6912
:10F120006D6174696F6E206D6F646520746F20254A
:10F13000640D0A00636F6D6D616E643A20736574CF
:10F1400020636F6C6F7220616E696D6174696F6EA0
:10F15000206D6F646520746F2025640D0A00000027
:10F16000636F6D6D616E643A2073686F77207465AC
:10F170006D7065726174757265000000636F6D6D0E
:10F18000616E643A2073657420646973706C617990
:10F19000206272696768746E65737320746F2025CE
:10F1A000642C2064697361626C65206175746D6F95
:10F1B0006D61746963206272696768746E657373E8
:10F1C00020636F6E74726F6C20706572204C4452B5
:10F1D0000D0A0000636F6D6D616E643A2073657493
:10F1E00020616D62696C6967687420627269676822
:10F1F000746E65737320746F2025640D0A0000001F
:10F20000636F6D6D616E643A20656E61626C65203E
:10F210006175746F6D617469632062726967687487
:10F220006E65737320636F6E74726F6C0000000004
:10F23000636F6D6D616E643A2064697361626C65C1
:10F24000206175746F6D61746963206272696768AB
:10F25000746E65737320636F6E74726F6C00000060
:10F26000636F6D6D616E643A2073657420646973B9
:10F27000706C617920666C61677320746F203078E0
:10F280002530327800000000636F6D6D616E643A66
:10F2900020737461727420646973706C6179207476
:10F2A00065737400636F6D6D616E643A207365748D
:10F2B0002074696D6520746F202573202534642DBA
:10F2C000253032642D2530326420253032643A25D1
:10F2D0003032643A253032640D0A0000636F6D6D80
:10F2E000616E643A207374617274206E6574207468
:10F2F000696D65207265717565737400636F6D6DFE
:10F30000616E643A206C6561726E20495220636FB1
:10F3100064657300636F6D6D616E643A207361762E
:10F320006520646973706C61792073657474696EAB
:10F3300067730000636F6D6D616E643A207072696F
:10F340006E74207469636B65723A202725732700F9
:10F350006C64723A206F6C64206272696768746EC4
:10F3600065733A202564206E65772062726967684C
:10F37000746E6573733A2025640D0A0065737038E6
:10F38000323636206E6F77207570000065737038E6
:10F39000323636206E6F77206F6E6C696E650000B6
:10F3A000202049502025730064636637373A2025B2
:10F3B00073202534642D253032642D2530326420AD
:10F3C000253032643A253032643A253032640D0AF1
:10F3D0000000000072656164207274633A20257336
:10F3E000202534642D253032642D253032642025CB
:10F3F0003032643A253032643A253032640D0A00E6
:10F40000466F756E642054696D65723A20257320CD
:10F41000617420253032643A253032640D0A0000D0
:10F42000676F742074656D706572617475726520A4
:10F4300066726F6D20445331387878783A202564AD
:10F4400025730D0A00000000676F742074656D70ED
:10F45000657261747572652066726F6D20525443D7
:10F460003A20256425730D0A000000006E6F207499
:10F47000656D706572617475726520617661696C25
:10F4800061626C65000000007570646174652064E1
:10F490006973706C6179000049524D503A20504FA9
:10F4A000574552206B65790049524D503A204F4BD9
:10F4B000206B65790000000049524D503A20646588
:10F4C0006372656D656E7420646973706C61792018
:10F4D0006D6F64650000000049524D503A20696E1E
:10F4E0006372656D656E7420646973706C617920F8
:10F4F0006D6F64650000000049524D503A2064650C
:10F500006372656D656E7420616E696D6174696F9B
:10F510006E206D6F6465000049524D503A20696E4F
:10F520006372656D656E7420616E696D6174696F7B
:10F530006E206D6F6465000049524D503A2064653D
:10F540006372656D656E7420686F757200000000EF
:10F5500049524D503A20696E6372656D656E742034
:10F56000686F75720000000049524D503A20646582
:10F570006372656D656E74206D696E7574650000EB
:10F5800049524D503A20696E6372656D656E742004
:10F590006D696E757465000049524D503A2064657E
:10F5A0006372656D656E742072656420627269674E
:10F5B00068746E657373000049524D503A20696E4D
:10F5C0006372656D656E742072656420627269672E
:10F5D00068746E657373000049524D503A2064653B
:10F5E0006372656D656E7420677265656E20627208
:10F5F000696768746E6573730000000049524D506E
:10F600003A20696E6372656D656E74206772656518
:10F610006E206272696768746E6573730000000023
:10F6200049524D503A2064656372656D656E742071
:10F63000626C7565206272696768746E65737300C9
:10F6400049524D503A20696E6372656D656E742043
:10F65000626C7565206272696768746E65737300A9
:10F6600049524D503A2064656372656D656E742031
:10F670006272696768746E657373000049524D5019
:10F680003A20696E6372656D656E74206272696797
:10F6900068746E657373000049524D503A20676577
:10F6A000742074656D706572617475726500000018
:10F6B000706F7765725F696E697428292063616C69
:10F6C0006C656400737769746368696E6720706F36
:10F6D000776572206F6E0000737769746368696E76
:10F6E0006720706F776572206F66660020206765FF
:10F6F000742074656D7065726174757265000000C8
:10F700002020706F776572206F66662F6F6E000025
:10F7100020206F6B00000000202064656372656D1F
:10F72000656E7420646973706C6179206D6F6465B7
:10F73000000000002020696E6372656D656E7420A4
:10F74000646973706C6179206D6F646500000000FE
:10F75000202064656372656D656E7420616E696DED
:10F760006174696F6E206D6F646500002020696EA2
:10F770006372656D656E7420616E696D6174696F29
:10F780006E206D6F64650000202064656372656D96
:10F79000656E7420686F7572000000002020696E2D
:10F7A0006372656D656E7420686F7572000000008D
:10F7B000202064656372656D656E74206D696E7579
:10F7C000746500002020696E6372656D656E74203B
:10F7D0006D696E7574650000202064656372656DE7
:10F7E000656E7420726564206272696768746E6504
:10F7F000737300002020696E6372656D656E7420FE
:10F80000726564206272696768746E657373000064
:10F81000202064656372656D656E7420677265652E
:10F820006E206272696768746E6573730000000011
:10F830002020696E6372656D656E74206772656500
:10F840006E206272696768746E65737300000000F1
:10F85000202064656372656D656E7420626C7565E9
:10F86000206272696768746E657373002020696E28
:10F870006372656D656E7420626C75652062726975
:10F880006768746E65737300202064656372656DCC
:10F89000656E7420676C6F62616C20627269676864
:10F8A000746E6573730000002020696E6372656D6D
:10F8B000656E7420676C6F62616C20627269676844
:10F8C000746E6573730000002020746F67676C6549
:10F8D000206175746F206272696768746E657373F6
:10F8E0000000000020205468616E6B20796F752144
:10F8F000000000003139322E35332E3130332E31B5
:10F90000303300004E65772074696D657A6F6E65DF
:10F910003A2025640D0A000043000000F801002091
:10F920001F0000001C0000001F0000001E0000005F
:10F930001F0000001E0000001F0000001F0000004C
:10F940001E0000001F0000001E0000001F0000003D
:10F950001F0000001D0000001F0000001E0000002E
:10F960001F0000001E0000001F0000001F0000001C
:10F970001E0000001F0000001E0000001F0000000D
:10F980006D0100006E010000232D302B2000686CFB
:10F990004C006566674546470030313233343536B2
:10F9A00037383941424344454600303132333435EB
:10F9B0003637383961626364656600002020202094
:10F9C000202020202028282828282020202020200F
:10F9D00020202020202020202020202088101010EF
:10F9E0001010101010101010101010100404040447
:10F9F00004040404040410101010101010414141BC
:10FA00004141410101010101010101010101010126
:10FA100001010101010101101010101010424242B9
:10FA200042424202020202020202020202020202F6
:10FA30000202020202020210101010200000000058
:10FA400000000000000000000000000000000000B6
:10FA500000000000000000000000000000000000A6
:10FA60000000000000000000000000000000000096
:10FA70000000000000000000000000000000000086
:10FA80000000000000000000000000000000000076
:10FA90000000000000000000000000000000000066
:10FAA0000000000000000000000000000000000056
:10FAB0000000000000000000000000000000000046
:08FAC0008006FF7F0100000039
:10FAC80030BD000818BD000834BD000838BD000866
:10FAD8003CBD000828BD00082CBD0008FF00000040
:10FAE800FF000000E803000001000000D0C2000889
:10FAF80000000000000000000000000004E500080D
:10FB0800000000000000000000000000D8C200084B
:10FB180000000000000000000000000074C200089F
:10FB280004000000040000000100000020000000A4
:10FB380020000000030000006CC20008E10F00086C
:10FB48000200000002000000000000007CC2000863
:10FB58005510000804000000040000000300000025
:10FB680084C20008111B0008020000000200000007
:10FB7800030000008CC20008C5180008020000003D
:10FB8800020000000300000094C20008390D0008BC
:10FB98000200000002000000000000009CC20008F3
:10FBA800FD1D000802000000020000000300000024
:10FBB800A4C2000815180008040000000400000092
:10FBC80003000000B0C20008591600080200000037
:10FBD8000200000003000000B8C200085521000818
:10FBE800030000000300000003000000C0C200087A
:10FBF8008114000802000000020000000300000059
:10FC0800C8C2000801130008040000000400000036
:10FC1800030000000F0000002000000001000000A9
:10FC280020000000160000003C0000000500000055
:10FC38006CC2000801000000010000000000000084
:10FC480074C2000804000000040000000100000065
:10FC5800050000000F00000001000000FFFF000089
:10FC6800FFFF0000D80E0000FF000000FF000000AA
:10FC7800FFFFFFFFFF000000010000003139322EB6
:10FC880035332E3130332E31303300000000000080
:10FC98000204060800000000010203040102030434
:10FCA8000607080900000000000000000102030424
:10FCB8000607080900A24A0400000000000000002E
:10FCC800000000000000000000000000000000002C
:10FCD800000000000000000018F900080000000003
:10FCE800000000000000000000000000000000000C
:10FCF80000000000000000000000000000000000FC
:10FD080000000000000000000000000000000000EB
:10FD18000000000000000000F8010020BBF9000806
:10FD280001000000000000004A0000000000000080
:10FD380000000000000000000000000000000000BB
:10FD4800000000004A000000000000000000000061
:10FD5800000000000000000000000000000000009B
:08FD680011010008ED00000884
:0400000508000000EF
:00000001FF
